:020000040800F2
:10000000F0FF001019C7050841E1000865A20408C7
:10001000B9C70508B9C70508B9C705080000000039
:100020000000000000000000000000003DE10008AA
:1000300039E100080000000035E100081163040800
:10004000B9C70508B9C70508B9C70508B9C705087C
:10005000B9C70508B9C7050805B3040831B40408D1
:10006000F5B30408B9B304087DB304080DAE050860
:10007000FDAD0508EDAD0508DDAD0508C9AD050808
:10008000B5AD0508A1AD0508B9C70508B9C705088C
:10009000B9C70508B9C70508B9C7050841B30408B9
:1000A000F94D0408794E0408E94D04089D4E0408F2
:1000B0006D4E04085D4E04084D4E04088DB60508CB
:1000C00095B6050881B6050889B60508B9C70508BB
:1000D000B9C705082167040865660408A96504080E
:1000E000C9B20408B9C70508250B0108D94D040891
:1000F000094E0408C94D04082D4E04088DAD0508AD
:10010000B9C70508B9C705083D4E0408B9C70508B1
:10011000ED6404083164040879D8030889D703081A
:1001200079AD050865AD050851AD05083DAD05087B
:1001300029AD0508B9C70508B9C70508B9C7050835
:10014000B9C70508B9C70508B9C70508C5DA000861
:1001500015AD050801AD0508EDAC0508756304088B
:1001600075B605087DB60508B9C70508B9C70508FD
:10017000B9C70508B9C70508B9C70508B9C705084B
:08018000B9C70508B9C705085D
:08018800C8C2050001000000DF
:100190000E02010002000000705400208454002070
:1001A0000000000010090008051001000600000012
:1001B000FC530020885400200000000012090008B1
:1001C000130201000400000094220020905400203B
:1001D00000000000180900080D1001006400000074
:1001E0002053002094540020000000001DFE03084E
:1001F000040008008000000060520020F854002035
:1002000000000000000000000902010001000000E1
:100210000852002078550020000000001C0900084A
:10022000FB01010001000000A05100207C550020CE
:1002300000000000F5570508FC010100090000005E
:100240006C50002080550020000000000558050873
:10025000F701010006000000605000208C550020CE
:10026000000000001E090008F90101000400000060
:100270005C5000209455002000000000C1330408A9
:100280000A8001002800000034500020985500200A
:100290000000000021090208160215003F000000BE
:1002A000D4260020C055002000000000D1580508C9
:1002B0003400010010000000604F002000560020B4
:1002C00000000000999402081102010008000000DB
:1002D000384F0020105600200000000024090008BC
:1002E0001212010004000000304F002018560020B8
:1002F000000000002C090008182001003200000056
:10030000FC4E00201C56002000000000415905084A
:10031000FF11010006000000C04E002050560020D2
:1003200000000000AD490508081203000F0000009E
:10033000CC4E00205856002000000000F14905086E
:10034000061001001C000000B8260020685600209E
:100350000000000021580508FD01010021000000F7
:10036000FC470020845600200000000017330408DA
:1003700012200100110000007C450020A85600203A
:100380000000000030090008000201000B0000001E
:10039000B8420020BC560020000000000000000011
:1003A0000202010003000000B0260020C856002011
:1003B00000000000000000000C020100040000002A
:1003C00090260020CC56002000000000C9490508F6
:1003D000FE01010014000000183D0020D05600204E
:1003E000000000003549050823120100100000003C
:1003F00058850020FC890020000000004409000806
:10040000371001002E000000A88900200C8A00206F
:10041000000000005409000816100100060000004A
:10042000508500203C8A002000000000820900085E
:100430002F10010022000000D8890020448A0020EB
:1004400000000000880900081E00010009000000EB
:1004500088830020688A002000000000AA090008A4
:10046000F581010068000000E0820020748A00200D
:100470000000000007170108232001001000000001
:1004800034860020DC8A002000000000350A0208C3
:10049000FD070100760000001E820020EC8A00208B
:1004A00000000000DD160108261001000E0000000B
:1004B000748B0020648B0020000000005915010897
:1004C0000B3001001A00000004820020B48B0020D1
:1004D00000000000B40900081F30010024000000E3
:1004E0001C840020D08B002000000000D0090008F0
:1004F000050201000400000000860020F48B0020AB
:1005000000000000F4090008030101000A000000D7
:10051000A0830020F88B0020000000005511010886
:100520000EF003009E010000409E0020A4A70020C2
:100530000000000075900208130001000400000094
:1005400078A7002044A9002000000000F809000856
:100550000101010004000000809D002048A9002046
:100560000000000000000000000101000400000085
:10057000789D00204CA9002000000000FC09000824
:100580000201010003000000749D002050A900201A
:1005900000000000B9CF0308220201001C01000086
:1005A00040A5002054A9002000000000895805083B
:1005B0000C200600CC00000004A0002070AA00203F
:1005C000000000007DCF0308010201000B000000C5
:1005D0008C9D00203CAB002000000000E149050894
:1005E0001B02010010000000E0A3002048AB002027
:1005F00000000000594A05081B1001000C00000013
:10060000888D002058AB002000000000DDA3010809
:1006100021020100F00000000C8C002064AB0020DF
:1006200000000000C5A201082C000400100000001A
:10063000DCB80020CCB8002000000000D51B020868
:100640002B0012002400000010B90020ECB800209C
:1006500000000000A91B02082920140078000000F7
:1006600054B7002034B90020000000000000000052
:10067000F62101000C00000060B50020ACB900209C
:1006800000000000000A00081C0202001C0000001C
:1006900004B50020FCB9002000000000655A0508E0
:1006A000282001001800000020B5002018BA002002
:1006B00000000000152202081400010004000000E0
:1006C000ECB4002030BA0020000000000C0A000842
:1006D000012001000C00000058AC002034BA0020BA
:1006E00000000000100A00081900010005000000C9
:1006F00080BF00209CC00020000000001C0A0008F1
:100700001A0001000E00000008BF0020A4C0002055
:1007100000000000220A0008203201000A00000048
:10072000D4BD0020B4C00020000000005190020899
:1007300015001000700000006CBB0020C0C000203D
:1007400000000000000000002A0008006000000017
:10075000C8BF002030C1002000000000299002081E
:100760000A0201001400000068C4002088C70020AD
:1007700000000000A5D003080300010001000000F4
:100780001CC400209CC700200000000000000000E6
:10079000031201003D00000048C70020A0C7002050
:1007A00000000000300A000825201E002C01000077
:1007B000B0C40020E0C700200000000000000000DE
:1007C0001010010002000000C8C300200CC9002066
:1007D000000000006E0A0008F82101000600000079
:1007E000FCC3002010C9002000000000700A0008AF
:1007F000020001000C00000044CA0020D8CA0020FA
:10080000000000000000000029020100400000007C
:100810007CC90020E4CA002000000000760A00081D
:10082000280204000400000060CF002034D1002022
:1008300000000000554A05082702040004000000DB
:100840005CCF002038D1002000000000494A050894
:100850001F02080010000000A0CC00203CD10020A6
:1008600000000000654905081A0201003C00000074
:1008700064CC00204CD1002000000000D9590508AC
:1008800038100100010000005CCB002088D100205E
:1008900000000000B60A0008270001000400000064
:1008A00010D2002014D2002000000000B80A000876
:1008B0001002010001000000BCEA0020B8EA00209C
:1008C00000000000BC0A000807020100020000004E
:1008D000A0EA0020C0EA002000000000BE0A0008D4
:1008E0001D0202000600000080EA0020C4EA002089
:1008F0000000000000000000060203000C000000E1
:1009000088EA0020CCF3002000000000B55905085B
:1009100000002000020100000000013D00003F0136
:10092000000000000000000001010101FFFFFFFFC7
:10093000000000010000054D46345300000800028D
:1009400000000000000000000000000000000000A7
:100950000000000020003200C800D00796001400FC
:10096000320028004C0440060005500014000F001F
:10097000080064000100010005000A000000F40105
:100980009600C409000019000000000000000000EB
:100990000000000000000000000000000000000057
:1009A0000000000000000000000000050100000041
:1009B00000000000AE014A015E012C01640101004B
:1009C000000001000A019A01001E0A000002000056
:1009D000000000000001000000050000010203000B
:1009E0000000000000000000000000000000000007
:1009F000008007000000000048044430B3000000FD
:100A000000000000010000000202000003000023BB
:100A1000E8036400040A000114001E00000028011D
:100A200000007E05EA05B4053200E803D0070000A7
:100A300000000000000000000000000000000000B6
:100A400000000000000000000000000000000000A6
:100A50000000000000000000000000000000000096
:100A60000000000000000000000000000100000580
:100A70000101F4011400000000000000000000006B
:100A80000000000000000000000000000000000066
:100A90000000000000000000000000000000000056
:100AA0000000000000000000000000000000000046
:100AB0000000000000000000200300000000003CD7
:100AC0000403090412010002EF02014083045632BC
:100AD00000020102030100001201000202020040B4
:100AE0008304405700020102030100001A030000C2
:100AF00000000000000000000000000000000000F6
:100B000000000000000000000403090412010002BC
:100B1000000000408304205700020102030100008E
:100B200009022000010104C0320904000002080685
:100B30005005070581024000000705010240000042
:100B400009026400030100C032090400000103002F
:100B50000000092111010001223600070583030965
:100B6000000A080B0102020201000904010001024F
:100B700002010005240010010524010002042402E2
:100B8000020524060102070582030800FF0904028A
:100B900000020A000000070501024000000705816D
:100BA0000240000009024300020100C032090400B3
:100BB00000010202010005240010010524010001CA
:100BC000042402020524060001070582030800FF31
:100BD00009040100020A00000007050102400000AC
:100BE0000705810240000000FF000000080000002F
:100BF00000600240106002400000000000000000A1
:100C0000000B0000000000000000000000000000D9
:100C10000060024028600240010000000000000067
:100C2000060C0000000000000000000000000000B2
:100C3000006002404060024002000000000000002E
:100C4000100D000000000000000000000000000087
:100C500000600240586002400300000000000000F5
:100C6000160E000000000000000000000000000060
:100C700000600240706002400400000000000000BC
:100C8000200F000000000000000000000000000035
:100C90000060024088600240050000000000000083
:100CA000261000000000000000000000000000000E
:100CB00000600240A060024006000000000000004A
:100CC00030110000000000000000000000000000E3
:100CD00000600240B8600240070000000000000011
:100CE000362F00000000000000000000000000009F
:100CF0000064024010640240000000000000000098
:100D000000380000000000000000000000000000AB
:100D1000006402402864024001000000000000005E
:100D20000639000000000000000000000000000084
:100D30000064024040640240020000000000000025
:100D4000103A000000000000000000000000000059
:100D500000640240586402400300000000000000EC
:100D6000163B000000000000000000000000000032
:100D700000640240706402400400000000000000B3
:100D8000203C000000000000000000000000000007
:100D9000006402408864024005000000000000007A
:100DA00026440000000000000000000000000000D9
:100DB00000640240A0640240060000000000000041
:100DC00030450000000000000000000000000000AE
:100DD00000640240B8640240070000000000000008
:100DE0003646000000000000000000000000000087
:100DF0007D00000001820008FD810008F9810008E3
:100E0000ED810008E9810008F5810008F181000802
:100E100085A30008958D00085D860008ADFF0008D9
:100E200029000108C5010108ED830008B18300080D
:100E3000A9830008010000000000803F3D46010832
:100E40009948010825410108A90C0108FD4701083E
:100E5000B90C0108D50C01089D8400088D84000898
:100E6000000000000000000015FF000819FE000847
:100E700005FF00083D820008B1FE000859FE000889
:100E800039820008F4050020019A0008E199000861
:100E90006D08010800000000000000001D98000817
:100EA000399700080000000000000000000000006A
:100EB00039840008C5820008B98200083999000801
:100EC00055990008718200081D99000801990008D1
:100ED00005010905A101A100050109300931093207
:100EE000093309350934093609371581257F750815
:100EF00095088102050919012908150025019508A1
:100F000075018102C0C0000009022200010100E059
:100F1000320904000001030102000921110100014E
:100F20002236000705830309000A00000080020240
:100F30001F00000053544D202020202050726F6469
:100F4000757420202020202020202020302E3031B9
:100F500000FF0000000000000000AA55070100008B
:100F60000101AA55050100007EFF0000FFFFFFFF01
:100F70000800000050070608FF1FFF1F00000000C8
:100F80000102030401020304060708092D202D2D88
:100F9000202D2D2D2D202D2D2D2D000000000000A9
:100FA0000000000000000000000000AA550B010036
:100FB00000AA5505010000AA550902000000AA5523
:100FC00003009F0001000000C0120000AC8B002055
:100FD00000000000848B002000000000987D0608BF
:100FE000147D06080000000025D00308A08601003B
:100FF00004000000000000000000000000000000ED
:1010000000000000000000000000000000000000E0
:10101000000000000000000000000000987D0608AD
:10102000A07D06080000000051440408E803000009
:1010300004000000000000000000000000000000AC
:1010400000000000000000000000000000000000A0
:10105000000000000000000000000000A87D06085D
:1010600000000000000000006D3F03087D0000004C
:10107000FF00000000000000000000000000000071
:101080000000000000000000000000000000000060
:1010900000000000000000000000000014F8060836
:1010A0000000000000000000014E03087D00000069
:1010B000FF00000000000000000000000000000031
:1010C0000000000000000000000000000000000020
:1010D000000000000000000000000000D08D0608A5
:1010E0000000000000000000996803087D00000077
:1010F000FF000000000000000000000000000000F1
:1011000000000000000000000000000000000000DF
:10111000000000000000000000000000B07D060894
:101120000000000000000000B53A0408E8030000D9
:1011300003000000000000000000000000000000AC
:10114000000000000000000000000000000000009F
:10115000000000000000000000000000B47D060850
:1011600000000000000000005D00030810270000E0
:10117000030000000000000000000000000000006C
:10118000000000000000000000000000000000005F
:101190000000000000000000000000001CF4060831
:1011A00000000000BD170208C9A204085F76000015
:1011B000050000000000000000000000000000002A
:1011C000000000000000000000000000000000001F
:1011D000000000000000000000000000B8F7060852
:1011E0000000000000000000CDBC04081027000033
:1011F00001000000000000000000000000000000EE
:1012000000000000000000000000000000000000DE
:10121000000000000000000000000000C07D060883
:101220000000000000000000AD310408E8030000E9
:1012300005000000000000000000000000000000A9
:10124000000000000000000000000000000000009E
:10125000000000000000000000000000CC7D060837
:101260000000000000000000E5D20308204E00004E
:10127000030000000000000000000000000000006B
:10128000000000000000000000000000000000005E
:10129000000000000000000000000000DC7D0608E7
:1012A0000000000000000000E1D00308204E000014
:1012B000030000000000000000000000000000002B
:1012C000000000000000000000000000000000001E
:1012D000000000000000000000000000EC7D060897
:1012E0000000000000000000C9400408400D030099
:1012F00003000000000000000000000000000000EB
:1013000000000000000000000000000000000000DD
:10131000000000000000000000000000FC7D060846
:10132000000000000000000055FF03081027000027
:1013300001000000000000000000000000000000AC
:10134000000000000000000000000000000000009D
:10135000000000000000000000000000407D0608C2
:10136000000000000000000025B001081027000068
:10137000030000000000000000000000000000006A
:10138000000000000000000000000000000000005D
:10139000000000000000000000000000047E0608BD
:1013A0000000000000000000D95D0208A0860100D6
:1013B000010000000000000000000000000000002C
:1013C000000000000000000000000000000000001D
:1013D0000000000000000000000000000C7E060875
:1013E00000000000000000003539040850C3000070
:1013F00001000000000000000000000000000000EC
:1014000000000000000000000000000000000000DC
:10141000000000000000000000000000147E06082C
:10142000000000000000000019350408A861000059
:1014300001000000000000000000000000000000AB
:10144000000000000000000000000000000000009C
:10145000000000000000000000000000207E0608E0
:1014600000000000000000006D020208A0860100DC
:10147000010000000000000000000000000000006B
:10148000000000000000000000000000000000005C
:101490000000000000000000000000002C7E060894
:1014A0000000000000000000C96B0408A00F00004D
:1014B000010000000000000000000000000000002B
:1014C000000000000000000000000000000000001C
:1014D000000000000000000000000000387E060848
:1014E0000000000000000000D9FC010810270000E7
:1014F00001000000000000000000000000000000EB
:1015000000000000000000000000000000000000DB
:10151000000000000000000000000000447E0608FB
:101520000000000000000000098501081A410000C9
:1015300001000000000000000000000000000000AA
:10154000000000000000000000000000000000009B
:10155000000000000000000000000000487E0608B7
:1015600000000000000000008D110108102700009D
:10157000010000000000000000000000000000006A
:10158000000000000000000000000000000000005B
:10159000000000000000000000000000287D060898
:1015A00000000000000000009940020850C3000045
:1015B000010000000000000000000000000000002A
:1015C000000000000000000000000000000000001B
:1015D000000000000000000000000000547E06082B
:1015E000000000000000000065220108400D03001B
:1015F00000000000000000000000000000000000EB
:1016000000000000000000000000000000000000DA
:101610000000000000000000000000005C7E0608E2
:10162000000000000000000061D00308400D03002E
:1016300000000000000000000000000000000000AA
:10164000000000000000000000000000000000009A
:10165000000000000000000000000000647E06089A
:1016600000000000000000003DE4010850C300003D
:101670000300000000000000000000000000000067
:10168000000000000000000000000000000000005A
:10169000000000000000000000000000707E06084E
:1016A000000000000000000089DC030840420F0039
:1016B000000000000000000000000000000000002A
:1016C000000000000000000000000000000000001A
:1016D0000000000000000000000000007C7E060802
:1016E00000000000000000004DD7030850C30000B8
:1016F00000000000000000000000000000000000EA
:1017000000000000000000000000000000000000D9
:1017100000000000000000000000000001000000C8
:1017200000000100E00101FF01000000419A0108F2
:1017300000000000000000005C0906080000000036
:101740000000000000000000C00F060800000000BC
:1017500000000000000000006C0F060808000000F8
:101760000000000000000000CDCA01084FA40020C6
:101770000101FF00FFFFFFFF85F2010800000000EC
:101780000000000094100608B1F5010800000000F8
:10179000000000004C1006082D202D2D202D2D2D91
:1017A0002D202D2D2D000000000000000000000065
:1017B0000000000000000000000000000000000029
:1017C0000000000008100608AC8500209CFF2C01DA
:1017D00000000000F0A60020E0150C17000000003B
:1017E0004DA400200200000040100608689D002063
:1017F00088136F17010000006A9D002088136F177F
:1018000000000000EE530020000000000000000077
:10181000EC5300200000000000000000EA5300200C
:101820000000000000000000E8530020000000005D
:1018300000000000E653002000000000000000004F
:10184000E45300200000000000000000900600208B
:101850000000000000000000F19C002003000000D8
:1018600030110608609D002088136F1701000000EA
:10187000F685002088136F1700000000019B010807
:101880000000000000000000401106084EA40020E7
:101890000100000094110608F885002001000000F6
:1018A000A0110608EE85002002000000A81106081D
:1018B000000000000000000000000000B411060855
:1018C000E99A01080000000000000000501206081C
:1018D000000000000000000000000000A412060844
:1018E00000000000000000000000000014130608C3
:1018F0006C9D0020020000004C130608F2850020B9
:10190000E0150C170000000000AE002054AE0020CF
:1019100001000000000000000000000000000000C6
:101920000C290608D601FF00FFFFFFFFC5DA0108FA
:1019300000000000000000009C28060801000000D4
:10194000FA0000000100000001000000010000009A
:10195000000101010000000020A100200000F401AE
:10196000010000001EA100200000F40101000000A1
:101970001CA100200000F401010000001AA10020B9
:101980000000F4010100000018A100200000F40193
:101990000100000016A100200000F4010100000079
:1019A00014A100200000F4010100000045A201087C
:1019B00009A20108000000006015060804A100202B
:1019C0000532010012A100206400F40101000000B2
:1019D00010A100206400C4090100000002A1002041
:1019E000E803D0070100000000A10020E803D007B1
:1019F00001000000FEA00020E803D0070100000065
:101A0000FCA000201E00B80B010000000AA100206D
:101A100005000F00010000000CA1002003000A00D7
:101A200001000000FAA000201E00F40101000000E7
:101A30000EA1002002000000EC150608F8A000200E
:101A4000140064000100000006A100203200E80339
:101A500001000000F6A000200000C8000100000006
:101A600001A0002000C8010000A0002000500100DB
:101A7000FF9F0020005A0100FD9F0020020000008F
:101A8000F81506083085060838850608AA53002090
:101A90000100C40900000000A85300200100C4098F
:101AA00000000000A65300200100C409000000004F
:101AB000A45300200100C40900000000A05300202E
:101AC0000100C40900000000A25300200100C40965
:101AD000000000009E5300200100C4090000000027
:101AE0009C5300200100C40900000000AB9D0020B1
:101AF00000C80100AA9D002000C80100A89D002088
:101B00000000FFFF0A000000A69D00200100C800A1
:101B100001000000A49D002032003075320000005A
:101B2000A29D002005820500A09D002005002C013B
:101B3000050000009F9D0020055A05009C9D002087
:101B400000FF01009E9D0020020000004C110020BB
:101B50009A9D002003000000200406089B9D0020A1
:101B600000FF01009D9D0020020000004C1100209C
:101B7000999D0020030000002004060899A1010897
:101B800029A10108000000000416060868AC002026
:101B9000EE02CA080100000066AC002000C8010087
:101BA0006400000065AC002000C801006400000073
:101BB00064AC00200200000010170608869D00207B
:101BC0000000803E05000000849D002080C1803E12
:101BD000050000007E9D00200083007D05000000C0
:101BE0007C9D002080C1803E05000000779D002084
:101BF00000FF0100709D00206400F401010000005E
:101C00006E9D0020040000001C1706086D9D00203A
:101C10000200000030170608319E00200D00000071
:101C20003C1706082E9E0020006401002C9E002018
:101C3000320010270A0000002A9E00200D0000003C
:101C40003C170608299E00200D0000003C170608DE
:101C5000289E002002000000741706086EAC0020C9
:101C60003E000000801706086CAC00200100FF7FDA
:101C7000010000006BAC0020020000007C18060888
:101C8000339E0020030000008C180608329E0020BE
:101C9000030000008C180608EE9F0020000A0100D7
:101CA000EC9F00200000E80301000000EA9F0020F4
:101CB0000000E80301000000E89F00200000E803A6
:101CC00001000000E69F00200000E8030100000082
:101CD000DE9F00200000E80301000000E49F0020D8
:101CE0000000E80301000000E29F00200000E8037C
:101CF00001000000E09F002000140100FC9F002074
:101D0000020000009C180608FA9F00200000F40161
:101D100001000000F89F00200000F4010100000015
:101D2000F69F00200000F40101000000F49F002055
:101D30000000F40101000000F29F00200000A00F4D
:101D400001000000F09F00200000A00F0100000033
:101D5000E3A0002019640100E2A0002002000000BE
:101D6000A8180608E0A00020E803D0070A00000039
:101D7000DEA00020006401000A000000D3A00020C3
:101D800000640100D2A0002000640100DAA000205D
:101D9000006401000A000000D9A0002000640100D6
:101DA0000A000000D8A00020006401000A00000022
:101DB000DDA0002000FF01000A000000DCA00020E0
:101DC00000FF01000A000000DBA0002000FF01006E
:101DD0000A000000D7A0002001FF01000A00000057
:101DE000D6A0002001FF01000A000000D5A00020BD
:101DF00001FF01000A0000003C9E00200000F401E9
:101E0000010000003A9E00200000A00F0100000029
:101E1000389E00200000A00F01000000369E002028
:101E20000000A00F01000000349E00200000A00F61
:101E30000100000097A4002000C8010096A4002023
:101E40000064010095A400200064010094A4002017
:101E50000064010093A400200064010092A400200B
:101E6000FF08010091A400200164010091A0010875
:101E700055A0010800000000B41806089AA400202C
:101E80000132010099A40020010000002419060875
:101E900098A40020040000002C19060890A400203B
:101EA000006401008EA400201400E803010000007B
:101EB0008CA40020E80330750A0000008BA40020E9
:101EC00000C801008AA4002000C8010089A40020E5
:101ED00000C8010088A40020003201009CA400205A
:101EE000004B01009BA400200400000040190608DC
:101EF00087A40020006401000A000000AAA40020BA
:101F00000000D00701000000A5A4002000C80100C7
:101F1000A4A4002000C80100A3A4002000C8010060
:101F2000A8A400200000D00701000000A2A4002007
:101F300000C80100A1A4002000C80100A0A4002046
:101F400000C80100A6A400200000D0070100000086
:101F50009FA4002000C801009EA4002000C801002A
:101F60009DA4002000C80100399E0108219E01089F
:101F70000000000054190608259E0020005A0100A8
:101F8000249E002000C80100229E0020E803D00704
:101F9000010000000000000000000000FD1D02081C
:101FA000F01906084D4154454B4634303553450031
:101FB000989D002000030100979D00200003010070
:101FC0005D9D0108119D010800000000441A0608EB
:101FD000D19C0108899C010800000000E01A060855
:101FE000A99D0108A9DA010800000000601B06088D
:101FF000889D0020010301006508020849080208C5
:1020000000000000B81E06080D9C0108C19B0108D5
:1020100000000000281F0608499E010891010208DF
:1020200000000000C41F0608CD1E02088108020837
:10203000000000006C200608A99E010800000000B6
:1020400000000000EC200608859F01082D9F010874
:10205000000000005021060819A00108DD9F0108BA
:1020600000000000F821060839070208CDA0010889
:102070000000000084220608F5A0002001060100EF
:10208000F19E0108BD9E01080000000080230608A3
:102090006D06020845DC010800000000F023060878
:1020A000810702080DDD0108000000004025060838
:1020B000F4A0002001030100F19D0108C19D010869
:1020C0000000000014260608658A020800000000CF
:1020D0000000000078260608599C010891DA0108E2
:1020E00000000000F82606080000000000000000C4
:1020F000000000008427060801A1010885DD010811
:1021000000000000F4270608FFFFFFFF0000803FEB
:1021100000000000000000000000000000000000BF
:1021200000000000000000000000000000000000AF
:10213000000000000000803F0000000000000000E0
:10214000000000000000803F0000000000000000D0
:10215000000000000000803F0000000000000000C0
:1021600000000000010000000000FA430000FA43F4
:102170000000803F6501040800000000000000002E
:1021800000000000FFFFFFFFFF0000000000000054
:1021900034CB0020080000000000000024CB002009
:1021A00008000000C5990008819A0008050B010885
:1021B000000000008984000855900008719800080C
:1021C000C98F0008000000000000000045840008DE
:1021D0001182000805820008C9980008E5980008E7
:1021E000AD98000891980008759800087D9900083E
:1021F0005D9A0008510A0108000000005D84000893
:10220000CD8F000845980008258F000800000000C9
:102210000000000051840008685E0C00020100000C
:10222000A00F0000B80B00000102FFFF010000003A
:10223000FFFF000010F40608000008020503030079
:102240000000000018F4060801000802050403005D
:1022500000000000E4A006080200FE0101100300D7
:10226000000000008088060803001402000300003C
:102270000000000020F4060804001F02020008000D
:102280000000000028F4060805001F0202010800F3
:1022900000000000FFFFFFFF00000401000000003D
:1022A00000000002100000000700FF01F401000020
:1022B000FF000000F47506080000000000000000A8
:1022C0000102030406070809010000009819002014
:1022D00000000000000000000000000000000000FE
:1022E00000000000000000000000000000000000EE
:1022F00000000000000000000000000000000000DE
:1023000000000000000000000000000000000000CD
:1023100000000000000000000000000000000000BD
:1023200000000000000000000000000000000000AD
:082800000000000000000000D0
:1080000070B4C3080D4CE25C00F00706B24004EB0C
:10801000D004D2B20020C6F108038B4228BF0B4621
:10802000C3F108052A419840C91A40EA02004FF0FE
:10803000000614F8012FEED170BC7047381A0020EA
:10804000084AD2E91C31994209D0D118013391F87C
:1080500078100170C3F30A031367012070470020F2
:10806000704700BFF8190020064AD2F87838D2F8D5
:108070007C28934294BF4FF400600020013B9B1A80
:1080800018447047F8190020012380F851307047D8
:1080900007B501A8FFF7D4FF0028FAD09DF8040027
:1080A00003B05DF804FB044BD3E91C03984288BF7E
:1080B00003F50063181A7047F81900200120704773
:1080C000024BC3F88028C3F884187047F8190020C1
:1080D000024BC3F88828C3F88C187047F8190020A1
:1080E0007047704730B4124DD5E91C239A4286BFC1
:1080F00003F50064A21A9A1A0A44B2F5006F12D866
:10810000A1B101444A1E013810F8014FE91882421A
:1081100003F1010381F87840C3F30A03F4D16B67DC
:10812000002030BC7047022030BC70470846F8E79A
:10813000F8190020212838B50C4605D022282ED069
:10814000202813D0002038BD0029FBD0072AF9D100
:108150001A4BD3F8900893F8941893F8952893F84D
:108160009638206021716271A371EBE70029E9D094
:10817000072AE7D1114DD5F884381BB10968D5F825
:1081800080089847206821796279A379C5F890081A
:1081900085F8941885F8952885F89638D2E700294F
:1081A000D0D0022ACED1054AD2F88C38002BC9D0C3
:1081B0000988D2F888089847C4E700BFF81900205A
:1081C000024B0020C3F89808704700BFF819002040
:1081D000044B00200522C3F89828C3F88C08C3F884
:1081E00084087047F8190020704700BF704700BF2F
:1081F000704700BF704700BF704700BF704700BFA7
:10820000704700BF042301480B807047880100209D
:1082100010B4074A074B92F89C08122403F1140289
:108220000C8001280CBF184610465DF8044B7047BF
:10823000F81900208C0100200020704700207047B2
:108240000023F0B452004F1C1E46B0F1204F4FEAFD
:10825000107404F130052ABF3734CD54CC54FE5489
:1082600002339A424FEA0010EFD1F0BC704700BFD2
:108270000B4A0C4B10681B681A22C0180A8001D1E7
:108280000948704710B5094B09491C680822FFF7D7
:10829000D7FF204607490422FFF7D2FF024810BD4E
:1082A000E8F7FF1FECF7FF1FB4010020EAF7FF1FFC
:1082B000B6010020C6010020042301480B8070474E
:1082C000D0010020122301480B807047D401002008
:1082D000A0B182680D4B12B107229A7070471978CD
:1082E000DA6003294FF004000CBF80214FF4807145
:1082F000C3E901111A611A7598707047034B41F276
:10830000E47101225A545A70704700BFE46600209D
:108310000378022B10D0006908B9012070470C4B7C
:108320001B78032B0EBF0B4B80B24FF6F7739842AE
:1083300094BF0020012070470549436841F6500270
:108340008A58B3EB422F2CBF01200020704700BF9A
:10835000E4660020F7FFFF0F0378022B14D030B43F
:10836000104A4368006941F6480402F5C2511559A4
:10837000096841F63C042B4012595B0A023801FBA4
:108380000030104430BC7047064B426841F634015F
:1083900041F630005958185800EB410000EB5220CC
:1083A000704700BFE466002000487047201A002094
:1083B000034B93F82400032894BF0020012070474A
:1083C000F819002010B5084CE26D13899907FCD507
:1083D00013891B06F9D40A203DF0D8FD206EBDE8B4
:1083E000104041F017BF00BFF8190020034B93F86D
:1083F0002400003818BF0120704700BFF819002082
:1084000010B40C4A92F8A03802EBC3010133DBB27E
:10841000042B4FF0050408BF00234FF4045081F8EB
:10842000A44882F8A038C1F8A8085DF8044B4FF0C2
:10843000FF307047F8190020202301480B80704757
:10844000E8010020642301480B80704708020020E7
:10845000432301480B8070476C02002010B5084C84
:10846000D4F82801FF2809D00649D1F8C42801F61C
:10847000C801FFF75FFEFF23C4F82831002010BDBC
:1084800088010020F8190020E8E700BF08B5D0F8FF
:10849000E4355B6A9847002008BD00BF08B5D0F8F6
:1084A000E4351B6A9847002008BD00BF08B5124B91
:1084B000D86D828940F2E9330289013B12F0020F44
:1084C0009BB212D0FF23838140F2E9330289013B42
:1084D00012F0010F9BB202D08089C0B208BD002B00
:1084E000F4D143F011F9C0B208BD002BE4D143F040
:1084F0000BF9C0B2F8E700BFF819002070B50546C7
:108500000E460924FFF7D2FFFF2803D1013CF9D121
:10851000012070BDFE2801D0022070BD06493346FF
:108520002A46C86D002152F079FCFFF7BFFFFFF724
:10853000BDFF002070BD00BFF819002010B51C4C15
:1085400000232362FFF7B2FFE06D828940F2E93336
:108550000289013B12F0020F9BB217D0FD238381E9
:1085600040F2E9330289013B12F0010F9BB212D0B5
:108570008389FFF79BFFFF2812D1FFF797FFFF28A2
:108580000ED10423022084F8243010BD002BDFD14B
:1085900043F0BAF8EDE7002BE4D143F0B5F8E8E793
:1085A000D4F8D03863610923002084F8243010BD4A
:1085B000F819002070B582B040F040060C0E054658
:1085C0000A0A080C95238DF801408DF804108DF8E7
:1085D00000608DF802008DF803208DF80530082426
:1085E000FFF764FFFF2802D0013CF9D11DBB1A4BF5
:1085F000D86D062583896E464FF47A734FF6FF7166
:108600003EB316F8012B0489013BA4079BB215D594
:1086100093B283814FF47A730489E40703F1FF3244
:1086200011D5013D8289EBD10924FFF73FFFFF28D7
:1086300002D1013CF9D1FF2002B070BD8B42E2D1E2
:1086400043F062F8F0E793B28B42E5D143F05CF877
:10865000EAE7FF22D7E700BFF81900202DE9F84329
:10866000194C94F82460042E0546894690461F460E
:1086700008D0082E02D00020BDE8F883FFF75EFF87
:108680000228F8D1206E41F0BFFDA37E93B96902A4
:108690001120FFF78FFF98B9D4F8D038C4F80090B4
:1086A0000522C4E90387656084F824206361012002
:1086B000BDE8F88329461120FFF77CFF0028EBD0A6
:1086C000FFF780FED7E700BFF8190020F8B56A4C25
:1086D00000234FF4F0722021054604F6D80084F8F8
:1086E000D43857F04CF904F6B8204FF4F07220213A
:1086F00057F045F994F8990C10B194F89A2C0AB9EE
:108700000020F8BD41F0ACFAC4F8A40C28B182797D
:108710000AB1412AF4D12322C28009213DF006F892
:10872000D4F8A40C554E41F075FD94F89A0C01381C
:1087300040B243F0E9F80223102184F89C3CC4F8CD
:10874000A00C4FF073FAB6F82C114D4842F0A4FF7C
:10875000D4F8A40C41F058FDFF218C204FF0B4FB5D
:108760000746D4F8A40C41F055FDD4F8A00C042120
:108770004FF05CFA1B2F05D0D4F8A40C20213CF05C
:10878000D5FFBDE7D4F8A43C012284F8D4280BB16E
:108790002322DA80B6F82C11394842F07DFFD4F854
:1087A000A40C41F031FD40210A204FF08DFBFF2148
:1087B0008A204FF089FBC0F38013D4F8A40C84F80E
:1087C000A83C41F027FDD4F8A00C04214FF02EFA6C
:1087D00094F8983C012B46D0022B3CD0002B3ED085
:1087E00094F8A93C182B09D194F8A82CB6F82C3190
:1087F000A4F8AC5CA4F8AE2CA4F8B03CB6F82C11EC
:108800001F4842F049FFB6F82C111D4842F044FFC2
:10881000D4F8A40C41F0F8FC022100204FF054FBE6
:10882000D4F8A40C41F0F6FCD4F8A00C04214FF0CD
:10883000FDF994F8B92C94F8BA3C94F8B81C84F873
:10884000B41CC2F12002C3F1100384F8BB2C84F8DD
:10885000BC3C0120F8BD0823A6F82C31C0E710234A
:10886000A6F82C31BCE7002DF5D094F8A83C002BDD
:1088700014BF08231023EFE7F81900208801002017
:10888000942600202DE9F04FCE4DDFF86883DFF805
:10889000709384460F4616460FCD44462DED068B49
:1088A0000FC40FCD0FC495E807008BB099F8C23CF8
:1088B000029684E80700CDE906C7042B00F25C812C
:1088C000DFE813F0BA015A0155010500CA019FED16
:1088D000BE8ADFEDBE8ABE49C8F81C10BD49BE4B3A
:1088E000BE4AC8F818100299002918BF134638EE7E
:1088F000887AF5EE006A86EE87AAC8F82430B84F69
:10890000B84B03930026DFEDB87A9FEDB89A28EEB6
:10891000278AF0EE679A079BB34200F02281039BFF
:1089200013F8014B039306F1010B5FFA8BF2002C55
:1089300000F09581DFF8CCC2002303E00133152B52
:1089400000F08D8103EB43015D001CF80100A042A3
:10895000F4D14944049291F8DD1C002900F087818C
:1089600020463CF0A5FC03680593824618463CF07F
:108970008BFC9AF805103CF0DFFC90F800E0BEF1AB
:10898000000F40F06C8109EB050025090321013D32
:10899000049A059B80F81D2D8D4280F81C1D04F063
:1089A0000F0C00F23581874800EB4500808D40FABE
:1089B0000CF414F0010400F03D81012404FA0CF3DE
:1089C000013B1840049253F02FFD7E4BDFF838C274
:1089D000049A1D44032195F834307A4D18440CEB69
:1089E000C0037B619971DA715CF830009AF8082055
:1089F00000F13F4101F57E0105EB912191F838101E
:108A000001F01F054909032904FA05F400F00D815E
:108A1000042900F00581022900F0FD809B8808935D
:108A2000B3FA83F3C3F11F03C3F3CC0100EB81015D
:108A300003F007030C6A9B000F259D4024EA050400
:108A40000C620C6A02FA03F323430B62022308A9A7
:108A500009930CF007FBDAF80030029A002A00F0C4
:108A6000A380B9F8C02C00EE102AB8EEC00AFCEEC4
:108A7000C07A17EE901A5E4A934200F08280A2F507
:108A8000806293427DD002F58042934279D002F514
:108A90008062934275D002F58062934271D0D9F81A
:108AA000482F50084FF6FF73B0FBF1F21A44120C36
:108AB000B0FBF2F20298002866D0B2FBF1F199F80F
:108AC000C20C04288BB264D007EE902AF8EE676AD5
:108AD00066EE887A29EE677A99F8C30C06990091B8
:108AE000A6EEA87A019051463846C7ED027A87ED86
:108AF000037A31F0C1F9002E61DD7B68D8F83820A7
:108B0000934200F08380012E59D0D8F85020934230
:108B10007CD0022E53D0D8F86820934276D0032E12
:108B20004DD0D8F88020934270D0042E47D0D8F88A
:108B3000982093426AD0052E41D0D8F8B0209342B5
:108B400064D0062E3BD0D8F8C820D31A18BF012312
:108B50005E460122082E3B747A7407F118077FF4F1
:108B6000DAAE24480BB0BDEC068BBDE8F08F9FED6C
:108B7000228AF0EE488AAEE69FED208AF0EE488A1F
:108B8000A9E6D9F8480F8DE799F8C20C04281946D0
:108B90009AD107EE901A07EE102AF8EE677AF8EEEF
:108BA000476A67EEA97A95E7B0EE4A0A049354F053
:108BB0003BFBFCEEC07A049B17EE901A5BE70123A7
:108BC000C6E700BF20FA0508ACC5A737ACC5A73675
:108BD000413F0308AD330408FD3A0308A1330408FC
:108BE00048000010BF2600206F12833A00007A442C
:108BF0000004014014000010282930386F12033996
:108C0000F8190020D42600204027002000239FE7E9
:108C1000C7F814E021E717494D6C2C434C64FDE67E
:108C200014490D6B2C430C63F8E612490D6C2C4370
:108C30000C64F3E67C6110E79FED0F8A0F4BC8F8D8
:108C4000183000230E4A069301230293C8F81C2013
:108C50000C4BF0EE488A4AE69FED0B8AEEE70B4A92
:108C6000084BC8F81C20C8F8243000207AE70B68AD
:108C7000FFDE00BF003802406F12833AAD330408B4
:108C8000413F0308A133040800000000F53D03083C
:108C9000F8B51A4C94F84C3F002BFBD159B3014462
:108CA0004E1E451ED4F87C28D4F8781815F8017F9C
:108CB000531CC3F30A038B422CBF4FF40060002007
:108CC000C91A224401440129C4F87C3882F8507F33
:108CD0000FD101203DF078FAD4F87838D4F87C1818
:108CE0008B4294BF4FF4006200225B1A1344012BA5
:108CF000EFD0B542D6D10020F8BD00BFF819002052
:108D000010B590F85010002380F8503081B10B4C12
:108D1000D4F8982872B1D4F89828052A0CD13C30A0
:108D2000D4F8D038FFF7B4FFD4F8D038012010BD04
:108D30000120FCE71046FAE71846F8E7F81900208A
:108D4000002280F85120DBE790F85020531C0244A9
:108D5000DBB280F8503082F83C1090F851200AB114
:108D6000132B00D9CCE7704710B5094CD4F89838CC
:108D7000084611465BB1D4F89838052B07D1002A74
:108D8000D4F8D03803DDFFF783FFD4F8D03810BD16
:108D9000F81900202DE9F04143794A4C002B14BF0B
:108DA0000122002284F8502003D184F82430BDE849
:108DB000F08190F8018008F1FF3676B20546304622
:108DC0000F4642F0A1FD0223E06584F858302B786D
:108DD000002B53D1ED78002D44D14FF48071E06D1C
:108DE00025664EF023FF4FF47A703DF0EDF9206ECA
:108DF00041F010FAE06D0A2683894FF6FF714FF4B7
:108E00007A73FF270289950718D587814FF47A7303
:108E10000289D20703F1FF3520D5013E8289F1D1C5
:108E2000294B0289920711D5028912F080020DD1D7
:108E3000D4F8D018227601236161B6E7013B9BB2DA
:108E40008B42DFD142F060FCE06DE9E7013BE8D105
:108E5000227E84F82430531C2376A8E7ABB28B42E1
:108E6000D6D1EFE7284640F0FBFE054608B11E23A9
:108E7000C380092128463CF059FCAEE706EB860684
:108E80003E44414696F9032000203DF02FFE064661
:108E900030B1406850F08CFDB36884F86C3018B97C
:108EA000002384F8643095E7084A431E02EB43131D
:108EB00017210022A36650F08DFD012384F8643051
:108EC00088E700BFF8190020A1860100B802002041
:108ED000114B70B5D3F8484F054600680E4664083C
:108EE0000BF0C4FFB4FBF6F1B1F5803F03D3012CC6
:108EF000FAD96408F6E72246284689B23CF056F8CB
:108F00000649074BC1F8BC3E28460022BDE8704028
:108F100001F6BC613BF0CABFF8190020F02A00201E
:108F200031F801082549D1F8C43E0F2B04D05A1C52
:108F3000C1F8C42E0020704770B5214C94F84C5FE6
:108F40000023C1F8C43EF5B9D4F87828D4F87C38A9
:108F5000B2F5006F19D09A422CD01AD9C2F500632D
:108F6000402B18D9403B02F14005C1F8C83E01230F
:108F700084F84C3FC4F8785892B2402311490A440F
:108F800081210BF013FB002070BDC4F878588BB121
:108F90002A469B1AE4E74FF0000502EB0306C1F8EE
:108FA000C85E0CBF02210121C4F8786892B284F82F
:108FB0004C1FE3E7002384F84C3FE4E7F02A00204D
:108FC000F819002048290020ACE700BF70B51E4CFE
:108FD00094F84C3F012B03D0022B0AD0002070BD27
:108FE00001461A48D0F8C83E53B984F84C3F0020D7
:108FF00070BD00231A4681210BF0D8FA0023F4E754
:10900000402BD4F8782810D9403B02F14005C0F835
:10901000C83EC4F8785892B240230D4C084622440A
:1090200081210BF0C3FA002070BD4FF0000503EB67
:109030000206C0F8C85E08BF0220C4F8786892B281
:1090400008BF84F84C0FE8E7F8190020F02A002048
:1090500048290020012905D008B503210BF0A6FC02
:10906000002008BDB2E700BF70B5104DD5F8D43E62
:1090700004462BB195F8D82E95F8EC3E134310D04A
:10908000812120460BF01AF895F8EC3E022B00D017
:1090900070BD2046064ABDE870401F2301210BF039
:1090A000A7BA01210BF00AF8EAE700BFF02A002076
:1090B000BC39002070B50C4C0C4BC4F8F03E04F5E4
:1090C0006F62054684F8FC1E00260D23812184F87A
:1090D000006F0BF06BFA284604F6CC621F23BDE844
:1090E000704001210BF084BAF02A002055534253FE
:1090F0002DE9F041B04C94F8DB3EC4F8040F82B087
:1091000088465A2B00F2B580DFE813F0C900B3009F
:10911000B300D900B300B300B300B300B300B30091
:10912000B300B300B300B300B300B300B300B300A7
:109130000D01B300B300B300B300B300B300B3003C
:1091400031017400B300B3007400B300B300B30086
:10915000B300BA01B3006201B300B3007C00B300F6
:109160000B02B300B300B300B3005B00B300B30065
:10917000B300B300B300B300B300B300B300B30057
:10918000B300B300B300B300B300B300B300B30047
:10919000B300B300B300B300B300B300B300B30037
:1091A000B300B300B300B300B300B300B300B30027
:1091B000B300B300B300B300B300B300B300B30017
:1091C000E60194F8DC3E9B0700F16E82B4F8E23EC3
:1091D000D4F8DD2ED4F8141F5BBA9BB212BAD018A3
:1091E0008842C4F81C3FC4F8182F03D9FFF708F9C8
:1091F000002851DB0020A4F80C0F0546284602B0D9
:10920000BDE8F08194F8003F002B40F0FF8094F916
:10921000D83E002B2DDAD4F8083F08469B689847C3
:10922000002840F02182B4F8E25ED4F8DD7ED4F864
:10923000143F6DBAADB23FBA7A199A42C4F81C5FB6
:10924000C4F8187F03D9FFF7DBF8002824DBD4F833
:10925000103FD4F8D46E03FB05F503FB07F20220A0
:10926000B542C4F8182FC4F81C5F84F8000F00F052
:10927000D380524A92F8A038591CC9B202EBC303FA
:1092800005244FF40050042982F8A01883F8A4485C
:10929000C3F8A80800F0A6814FF0FF35AEE7D4F878
:1092A000D43E002BE5D1D4F8083F08469B68984788
:1092B0000546002840F0D881A4F80C0F9EE7404BEB
:1092C000002203F1120103F8012F8B42FBD13B492D
:1092D0003C4891F8A05894F80E3F702606709D42C5
:1092E0004FF00C06C67110D001EBC301013391F8A9
:1092F000A4588570B1F8A818DBB2042B49BA818153
:1093000014BF84F80E3F84F80E2F94F8DF3E12222B
:109310009342A4F80C2F98BFA4F80C3F00252846D0
:1093200002B0BDE8F08194F8DC3EDA0700F142813A
:10933000D4F8083F94F8DF0EDA6901EBC10102EBC3
:1093400081010A79531D834228BF0346A4F80C3FCC
:10935000002BE3D0013B1B489BB20133194403446B
:1093600011F8012D03F8012D8342F9D1D6E7164EED
:10937000164F35460823073EC5F10700A4F80C3FF9
:10938000002202E092F848201D462B46B54203F821
:10939000012900EB030217FA82F2F3D1D4F8083F57
:1093A0004046DB6898470028B8D0AB7863F07F036D
:1093B000AB70002522E700BFF02A0020F81900203A
:1093C000E3560020E4560020EB56002020FA050862
:1093D000D4F8083FC94A5B680846111D98470546FE
:1093E000002840F04181D4F8143FC54AD4F8101F3A
:1093F000013B180E1070180C09BAD37050701B0A7C
:10940000082093705160A4F80C0FF7E6D4F81C6F95
:10941000D4F8182FD4F8103FD4F8085FB2FBF3F259
:10942000B6F5805F28BF4FF480562D69B449B6FB6E
:10943000F3F340469BB24FF48057A4F80C7FA84743
:109440000028C0F2BC803346AD4AD4F8040F812115
:109450000BF0ACF8D4F8182FD4F81C0FD4F8F83E61
:109460003244851B9E1BC4F8182FC4F81C5FC4F837
:10947000F86E002D7FF452AF032384F8003FBDE661
:109480009F4E0027334606F10C0203F8017B9A42F7
:10949000FBD1D4F8083F40465B686A4601A998476B
:1094A0000546002840F0EB80019BBDF80020013B01
:1094B000190E52BAF3713171190C1B0A717108201F
:1094C000B371022172810C23BDF80220F070317259
:1094D0007272A4F80C3F91E68A4E8B4F30460823F7
:1094E000073EC0F10705A4F80C3F002202E092F805
:1094F000502018460346864203F8012905EB030273
:1095000017FA82F2F3D1D4F8083F4046DB68984757
:1095100000283FF403AFF37863F07F03F370002576
:109520006CE694F8003F002B62D194F9D83E002BF2
:10953000FFF69FAED4F8083F08469B68984700287E
:1095400040F09280D4F8083F4046DB6898470546D3
:10955000002840F0BA80B4F8E23ED4F8DD6ED4F8CA
:10956000142F5BBA9FB236BAF3199342C4F81C7F2A
:10957000C4F8186F00F2A380D4F8103FD4F8D42EAA
:1095800003FB06F603FB07F39342C4F8186FC4F815
:109590001C3F7FF46EAEB3F5805F28BF4FF480535D
:1095A0000121D4F8040F564A84F8001F9BB20BF037
:1095B0001FF823E607235549A4F80C3FCAE6544A8E
:1095C00092F8A038591CC9B202EBC30304244FF42B
:1095D0008850A14282F8A01883F8A448C3F8A808CC
:1095E0007FF45AAE002382F8A0384FF0FF3505E62D
:1095F000D4F81C6FD4F8080FD4F8103FD4F8182F03
:109600004569B2FBF3F2B6F5805F28BF4FF4805690
:109610000846B6FBF3F33A499BB2A847002862DB41
:10962000D4F8182FD4F81C5FD4F8F83E3244AD1BA0
:109630009B1BC4F8182FC4F81C5FC4F8F83E2DB962
:10964000D4F8040F2946FFF735FDD7E5B5F5805F5F
:1096500028BF4FF48055ABB2D4F8040F284A01213B
:109660000AF0C6FF0025C9E5294A92F8A038591C1E
:10967000C9B202EBC30302244FF4685003E6244A44
:1096800092F8A03802EBC3010133DBB202244FF49D
:109690006850042B81F8A448C1F8A80820D082F8AB
:1096A000A0384FF0FF35A9E5194A92F8A038591CA7
:1096B000C9B202EBC30305244FF41050E3E5FEF7F3
:1096C0009FFE0028BFF658AFE6E5114A92F8A03891
:1096D000591CC9B202EBC30302244FF41C50D2E55B
:1096E00082F8A078D8E50A4A92F8A038591CC9B285
:1096F00002EBC30304244FF440706AE7003A0020F1
:10970000E4560020EB56002020FA050860FA050810
:10971000F819002010B5074B93F8D91E0446FFF73F
:10972000E7FC002800DB10BD20460121BDE8104009
:10973000C0E400BFF02A002070B5344C94F8005FFC
:109740002DB1012D01D1FFF7E5FF002070BDB0F86C
:10975000B433D4F8D02EC4F8F42E1F2BD4F8D42E62
:10976000C4F8F82E064608D1294BD4F8CC2E9A42DC
:1097700003D194F8D91E01291AD9264A92F8A038A3
:1097800002EBC3010133DBB2042B08BF0023052524
:109790004FF40050C1F8A80882F8A03830460223E0
:1097A00081F8A45884F8EC3EFFF75EFC002070BD01
:1097B00094F8DA3E013B0F2BDFD8FFF799FC002825
:1097C0001CDB94F8003F013B022BBED9B4F80C1F00
:1097D000C1B1D4F8D43ED4F8F82E84F8FC5E8B42A4
:1097E00028BF0B46D11A0425C4F8F81E0A4A84F88B
:1097F000005F304681210AF0D9FEA6E73046FFF728
:1098000033FCA2E73046FFF755FC9EE7F02A002024
:1098100055534243F8190020E456002008B5084B80
:1098200093F8003F022B07D0033B012B02D8002105
:10983000FFF740FC002008BDFFF76CFF002008BDCB
:10984000F02A002010B501EB8101084A00EBC101AC
:109850000446B1F88C131046FEF744FC034A204638
:10986000402301210AF0C4FE002010BD103A002060
:10987000E8E700BF10B5044C04480A4621460AF048
:10988000F7FB204610BD00BF503A002024760608A2
:1098900010B5044C04480A4621460AF0E9FB20466C
:1098A00010BD00BF503A00203476060810B5044CB5
:1098B00004480A4621460AF0DBFB204610BD00BFE3
:1098C000503A00204076060810B5044C04480A4679
:1098D00021460AF0CDFB204610BD00BF503A0020C3
:1098E0004C76060810B5044C04480A4621460AF096
:1098F000BFFB204610BD00BF503A00205876060836
:1099000010B5044C04480A4621460AF0B1FB204633
:1099100010BD00BF503B00206476060810B5044C13
:1099200004480A4621460AF0A3FB204610BD00BFAA
:10993000503B00207476060810B5044C04480A46D3
:1099400021460AF095FB204610BD00BF503B002089
:10995000807606080A4608B5054920B905480AF088
:1099600087FB034808BD04480AF082FB004808BD95
:10997000503B002094760608AC76060810B502230A
:109980000446402281210AF0CDFE204602234022D7
:1099900001210AF0C7FE82212046032308220AF093
:1099A000C1FE064B02229A83FEF712FC044A2046AF
:1099B000402301210AF01CFE002010BD8801002078
:1099C000103A002038B509220D46044603238321AE
:1099D0000AF0A8FE29462046FFF7D0FF002038BD38
:1099E00010B5812104460AF067FE204601210AF0E5
:1099F00063FE024B002083F8000F10BDF02A002008
:109A000070B50446144EFFF7EBFF204602234022B8
:109A100081210AF087FE40220121204602230AF01C
:109A200081FED6F8083F00251B6886F8005F2846AF
:109A300086F8EC5E984720460AF09EFF20460121FA
:109A40000AF0B4FF204606F6CC621F2301210AF07B
:109A5000CFFD284670BD00BFF02A002010B581213F
:109A600004460AF029FE204601210AF025FE822143
:109A700020460AF021FEFEF7A3FB002010BD00BF28
:109A800038B50D46044683210AF016FE29462046C5
:109A9000FFF7E4FF002038BD00F01F02400901235A
:109AA000032803FA02F304D004280CD0022805D0BE
:109AB0007047074A116C0B4313647047044A516C9A
:109AC0000B4353647047024A116B0B431363704797
:109AD0000038024000487047A0270020002870D0BE
:109AE000F0B58388B3FA83F3202B0A4683B004468B
:109AF000C3F11F014FD0334F334D07EB81036E1875
:109B00009A66002196F858603BF010FEA388216801
:109B10002E48B3FA83F3C3F11F0202F0FC0404F1F0
:109B2000804404F59C3402F003024FEA820E4FF0A9
:109B30000F0C01F13F42A1680CFA0EFC21EA0C0166
:109B4000A16002F57E02A168C2F387224FF0004CAB
:109B500002FA0EF22CFA03F30A43A2604361026890
:109B60001B4922EA03020260426822EA03024260C1
:109B700002681A430260826822EA03028260C268B5
:109B800022EA0302C2600A68374413430B6097F865
:109B9000A830F02B01D803B0F0BD3544F02195F882
:109BA00068308DF8043003224FF4807301A887F8E1
:109BB000A8108DF80520ADF806300AF015FF03B0A7
:109BC000F0BD7047E83B002020FA0508003C01404A
:109BD000083C014000285FD00368374A2DE9F04176
:109BE00003F13F4404F57E0402EB9422012492F831
:109BF000382002F01F055209032A04FA05F456D052
:109C0000042A4FD0022A48D08588B5FA85F0C0F1E1
:109C10001F00C0F3CC0603EB860600F007008200AD
:109C20000F24306A944020EA04003062306A01FA5E
:109C300002F20243002132624FF0010E0A464FF059
:109C4000030C02270EFA02F838EA050002F10102BD
:109C50001CD118680CFA01F420EA04001860186896
:109C600007FA01F606431E609E6826EA04069E6017
:109C700098689860586820EA0800586058685860EA
:109C8000D86820EA0400D860D868D860102A01F1AA
:109C90000201D7D1BDE8F0817047084A556C2C43CA
:109CA0005464B1E7054A156B2C431463ACE7034ACF
:109CB000156C2C431464A7E720FA0508003802400D
:109CC0002DE9F84FCB4C94F8AF100546C1F3400195
:109CD000D4F8B40040F0A4FA94F8AF10D4F8B0006F
:109CE000C94301F0010140F09BFA002D00F0E7802C
:109CF00005F1FF39C04EC14FC14D5FFA89F94FF0F0
:109D00001008D4F8B43033B11A689B8851690B42FB
:109D100014BF53831383D4F8B03033B11A689B88CF
:109D200051690B4214BF53831383B4F8BC30002B2A
:109D300040F0578194F8BE10D4F8C00040F070FA9B
:109D4000FA204FF47A714FF0010C7B68C3F30803DB
:109D5000002B40F01981EFF31183002B40F01481A8
:109D6000D6F8D028D5F808E0D6F8D0389A42F7D1FE
:109D7000D4F8E4309E45F3D8D4F8E0A001FB0AF310
:109D8000A3EB0E03B3FBFAF301FB02327B68C3F3D0
:109D90000803002B40F0B680EFF31183002B40F056
:109DA000B180D6F8D038D5F808B0D6F8D0E87345E9
:109DB000F7D1D4F8E4E0F345F3D8D4F8E0A001FB00
:109DC0000AFEAEEB0B0EBEFBFAFE01FB03E39B1A91
:109DD000B3F57A7FDAD30138B7D1D4F8B43033B1E0
:109DE0001A689B8851690B4214BF53831383D4F8BC
:109DF000B03033B11A689B8851690B4214BF53834A
:109E00001383B4F8BC30002B40F0DF8094F8BE1010
:109E1000D4F8C00081F0010140F002FAFA204FF4BA
:109E20007A714FF0010C7B68C3F30803002B40F0FC
:109E30008A80EFF31183002B40F08580D6F8D0287C
:109E4000D5F808E0D6F8D0389A42F7D1D4F8E43003
:109E50009E45F3D8D4F8E0A001FB0AF3A3EB0E0370
:109E6000B3FBFAF301FB02327B68C3F3080343BB85
:109E7000EFF311832BBBD6F8D038D5F808B0D6F85D
:109E8000D0E87345F7D1D4F8E4E0F345F3D8D4F83B
:109E9000E0A001FB0AFEAEEB0B0EBEFBFAFE01FBDF
:109EA00003E39B1AB3F57A7FDED30138BBD109F106
:109EB000FF395FFA89F9B9F1FF0F7FF422AFBDE8EE
:109EC000F88FEFF3118A88F31288D5F808B02B6861
:109ED000DB0344BFC4F8DCC0D5F808B0D6F8D038EE
:109EE000D4F8DCE05FFA8AFA8AF31188D4F8E0A0AB
:109EF000734401FB0AFEAEEB0B0EBEFBFAFE01FB48
:109F000003E3CEE7EFF3118A88F31288D5F808B09F
:109F10002B68DB0344BFC4F8DCC0D5F808B0D6F822
:109F2000D038D4F8DCE05FFA8AFA8AF31188D4F8E2
:109F3000E0A0734401FB0AFEAEEB0B0EBEFBFAFE83
:109F400001FB03E343E7EFF3118E88F31288D5F8A2
:109F500008A02B68DA0344BFC4F8DCC0D5F808A019
:109F6000D6F8D038D4F8DC205FFA8EFE8EF3118854
:109F7000D4F8E0E01A4401FB0EF3A3EB0A03B3FBB1
:109F8000FEF301FB02326FE7EFF3118E88F31288C4
:109F9000D5F808A02B68DA0344BFC4F8DCC0D5F8B4
:109FA00008A0D6F8D038D4F8DC205FFA8EFE8EF305
:109FB0001188D4F8E0E01A4401FB0EF3A3EB0A0386
:109FC000B3FBFEF301FB0232E0E6D4F8D830002BFD
:109FD0003FF424AFD4F8C4200023136084F8D530B4
:109FE0001CE7D4F8D830002B3FF4AAAE3CF0B0F90F
:109FF000A6E600BFE83B0020F819002000ED00E0D5
:10A0000010E000E02DE9F04FCA4CCB4E94F8AF10B1
:10A01000D4F8B400DFF82883C84D83B0C1F3400101
:10A0200040F0FEF894F8AF10D4F8B000C94301F046
:10A03000010140F0F5F8052301934FF01009D4F821
:10A04000B43033B11A689B8851690B4214BF5383F3
:10A050001383D4F8B03033B11A689B8851690B422E
:10A0600014BF53831383B4F8BC30002B40F05981E4
:10A0700094F8BE10D4F8C00040F0D2F832204FF46B
:10A080007A710127D8F80430C3F30803002B40F09D
:10A090001B81EFF31183002B40F01681D6F8D028F6
:10A0A000D5F808E0D6F8D0389A42F7D1D4F8E430A1
:10A0B0009E45F3D8D4F8E0A001FB0AF3A3EB0E030E
:10A0C000B3FBFAF301FB0232D8F80430C3F3080300
:10A0D000002B40F0B780EFF31183002B40F0B280EB
:10A0E000D6F8D038D5F808B0D6F8D0E87345F7D10F
:10A0F000D4F8E4E0F345F3D8D4F8E0A001FB0AFE7D
:10A10000AEEB0B0EBEFBFAFE01FB03E39B1AB3F5AD
:10A110007A7FD9D30138B5D1D4F8B43033B11A68C5
:10A120009B8851690B4214BF53831383D4F8B0301A
:10A1300033B11A689B8851690B4214BF5383138350
:10A14000B4F8BC30002B40F0E08094F8BE10D4F896
:10A15000C00081F0010140F063F832204FF47A71C1
:10A160000127D8F80430C3F30803002B40F08B809C
:10A17000EFF31183002B40F08680D6F8D028D5F875
:10A1800008E0D6F8D0389A42F7D1D4F8E4309E45AA
:10A19000F3D8D4F8E0A001FB0AF3A3EB0E03B3FB62
:10A1A000FAF301FB0232D8F80430C3F3080343BBCF
:10A1B000EFF311832BBBD6F8D038D5F808B0D6F81A
:10A1C000D0E87345F7D1D4F8E4E0F345F3D8D4F8F8
:10A1D000E0A001FB0AFEAEEB0B0EBEFBFAFE01FB9C
:10A1E00003E39B1AB3F57A7FDDD30138B9D1019B24
:10A1F0005F1E17F0FF0301937FF421AF03B0BDE8AA
:10A20000F08FEFF3118A89F31288D5F808B02B6824
:10A21000DB0344BFC4F8DC70D5F808B0D6F8D038FA
:10A22000D4F8DCE05FFA8AFA8AF31188D4F8E0A067
:10A23000734401FB0AFEAEEB0B0EBEFBFAFE01FB04
:10A2400003E3CEE7EFF3118A89F31288D5F808B05B
:10A250002B68DB0344BFC4F8DC70D5F808B0D6F82F
:10A26000D038D4F8DCE05FFA8AFA8AF31188D4F89F
:10A27000E0A0734401FB0AFEAEEB0B0EBEFBFAFE40
:10A2800001FB03E342E7EFF3118E89F31288D5F85F
:10A2900008A02B68DA0344BFC4F8DC70D5F808A026
:10A2A000D6F8D038D4F8DC205FFA8EFE8EF3118811
:10A2B000D4F8E0E01A4401FB0EF3A3EB0A03B3FB6E
:10A2C000FEF301FB02326EE7EFF3118E89F3128881
:10A2D000D5F808A02B68DA0344BFC4F8DC70D5F8C1
:10A2E00008A0D6F8D038D4F8DC205FFA8EFE8EF3C2
:10A2F0001188D4F8E0E01A4401FB0EF3A3EB0A0343
:10A30000B3FBFEF301FB0232DEE6D4F8D830002BBB
:10A310003FF423AFD4F8C4200023136084F8D53071
:10A320001BE7D4F8D830002B3FF4A8AE3CF010F86F
:10A33000A4E600BFE83B0020F819002010E000E090
:10A3400000ED00E010B4B8B10D4CD4F8E830102B9B
:10A3500005D15DF8044B052100203BF0CFBC03EB99
:10A360004302224482F8ED1001210B4482F8EC00F4
:10A3700082F8EE10C4F8E8305DF8044B704700BF77
:10A38000E83B0020C0782021DCE700BF2DE9F04F3A
:10A39000DFF87CA32DED028B9AF830110022CAE978
:10A3A0004822CAE94A2297B0CAF81C2119B19AF882
:10A3B00031218AF81C219AF832211AB19AF83321F6
:10A3C0008AF82B219AF836211AB19AF837218AF89F
:10A3D00026219AF834211AB19AF835218AF82121D8
:10A3E0009AF8383105935A1ED3B257B204937B1CA6
:10A3F00000F0AA80BC4ABD4E52F83780029602EBAC
:10A40000C70200231279019308EE102A1D46344634
:10A41000994626783946304642F0B8FC83463046A5
:10A42000BBF1000F1ED03FF01BFCEA1D1321D2B27E
:10A4300020B14FF0000E827180F807E03BF076F912
:10A44000207842F0D5FC4FF0070309F10102237197
:10A450004FF0010384F802906070CDF804B05FFA09
:10A4600082F9E3700135042D04F10504D1D118EE11
:10A47000100A029ECDF80C90FFF70EFB9C499D4AF6
:10A480004868024042F440324A600FB9019B5BB910
:10A49000994C4820FFF700FB2046022151F00CF9AF
:10A4A000A26842F00102A2609148934A4168BAF85A
:10A4B0003A4141F400014160516821F480515160FA
:10A4C000916B21F4401141F480119163D16841F402
:10A4D0006001D160956B85F44011C1F3015101EB2E
:10A4E00081011F2000FA01FC25EA0C0C112505FA58
:10A4F00001F141EA0C019163D16841F4E011D160AE
:10A50000956BC5F30151C1F10401C9B201EB8101A1
:10A5100088404FF0100C25EA00000CFA01F10843C6
:10A520009063E4B1BAF83C11CAF84441A1B1BAF859
:10A530003E21CAF8481162B1019B7048521A90FB43
:10A54000F2F2CAF84C216BB917B0BDEC028BBDE832
:10A55000F08F6B4A1288EFE76A4A1188E7E76A4A88
:10A560001488DFE74046039951F0A6F85F4B0120BD
:10A5700003F114090723F278441CE4B252B375784E
:10A580003279A5F10A0101EB410105EB450C092DDA
:10A5900003FA01FE03FA0CFB02FA01F140F28E808D
:10A5A000D8F80C2022EA0E0E41EA0E01C8F80C1071
:10A5B000421E02EB82021F21062801FA02FC05FA64
:10A5C00002F261D8D8F8341021EA0C010A4320467F
:10A5D000C8F834200536B145CDD1D8F80820049903
:10A5E00042F40072C8F80820D8F8082042F48072BB
:10A5F000C8F80820D8F80820574442F00102C8F8EB
:10A60000082097F9402102203CF070FA0446002807
:10A610009AD040684FF0CCF9059A06214FF0DAF94C
:10A6200060680AF089FA07A80AF048FA039EA3684E
:10A63000364A0793012E8CBF4FF480600020002320
:10A640000D9008F14C054FF40060089509920A93AB
:10A650004FF480720C930E904FF4003360680B96A9
:10A6600007A94FF40055CDE90F5211930AF038FABB
:10A670006268136843F001031360D8F8083043F0B0
:10A680008043C8F808305FE7C11FA0F10D0201EB5D
:10A6900081014FF01F0E02EB82020C280EFA01FC22
:10A6A0000EFA02F005FA01F113D8D8F8302022EAA8
:10A6B0000C0211432046C8F830108BE7D8F8101070
:10A6C00002FA0CF221EA0B0B42EA0B02C8F8102046
:10A6D0006EE7D8F82C1005FA02F221EA00010A43CD
:10A6E0002046C8F82C2075E790FA0508043D0020A4
:10A6F00000230140E030FCFF0020014080380100D1
:10A700002E7AFF1F2C7AFF1F2A7AFF1F383D002068
:10A71000E83B0020F8B5264E00EBC00406EB8404AD
:10A72000D4F85C51002D36D094F86DC10CF0FF07C1
:10A73000BCF1000F2FD149004FF0010CC9B284F8D1
:10A740006E1184F86F2184F871C184F8727184F8F5
:10A7500070C184F86DC184F86C71AA88C4E95D3356
:10A76000940502D501273846F8BD2B88D9050CD4AD
:10A770004FF4805301E0013B10D02A889205FAD4AF
:10A780002B889BB243F480732B80AB889BB243F43D
:10A790004073AB80E6E700273846F8BDB6F8C43111
:10A7A00001339BB2A6F8C43150F02EFCDBE700BFAA
:10A7B000E83B002070B44E4A92F8C63103EB4300E8
:10A7C00002EBC000590090F8C80103281ED8DFE84A
:10A7D00000F00E200250C81802EBC000D0F8CC41A7
:10A7E0000CB3013CC0F8CC41002070BC704741481C
:10A7F00090F82061002E63D03F4C002001E086429B
:10A800005ED0258801308C34002DF8D0012070BC3A
:10A810007047C81802EBC000D0F8CC41002CE0D142
:10A82000022480F8C841194402EBC10191F8D40117
:10A830000138C0B281F8D401B0BB304892F88856D4
:10A84000D0F83003D1F8D041013303F00303421EA6
:10A850000326AB42224481F8C861B2FBF0F4C1F890
:10A86000CC41D3D090429CBF04F1FF34C1F8CC411D
:10A87000CCE7194402EBC101D1F8CC0190BB92F8AE
:10A8800088168B42C2D0013303F00304A14282F840
:10A89000C641BBD004EB440302EBC3020223C2F85F
:10A8A000CC0182F8C831B2E7144BD3F83023012031
:10A8B00002F2E73370BCB3FBF2F3C1F8CC3170475E
:10A8C0000E480B44D0F8301302EBC302012001F50F
:10A8D0001C530F3370BCB3FBF1F382F8C801C2F80C
:10A8E000CC3170470138C1F8CC0100208FE700BFA0
:10A8F000E83B002014000010103E002088010020DA
:10A9000030B583B00D46012301460DF10702044620
:10A91000074841F007F89DF8072035EA020304D004
:10A9200003482A43214641F053F803B030BD00BF2D
:10A930007442002070B5244D95F88C46022C1346C5
:10A9400082B00A4607D0014605F28C6002B0BDE82D
:10A95000704040F0E7BFD5F8941611B10C688988B3
:10A960006183D5F890168E8940F2E9340E89013C56
:10A9700016F0020FA4B223D084B28C8140F2E934E5
:10A980000889013C10F0010FA4B20DD08889084657
:10A99000002150F043FAD5F8943613B11A689B8819
:10A9A0001383012002B070BD002CE9D10846CDE927
:10A9B000002340F0A9FEDDE90023D5F89016E6E774
:10A9C000002CD3D1F2E700BFE83B002010B502789D
:10A9D000022A044613D0012A01D0002010BD2D4BBD
:10A9E00090F9040083F8CC26421CF6D00328F4DC4E
:10A9F0000A4603F2CC636179BDE810408AE68368B9
:10AA000013B11A689B8853836368988940F2E932CE
:10AA10001889013A10F0020F92B225D089B29981BB
:10AA200040F2E9321989013A11F0010F92B22BD0AC
:10AA30009A899A8940F2E9321989013A11F0020F94
:10AA400092B21ED001229A8140F2E9321989013A6C
:10AA500011F0010F92B20ED09B89A368BBB11A68A6
:10AA60009B881383012010BD002AD1D1184640F0E5
:10AA70004BFE6368DDE7002AE8D1184640F044FE4B
:10AA8000EBE7002AD8D1F8E7002ACBD1EEE7012086
:10AA900010BD00BFE83B00202DE9F04F2DED108BDD
:10AAA000034697B004331593DFEDCACA149002230E
:10AAB0008A4613928B461293149C4FEADB0604EBF2
:10AAC000461202EB06103101A6EB86034FEAC608D8
:10AAD00006EB4605CDE9000100EBC303043108F1A4
:10AAE00004001196204421442C01C6EBC60C0394AB
:10AAF000EC00119D04944FEACC0405946C0106EB24
:10AB0000860E0294159D009C03EB46174FEACE0E6D
:10AB100002EBC6064FEACB094FF0000C51ED01AA3B
:10AB2000D3ED001A92ED007A94ED005A96ED004AAA
:10AB3000D7ED007A15ED012A50ED016A32EE07BA21
:10AB400076EE840A7AEE855A31EEA70A3BEE256A44
:10AB500070EE804A76EEC46A36EE244A36EE646AB7
:10AB600005ED014A82ED006AD0ED00BAD6ED012A6A
:10AB7000D3ED019A95ED00AA92ED016A97ED013AA5
:10AB800091ED00CAD4ED014A7BEEE23A36EEE19A4D
:10AB900032EE472A73EEE98A3AEE464A39EE279AB0
:10ABA00078EE838AB0EE428AA9EE6C8ADC44E245F4
:10ABB00073EEC33AB0EE441AA8EEEC1A76EEE77ADA
:10ABC00033EEA97A7CEE643A77EEA17A3AEE066A21
:10ABD0007AEEC51A3CEE24AA74EECC4A39EE833ADA
:10ABE00035EE6A5AF0EE639AF0EE48AAE7EE2C9A38
:10ABF000A8EEAC4AE7EE2C4AE7EE6CAAF0EE418AEA
:10AC0000B0EE427AB0EE612A7BEE656A7BEEA22A54
:10AC100076EE4A5AA9EE2C7AA7EEAC2AA7EEAC5AE9
:10AC2000E7EEEC8A32EE83BA76EEC3BA35EEE09AFE
:10AC300075EEC07A36EE0A6A76EEE26A36EE0BAA56
:10AC400076EE836A77EEA07A34EE423A77EE290AFE
:10AC500036EE4B6A7BEEA22A39EE000A73EEAA3A70
:10AC600078EE244A37EE697A31EE055A71EEA85A29
:10AC700032EE044A85ED00AA82ED016A4D4441EDB1
:10AC8000012A4A44C4ED006A81ED000AC4ED017A4C
:10AC9000494440ED010A4C4487ED007AC6ED003A84
:10ACA000C3ED004A80ED003A87ED014A484486ED45
:10ACB000015A4F44C3ED015A4E444B443FF62EAF68
:10ACC000119B072B40F2C781029D149E019B0398A4
:10ACD0000499059A083575190C330E95354608F117
:10ACE00008080EF10804EB18083008310832464411
:10ACF0002C1928186918AA18079305F10C030D964A
:10AD00000C940B900A91099208934FF001084FF0B0
:10AD1000000E129B9E44139B03EBCE0303EBCE026B
:10AD2000109302EBCE0303EBCE01029101EBCE01B7
:10AD300001EBCE0505EBCE06D6ED007A0F93AEEB18
:10AD40008E03019106EB031303EBCE07D3ED01AAAB
:10AD5000CDED067A019BD5ED007A97ED01BACDEDE8
:10AD6000057AD3ED007A029BCDED047AD3ED007A1B
:10AD70000F9BCDED037A07EBCE0CD3ED007ADCED23
:10AD800001BACDED027A0CEBCE01D2ED007A109A29
:10AD9000009101EBCE00014691ED01DACDED017A93
:10ADA0000099D2ED007A91ED01CA00EBCE0000EBE4
:10ADB000CE0494ED01EAD0ED01DACDED007ADDE9C3
:10ADC0000776DDE90954DDE90B01DDE90D23C44611
:10ADD00002E000BFF304353F94ED009A90ED00FAD5
:10ADE00091ED006AD5ED007AD3ED006A57ED014A86
:10ADF00092ED005A56ED013A96ED00AA35EE060A9C
:10AE000073EEA65A39EE278A34EE8F7A70EE082A4E
:10AE100075EE87EA35EE465A3EEEA26A73EEE63AE2
:10AE200006ED016AD1ED019AD2ED01FAD4ED016A85
:10AE3000D3ED011A95ED013AD0ED018A97ED004A64
:10AE40003FEEE96A35EE491A76EE660A31EE271AC8
:10AE50003AEE612A75EE677A70EE830A3FEEA95AE0
:10AE600074EECF9A77EE897A7AEE211AB0EE42AA82
:10AE700074EE68FAA0EEECAADC44E24535EEC77A3F
:10AE8000B0EE639A74EE285A38EEC44AF0EE698A3E
:10AE9000A1EE6C9AE7EEAC8A36EE436A7FEE644A26
:10AEA00036EE266AA0EEAC2AF0EE4A0AE7EEEC0A8D
:10AEB000E7EEAC4AF0EE687AF0EE498A36EE833A75
:10AEC000E6EE6C8AE1EE2C3AB0EE6F1AA6EE2C1A82
:10AED00071EEE56AA6EE2C4A71EEA55A75EE031ADC
:10AEE0007EEEE22A37EE43FA75EEE1EAB0EE686AEA
:10AEF00076EEC08A39EE044A7FEE86FA76EEC86AAC
:10AF000033EE816A38EE888A73EEC13A37EE457ABD
:10AF10002CEE2E1A3FEE055A22EECC9A9DED03FA46
:10AF200070EE266A33EE077AAFEE221AAFEE2E9A53
:10AF30007AEE244A9DED01FA79EEA09A25EE4BAA0D
:10AF400072EE670A37EE822A6BEE087AAFEE08AA35
:10AF5000EFEE057A2DEEA63A9DED05FA67EE6D8AC5
:10AF6000AFEE073AEFEE268A66EE6A2A9DED00FA0A
:10AF70002AEEA00AEFEE202A6EEE02EADDED060AC6
:10AF800023EECE5AE0EEA3EA2BEEA98ADDED023ADB
:10AF9000AFEE060AA3EE848A24EE6B7A6DEE246A85
:10AFA0009DED044A2FEECD6AA0EE825AA3EEA97A57
:10AFB000E4EE2F6AA4EE246A75EEA15AC6ED005A9B
:10AFC00083ED001A83ED019A4E4447ED017A87ED37
:10AFD00000AA4B4480ED003AC0ED018A4F4482ED57
:10AFE000000A4844C2ED012AC5ED00EA85ED015A88
:10AFF0004A44C1ED006A81ED016A4D4484ED008A46
:10B0000084ED017A49444C443FF6E6AE0E9B08338A
:10B010000E930D9B08330D930C9B08330C930B9BE5
:10B0200008330B930A9B08330A93099B083309934F
:10B03000089B08330893079B08330793119B08F17B
:10B04000010843457FF465AE129BDDF844B0DB0098
:10B050009BB2129330E517B0BDEC108BBDE8F08FBA
:10B06000036870B55E6A26B133460522BDE87040BC
:10B07000184704460D464E1D00E023689B68204695
:10B0800098470028F9D0236815F8011B1B68204653
:10B090009847B542F1D170BD2DE9F047164D0746EE
:10B0A000002095F9D59605F2DC6684B007EB01081F
:10B0B00005F67C1504464FF0B60A3368ABB193F839
:10B0C0003830142B11D0B9F1FF3F01D04B450CD1D2
:10B0D000002269463046CDE90244CDE90078ADF85A
:10B0E00008A08DF80E4032F01DFFE036B542E4D1E5
:10B0F00004B0BDE8F08700BFE83B0020F0B40D6865
:10B1000000240CE0BCF1050F18D8A0F137030A2B7E
:10B1100014D104EB840415F8010B03EB4404A0F1F3
:10B120003003DEB2092EA0F16107A0F1410CF0D985
:10B13000052FE7D8A0F157030A2BEAD00D60146061
:10B14000F0BC70472DE9F743124E0124A0231825C7
:10B150005FFA84F8FF2B14DCD6F87C09E9B2C1F160
:10B160001C0282725F1C026880F80B80DBB20093C5
:10B17000C1F11B01D2F8189000234246C9B2C8475A
:10B180003B46013DE6D10134052CE0D103B0BDE8DA
:10B19000F08300BFE83B002010B50A4C94F89909F1
:10B1A000003818BF0120FDF791FA50B1064904F5A7
:10B1B000186040F005FA04F5186011F0CBFE04F5B4
:10B1C000186010BDE83B0020A8FA050870B4447967
:10B1D00041BB03684FF400524FF400762025022152
:10B1E0003CBB1A8C22F001021204120C1A841A8B36
:10B1F000188C22F0F30280B2120420F00A00120C24
:10B20000014342F0010241F001011A8319841A8BB3
:10B2100022F00C021204120C1A831A8B92B270BC28
:10B220001A83704700220368164615461146002C03
:10B23000D7D0042C21D0082C38D0198C21F480517F
:10B240000904090C19849C8B1D8C45F6FF7040F68F
:10B25000FF4128402140024342F4805241F4807172
:10B2600099831A849A8B22F440621204120C9A83F6
:10B270009A8B92B270BC9A8370471A8C22F010029B
:10B280001204120C1A84188B198C89B240F6FF42F2
:10B2900021F0A00102400D4342F4807245F01005F8
:10B2A0001A831D841A8B22F44062B3E71A8C22F4AD
:10B2B00080721204120C1A84998B1A8C21F0F301FB
:10B2C00092B2090422F42062090C324342F48072E3
:10B2D00041F0010199831A849A8B22F00C02C4E791
:10B2E00010B50446006809F0C1FD0C4BD3F8482F97
:10B2F000204652084FF6FF7139F058FE20460021D3
:10B30000FFF764FF0649074BC1F8C03E2046002204
:10B31000BDE8104001F56C6139F0C8BDF819002096
:10B32000F02A0020F1D001082DE9F04F824C94F86A
:10B330001E8C94F829AC87B016460B220546894628
:10B340004046114602959DF840701D463AF044F87B
:10B35000C245834640F0B080039040463EF080FCFA
:10B3600017F008030246019300F09A80BBF1000F2A
:10B3700000F092809BF80710890700F18D80C4F8D7
:10B38000ECB9C4F8E809C4F8E40910B140F60B318F
:10B39000C18005F0020ADFF8B881029B674A84F891
:10B3A000AC5908F5807100255846C4F8D439C4F862
:10B3B000C0194FF480733146C4F8A829C4F8B439D1
:10B3C000C4F8B839C4F8B06984F8AD79C4F8D8992C
:10B3D000C4F8BC89C4F8C859C4F8C459C4F8D059D1
:10B3E000C4F8CC59C4F8005C84F8045CA4F8F85B99
:10B3F0002EF0ACFBD4F8EC0907F00101FFF7E6FEF4
:10B400004F4A504BD4F8EC09C4F80C5CC4F8102C2B
:10B41000C4F8083CBAF1000F25D0D4F8F07917B37E
:10B420003A6803689A421ED001233146384684F8B0
:10B43000053C2EF08BFBD4F8F00908F5057229467F
:10B4400039F034FDD4F8EC092A4608F5077139F0D3
:10B450002DFD019B93B93C482EF094FB3A48012105
:10B460002EF0C8FB0AE0394A002302F1080184F8F3
:10B47000053C39F01BFD019B002BECD032482EF02F
:10B480008DFB314807B0BDE8F08FCDE90403039B85
:10B4900013B1D9798B0716D5002007B0BDE8F08F1E
:10B4A00015F00103F1D105F002018A46BAF1000F4F
:10B4B00022D1D4F8ECB96EE70B220C21504639F0BA
:10B4C0008BFF039049E750463EF0CAFB039AC4F84D
:10B4D000EC2915F0020ADDE90423C4F8E40905F0BB
:10B4E000020123D0904219D0C0B140F60C3CA0F824
:10B4F00006C0BAF1000FDCD0B8F1000FCCD0C4F810
:10B50000E82983B9BBF1000FC6D0C4F8ECB912B179
:10B5100040F60B33D3805FFA81FACAE7B8F1000F27
:10B52000BAD0C4F8E829C4F8F0B9F0E70028DCD1B3
:10B53000DDF80CB02FE700BFE83B0020F8FA050863
:10B54000E14003080D9C030890450020F0470020CF
:10B55000DC4500202DE9F041C84BC94EC94DCA4C0D
:10B560000822C3F88820336B82B043F001033363B1
:10B570000746884628464FF4C05240F202336946D7
:10B58000CDE9002309F06EFD6B6AC049C4F8381C90
:10B5900023F470436B626B6ABD49C4F83C1C43F4EE
:10B5A00020436B626B6ABB49C4F8481C23F47023C8
:10B5B0006B626B6ADFF820C3B74A01F5807143F410
:10B5C0002023C4F8501C6B62736C01F5007143F4C6
:10B5D0008043C4F88C1C7364736BA1F5F071C4F8DC
:10B5E000541C41F21C2041F2242143F0800344F812
:10B5F0000080675073634FF0A041A84EC4F8441C0C
:10B60000A74FA84BC4F890CC01F5366104F59155CD
:10B61000C4F8586CC4F8947CC4F85C3CC4F8981C1A
:10B620000123A14F2F604FF0020EACF5E46CA6F59C
:10B63000A066A1F5CC6184F840ECC4F84CCCC4F809
:10B64000046D84F8433C994F536106F58076C4F845
:10B65000C81C84F84A3D1946954B964AC4F8D06CEC
:10B660000CF5C07CA036C4F8DC7C934FC4F8D8CC71
:10B67000C4F8E03C0CF5D45C03F56953C4F8E46C01
:10B680004FF050260020DFF85482DFF854E2C4F86F
:10B69000082DC4F80CCD02F5A0420CF5A04CC4F85E
:10B6A000107DC4F8143D07F5A047A3F54853C4F82E
:10B6B000186D04F63846C4F81C2DC4F8247DC4F86F
:10B6C000443DC4F8CC8CC4F8D4EC0246C4F820CD78
:10B6D000334684F84C0D402783F81C21A3F822211F
:10B6E0000132042AC3E9497083F81D1183F81F0150
:10B6F000C3F8300103F12803EED10022114633468E
:10B70000402083F87423A3F87A230132042AC3E982
:10B71000DF0183F8751383F87713C3F8881303F1F7
:10B720002803EED14FF0A04364489A6822F001024A
:10B730009A60DA6842F04002DA6009F077F894F82B
:10B74000413C0022212161F317420BB142F48012E7
:10B7500094F83B1CD4F8443C01299A6300F0E7803C
:10B76000DA68D4F8447DD4F8480CC2F3076121F0BC
:10B77000600141F0400161F31F620021DA6039602D
:10B78000026861F3CC22026094F8432C012A00F095
:10B79000BB8010214A4809F009F9494809F0ECF842
:10B7A000D4F8481C94F8397C00224FF0FF300A612D
:10B7B0004A618861CA616FB306F11400DFF824E1C1
:10B7C00000EB87009446BF004FF0FF085EF8042F9F
:10B7D0001368002BACBF00234FF0904370451360FB
:10B7E000C2F810C0C2F80880F0D106F15003354805
:10B7F0003B444FF0000CFF2750F8042F1668002E32
:10B80000ACBF00264FF0904698421660C2F810C0B8
:10B810009760F1D10B6994F83B0C43F480730128D5
:10B820000B6161D0D4F8442C274C0023936100288D
:10B830004FF0FF336FF0804151615360516114BF8D
:10B8400000231023946143F470139069296843F432
:10B85000605343F00803034393619368096843F01E
:10B86000010393608847194B194ADA606846194BFF
:10B87000009309F0B9F802B0BDE8F08100E100E002
:10B880000038024000000240E83B002008040100AC
:10B890004000400100080050003C014040090050B9
:10B8A000400B005060090050BC040020A00500506F
:10B8B000C005005000100050003000502C480020FF
:10B8C00020480020704800200008008000ED00E0C3
:10B8D0000005FA0543020001200B0050200500502E
:10B8E0006005005034480020D4F8442C144B0B63FE
:10B8F00014486FF0804100234FF0FF349361516191
:10B900005460516190619EE701680F4A0F4F41F00A
:10B9100003010160802159629F62C3F80421E02283
:10B92000C3F80821C0F24002C3F80C2131E79A683D
:10B9300022F03E0141F02A0161F307029A600FE70D
:10B940000301810000080080A0004000800020006A
:10B95000094B93F8C23C042B08D9053B032B08D8AC
:10B9600001231A4600B103701046704700230122DC
:10B97000F8E700231A46F5E7F81900202DE9F0470B
:10B980009AB0DDE9226ADDF8909004460D4617462C
:10B99000984602E020683BF007F920683BF00CF97C
:10B9A0000028F7D10146642201A853F0E8FF264B96
:10B9B0008DF80450CDF85CA00293002D40D0AB1E52
:10B9C000012B3FD9042D14BF002203221F4B0396E5
:10B9D000D3F8D0388DF805201E440123CDE9059415
:10B9E00004968DF85B3037B14246394607A853F0CC
:10B9F00065FF8DF85A80164E96F8769100231893BD
:10BA0000B9F1000F19D196F87501642202FB0060AC
:10BA100001A900F5BC7053F051FF012386F8759120
:10BA200086F87631236843B143463A462946204694
:10BA30001AB0BDE8F04712F0DFBC1AB0BDE8F087DD
:10BA40000522C3E70222C1E7144E0020F8190020A6
:10BA5000E04C00209FED737A07EE901A20EE070A63
:10BA6000F8EE677A27EE800AFDEEC07A17EE903A7C
:10BA70002033402B00F2C780DFED6B7AB4EEE70A8B
:10BA8000F1EE10FAF0EE407A0CDD9FED686ADFED22
:10BA9000686AB0EE677AB4EEE67AF1EE10FA77EE05
:10BAA000C67AF6DC9FED637AF4EEC77AF1EE10FA0F
:10BAB0000CD59FED5E6ADFED606AB0EE677AB4EE9A
:10BAC000E67AF1EE10FA77EE867AF6D49FED5B7A9D
:10BAD000F4EEC77AF1EE10FA00F38D809FED587AFC
:10BAE000F4EEC77AF1EE10FA44BF9FED527A77EE8A
:10BAF000677A27EEA76ADFED535A9FED537ADFEDA1
:10BB0000536AA6EE257A67EE865AE6EE076AB6EE27
:10BB1000007AE5EEA67A27EE877ADFED486A70EEC6
:10BB2000267ABDEEE76A16EE103A2033402B67D82E
:10BB3000B4EEE60AF1EE10FA0CDDDFED3C5A9FEDB3
:10BB40003C6AF0EE676AF4EEC66AF1EE10FA77EE40
:10BB5000E57AF6DCDFED376AF4EEE67AF1EE10FA1C
:10BB60000CD5DFED325A9FED346AF0EE676AF4EEE1
:10BB7000C66AF1EE10FA77EEA57AF6D4DFED2F6AF9
:10BB8000F4EEE67AF1EE10FA40DDDFED276A76EEAC
:10BB9000E77A67EEA75A9FED2B5A9FED2B6ADFEDF0
:10BBA0002B6AA5EE856A27EEA55AE5EE866AB8EE01
:10BBB000006AE5EE267A67EE867AC7EE206A0023F1
:10BBC000836143610362C361B7EE006A76EE865A11
:10BBD00076EE666A86EE257A67EE277A66EE876AE3
:10BBE000C0ED017AC0ED037A80ED007A80ED027A33
:10BBF000C0ED046A70479FED0C7A77EE677A78E7BC
:10BC0000DFED137AD9E79FED127A86E7DFED0C6A54
:10BC1000F4EEE67AF1EE10FA44BFDFED066A76EE56
:10BC2000E77AB6E727D4D236DB0F4940DB0FC940AD
:10BC3000E4CB1641DB0F49C0E4CB16C1DB0FC93F93
:10BC4000DB0FC9BF92E741B99730083C15A82ABE5F
:10BC50000000000010B5184C94F8E20188B9174BA9
:10BC600083F85100586594F8E531012B1FD0D4F8C2
:10BC7000E83103B312495B68BDE81040A1F10C0044
:10BC800018473DF0EDFF94F8E4210C49003A18BF45
:10BC9000012281F8512048650028E4D01F22C2808B
:10BCA000202139F043FD94F8E531012BDFD1054B1C
:10BCB000C4F8E831DEE710BDE04C0020F8190020A0
:10BCC000CC4E0020D80400200C480D4BD0F81412A4
:10BCD00010B40C4CC0F804328A1E2231B0F82E3257
:10BCE0001B01A4FB03C3DB08A3F5B06322F8023FEA
:10BCF0009142F3D15DF8044B704700BFE04C002047
:10BD000015150208CDCCCCCC70B5084C251D2E469F
:10BD100014F8010B32F0D6FA28B1037805F8013B8C
:10BD2000B442F5D170BDFF23F8E700BF304F0020CB
:10BD30002DE9F0471D4F012607F10805B2464FF0E7
:10BD40003C094FF0000817F8010B3DF089FF04464D
:10BD500090B180F80690C671FB7803F07F02012A4B
:10BD600018D013F0800F20460DD185F804803EF0E6
:10BD70004BFA85F805802C600136052E05F1080583
:10BD8000E1D1BDE8F08785F804A03EF043FA85F8DC
:10BD900005A0F0E71B0605D40121204639F0C6FCBA
:10BDA000FB78DEE73EF036FAF6E700BF384F0020BA
:10BDB0002DE9F04FDFF8E091DFF8E0A183B009F161
:10BDC0000C05012419F8018BB8F1000F00F0BF80B9
:10BDD0004FEA1817013F032F08F00F0200F2BA8054
:10BDE0000AEB4703988D40FA02F616F0010600F0C0
:10BDF000C38001239340013B1840574450F014FB8B
:10BE000097F834305E4E184406EBC00604236E618A
:10BE1000F471B371002303E00133152B00F0978018
:10BE2000584903EB43025F00895C4145F4D1564B0E
:10BE30001A4492F8DD1C002900F0A080404639F039
:10BE400037FA8046006839F01FFA98F8051039F083
:10BE500073FA0378002B7AD14B4B3B44042283F8CE
:10BE60001D4D83F81C2D002E58D0336898F808001B
:10BE700003F13F4202F57E020AEB9222012792F87B
:10BE8000382002F01F015209032A07FA01F169D094
:10BE9000042A62D0022A6AD0B6F804C0BCFA8CF236
:10BEA000C2F11F02C2F3CC0103EB810102F00702D1
:10BEB0000E6A92000F27974026EA07060E620E6A66
:10BEC00090403043002208624FF0010B11460BFAFC
:10BED00001FE3EEA0C001CD118680326964020EAB9
:10BEE000060018601F6802209040384318609F6861
:10BEF00027EA06079F6098689860586820EA0E0055
:10BF0000586058685860D86820EA0600D860D86839
:10BF1000D8600131102902F10202D8D11B4B1C4A12
:10BF2000B3F88012B3F882320091002001340190FE
:10BF3000B2FBF3F328469BB24146E4B22DF09CFFDE
:10BF40000123092C6B7405F118057FF43BAF03B096
:10BF5000BDE8F08F00266E615CE70E4F3A6B0A4336
:10BF60003A6399E70B4A176C3943116494E7094A1D
:10BF7000576C394351648FE76E614BE70B68FFDE06
:10BF800040270020D4260020F8190020E04C002093
:10BF900040420F0000380240644F002020FA05089C
:10BFA0002DE9F0418C4B82B093F850230190002A88
:10BFB00040F00C8193F87423B3F87613DFED876AB1
:10BFC000B3F87883864D07EE102A07EE901AB8EE84
:10BFD000C76AB7EE007AB3F87213A5F83481F0EEB1
:10BFE000475A4FEA4804E6EE665A8C42B8BF0C4600
:10BFF000A6EE267AA6B20121F8EEE77AA5F8386116
:10C0000067EEA67AC5ED4A5A85ED4B7AC5ED4C7AB6
:10C0100083F85013002A00F0D680DDED017A9FED01
:10C02000710AF8EE677AA4B280EE270A51F042F95D
:10C030006400B0FBF4F4012CB8BF0124E4B2B0FBFF
:10C04000F4F39BB2074685F83C4100EE103ABBEE94
:10C05000ED0A85ED500A51F02DF9634BDFED636A6F
:10C06000B8FBF0F0A3FB0737FF0807EE907AF8EE75
:10C07000E77A022886EEA77AB8BF02205C4985F8E5
:10C08000440100239FED5B1A9FED5B6ADFED5B1AB5
:10C09000DFED5B5A9FED5B2ADFED5B2A9FED5B3A9C
:10C0A000DFED5B3A9FED5B4A85ED527A07EE903A01
:10C0B000B8EEE77AF0EE467AE7EE017AFDEEE76A4F
:10C0C00016EE902A2032402A7AD8B4EEE17AF1EEC8
:10C0D00010FA0CDDDFED506A9FED507AB0EE675A32
:10C0E000B4EEC75AF1EE10FA77EEE67AF6DCF4EE2B
:10C0F000E57AF1EE10FA0CD5DFED476A9FED487A4C
:10C10000B0EE675AB4EEC75AF1EE10FA77EEA67A9F
:10C11000F6D4F4EEC67AF1EE10FA49DD74EE677AE1
:10C1200067EEA76AF0EE624AE6EE824AF0EE430A54
:10C13000E6EEA40AB7EE007A27EEE65A77EE677AC3
:10C14000B6EE007AE5EE207A67EE877A0133202B8F
:10C15000E1EC017AAAD107EE904AF8EEE77AF7EE21
:10C16000006A86EEA77A2F4B2F4AC5F8E83703F10D
:10C170002801A833C5F8E4171020C5F8F4372021AA
:10C18000142385F84546A5F8E007A5F8F01707EE53
:10C19000906AF8EE677AA5F8EC3782ED007AC2ED86
:10C1A000AC7AC2EDAD7AC2EDAE7A02B0BDE8F081F4
:10C1B000F4EEE37AF1EE10FA48BF75EEE77AAFE7F6
:10C1C000F6EE007AC2E7194B1A7026E7044D95F88F
:10C1D0003C41B5F83861BEE7E04C00200AD7233C6B
:10C1E0001400001000247449ABAAAAAADB0FC941AD
:10C1F000600100103C8C4F3EDB0FC93F0100F8404E
:10C20000DB0F49C092E741B99730083C15A82ABE18
:10C21000DB0FC9BFDB0F4940DB0FC940E4CB164140
:10C22000E4CB16C128FB05085C06001000000010D6
:10C230002DE9F041214E224F96F87F3387F8AF3039
:10C2400006F55F7607F1B00500244FF0050816F8F3
:10C25000010B20BB28600134032C05F10405F6D145
:10C2600097F8AF10D7F8B000C94301F001013DF0D5
:10C27000D7FF97F8AF10D7F8B40081F00201C1F3EF
:10C2800040013DF0CDFF97F8AF10D7F8B80081F02E
:10C290000401BDE8F041C1F380013DF0C1BF3DF0B4
:10C2A000DFFC013401212860E3B210B180F8068080
:10C2B000C371286839F03AFACEE700BFE04C00209D
:10C2C000E83B00202DE9F0412A4C2B4DB4F8846363
:10C2D000A5F8BC6082B0EEB994F880033DF0C0FCD4
:10C2E00094F88123C5F8C000003A18BF012285F8F0
:10C2F000BE2048B194F882132B22002914BF1121CB
:10C300000121C28039F012FA002002B0BDE8F041EC
:10C310003EF09CBF94F88083002240462B2139F0E8
:10C320005BF8074640463DF09BFCF8B1F7B12B2285
:10C33000C5F8D800C280397AFDF74CFC4FF00008F0
:10C340000E4AB2FBF6F3C3F34F0000909BB239469E
:10C35000CDF8048005F1C400A4F886632DF08CFDAF
:10C36000D5F8C430C3F8008085F8D58002B0BDE8A8
:10C37000F08100BFE04C0020E83B002040420F006D
:10C380002DE9F84F254C94F8943384F8883304F25F
:10C390008B37002604F56A745FFA86FB0BF10108FF
:10C3A0005FFA88F8012117F8010F42460E448A46C9
:10C3B00039F012F84FF00009054640B3387804F818
:10C3C0000E9C04F80D9C04F80FBC04F810AC44F863
:10C3D000045C3DF045FC18B180F806A080F80780A9
:10C3E000297AFDF7F7FB0E4A0021284638F0DEFDDA
:10C3F0000C4B23600C4B221D21462846C4E9013911
:10C4000038F054FD697928684A462DF0EDFC082E75
:10C4100004F11C04C0D1BDE8F88F00BFE04C00203F
:10C4200040420F00219E0308D538030870B52C4CFC
:10C430002C4B94F8C004C4F8B83400220221C4F88C
:10C440007824C4F87C24C4F88024C4F8B424A4F864
:10C45000BC2438F0C1FF002841D0234B06680546B4
:10C4600003F1C0015A7C12B15A6896422BD018339E
:10C470008B42F7D1002394F8C004C4F8A45384F885
:10C4800098333DF0EDFB08B10223C380297AFDF714
:10C49000A1FB2846154A002138F088FD144A1549A9
:10C4A000C4F8A8130026111F2846134BC4F8AC3358
:10C4B000C4F8B06338F0FAFC697928683246BDE800
:10C4C00070402DF091BC30464CF0D8FF328D0B49B6
:10C4D00092B2531CB0FBF3F081F87403CAE770BD4D
:10C4E000E04C002000FFFF004800001040420F0019
:10C4F0008C500020FD3803089D3A03088801002075
:10C500002DE9F04FCD4CDFF8689383B006460D4619
:10C5100004F13400C022002153F031FA99F8C134FB
:10C52000002B00F0DB8099F8C234002B00F0F4807F
:10C53000C34E96F8D03C012B6CD0022B00F0F98052
:10C54000C04BDFF830C301931F46BCE80F000FC794
:10C55000BCE80F000FC796F8C6EC96F8C23C9CE802
:10C560000700DFF814C3C4F80CC1BEF1000C18BFFB
:10C570004FF0010C072B87E8070084F84CC900F244
:10C580002D81042B00F23B81AF4BDFF8F0A200932A
:10C590004FF000085FFA88FB0BF101095FFA89F997
:10C5A00045454A464FF0030132DD009B13F8017BFD
:10C5B0000093384638F010FF034638461F46002BDC
:10C5C00000F015813DF04CFBCAF8140020B14FF08B
:10C5D0000303837180F8079096F8C33C96F8C22C49
:10C5E000002B00F00281FB7983F0010359463846A5
:10C5F00008F101084DF0A2FA002800F0F8804FF091
:10C600000103B8F1080F8AF811300AF1180AC1D1F4
:10C61000019B61E08D4FDFF84C8296F8C6CCC4F8E0
:10C6200050590FCFA8E80F000FCFA8E80F0097E8E8
:10C63000070096F8C23C89F8FC34BCF1000C824B30
:10C640004FF0000718BF4FF0010C88E80700CDE954
:10C65000003508F1280A84F84CC9A8F5106889F853
:10C66000C4743D46D4F85029AA4240F3AE80009BE2
:10C6700013F8017B0093384638F0E2FE83463846D3
:10C680003DF0EEFA96F8C32C0746002A00F0A08091
:10C690009BF8072082F0010B0BF0010094F84C3955
:10C6A000013089F8C3040BB18BF0010B002F00F0AF
:10C6B000B680BB79002B5DD0412B5BD0644B6549C4
:10C6C000654AC4F83039019DC4F82C19012389F852
:10C6D000C434C4F838290023C4F84839D4F8483998
:10C6E0005BB10022012183F82C5083F82D101A63CE
:10C6F00083F82E2003B0BDE8F08F584E584D0FCE72
:10C700000FC50FCE0FC596E80700A5F1200385E8F9
:10C710000700C4F84839EDE7494B93F8C42C003AB8
:10C72000304618BF01222946FCF7ACF8C4F8480986
:10C73000D4E796F8C63C002B3FF402AF96F8C23C13
:10C74000082B7FF467AFDFF82CC1DFF82CE1BCE8E1
:10C750000F0004F1F40701970FC7BCE80F000FC7E3
:10C760009CE80700012387E8070084F84C39C4F8E7
:10C770000CE136E0B7F804C0CAF80C704001BCFA0E
:10C780008CFC40F009000135CCF11F014FF0030390
:10C79000CAF80410CAF814008AF810B0FD71BB7111
:10C7A0000146384638F0C2FF1BF0010F384612D060
:10C7B0003DF02AFDDAF80C20C8F81420082D0AF103
:10C7C000200A08F118087FF44DAF019D254B83E73F
:10C7D0009BF807B060E73DF01DFDEBE7082B7FF409
:10C7E000D3AE214BC4F85439CEE6FB79FEE61A4BA2
:10C7F000174AC4F81831C4F8102100236CE796F8E2
:10C80000C53C1A4AC4F85429012B05D0022B06BF97
:10C81000BEFA8EF35B09002384F85839B4E6400170
:10C8200040F009004FF0FF33CAF81400CAF8043092
:10C83000CAF80C708AF810B00135B1E71400001086
:10C84000F819002008010010BF260020A8FC0508E8
:10C85000A9330408AD330408A133040850FC0508CB
:10C86000A851002028090010ED3304081D340408E5
:10C87000E04C00207CFC0508D55F0508480000104E
:10C88000F8B5704F97F8280297F829523DF0E8F96B
:10C8900060B12D23C3802021044638F047FF0A20D1
:10C8A00039F074FB20463EF005FD18B9D7F8003585
:10C8B000DA0000D5F8BD013D092DFBD897F82752C5
:10C8C000EDB9402033F04AF90028F3D090F9044044
:10C8D00097F8FD11092CD4BF2346A4F114035A4C38
:10C8E0001C440A2994F8145C00F09D8094F81F3CC5
:10C8F00097F82622002A08BF1D46002DDAD02846C8
:10C900003DF0AEF90546002800F085802D23C38058
:10C91000012138F00BFF012108463DF089FC2B680E
:10C92000AA881A833C2039F04FFC002101203DF0F9
:10C930007FFC97F82932002B4CD0434C00261FE097
:10C940002B68AA885A8339F021FB94F8AF10D4F8E9
:10C95000B00001F001013DF063FC94F8AF10D4F891
:10C96000B800C1F380013DF05BFC2B68AA881A83F4
:10C97000782039F00BFB97F8293201369E4229DAEC
:10C9800094F8AF10D4F8B000C94301F001013DF0B4
:10C9900047FC94F8AF10D4F8B80081F00401C1F35B
:10C9A00080013DF03DFC7820002DC9D1782039F080
:10C9B000EDFA94F8AF10D4F8B00001F001013DF0A9
:10C9C0002FFC94F8AF10D4F8B800C1F380013DF00B
:10C9D00027FCCDE797F82732ABB997F82832002B20
:10C9E0007FF468AF97F82A32012B7FF463AFD7F852
:10C9F000003513F080537FF45DAF87F82932BDE82E
:10CA0000F84043F009B9322039F0DEFB2846002116
:10CA100038F08CFEE1E7012138F088FE012108465C
:10CA20003DF006FC7EE7D7F804355B057FF542AFA5
:10CA30000AF0C2FF00287FF43DAF002D7FF45FAF06
:10CA400038E700BFE04C0020E83B0020084B03F52E
:10CA5000A1600DC8904202DC114602460846984289
:10CA600004DD9A42B8BF1A4610467047704700BFAF
:10CA7000E04C00200B6810B414681B1B0360546862
:10CA80004B681B1B43608B6892685DF8044B9B1AD4
:10CA9000836070472DE9F047041E0D4612DB092C18
:10CAA00026DC824A0B468248A0FB0410C00800EB3B
:10CAB0008000A4EB40000021125C1A7059702846D7
:10CAC000BDE8F08764422D23092C01F8013B24D8EE
:10CAD000764A774BA3FB0403DB0803EB8303A4EB49
:10CAE00043030020D35C48700B702846BDE8F087F4
:10CAF0006F4B632CA3FB04264FEAD60621DC6B4A5E
:10CB00000B466B49A1FB0601C90801EB8101A6EBAD
:10CB10004101515C03F8011BC5E7654A632CA2FB88
:10CB200004364FEAD60637D8604A614BA3FB0603AA
:10CB3000DB0803EB8303A6EB4303D35C01F8013B63
:10CB4000C7E7A3FB0627B4F57A7F4FEAD7070DD2D4
:10CB5000564A0B465649A1FB0701C90801EB810162
:10CB6000A7EB4101515C03F8011BCAE7A3FB0728AF
:10CB700042F20F7294424FEAD80836D84B4A0B461D
:10CB80004B49A1FB0801C90801EB8101A8EB410158
:10CB9000515C03F8011BDDE7A2FB0637B4F57A7F91
:10CBA0004FEAD7070CD2414A414BA3FB0703DB08EE
:10CBB00003EB8303A7EB4303D35C01F8013BB4E72A
:10CBC000A2FB073842F20F739C424FEAD80821D8E3
:10CBD000364A374BA3FB0803DB0803EB8303A8EBC0
:10CBE0004303D35C01F8013BDEE7324AA3FB0809AB
:10CBF00094424FEAD90921D82C4A0B462C49A1FB73
:10CC00000901C90801EB8101A9EB4101515C03F85D
:10CC1000011BB5E7274BA2FB08099C424FEAD90943
:10CC200021D8224A224BA3FB0903DB0803EB830331
:10CC3000A9EB4303D35C01F8013BCAE71E4AA3FBFF
:10CC4000090394424FEAD30A21D80B461849174AE0
:10CC5000A1FB0A01C90801EB8101AAEB4101515C6A
:10CC600003F8011BCAE7144BA2FB09029C424FEADE
:10CC7000D20A13D80E4B0D4AA3FB0A03DB0803EBC1
:10CC80008303AAEB4303D35C01F8013BCAE70A2202
:10CC9000BAFBF2F047F0C2F80346D7E70A22BAFB24
:10CCA000F2F047F0BBF80146E4E700BFC47606089F
:10CCB000CDCCCCCC9F8601003F420F0070B43448ED
:10CCC00090F81435A3F13001092957D800F2145413
:10CCD000224600F2235012F8015FA5F13001092924
:10CCE00004D88242F7D1002070BC7047141B022C7C
:10CCF0004ADD2848002101E010F8013B01EB8101E9
:10CD000003EB4103161A303B022E044603F0FF01E9
:10CD1000F2DC214B03FB01F1A2424FF000030DD9DD
:10CD200003EB830314F8016B5B00303B3344A242F6
:10CD300003F0FF03F4D1194800FB03F32E2D06D0B6
:10CD40001748A0FB032301EB930070BC704701322E
:10CD500004200024157804EB8404303D6400092D80
:10CD600000F1FF30A4B202D82C44A4B2013210F07A
:10CD7000FF00EFD1642202FB0433E1E700211D46EE
:10CD800000F214520B46D9E7064C0021C4E700BF5D
:10CD9000E04C0020F55100208096980040420F00A2
:10CDA000ABAAAAAAF451002038B504460D460A469B
:10CDB0000068FF2152F0E3FD21682944216038BD5D
:10CDC00083B50C461646054631F0D0FA204631F0C0
:10CDD000CDFA0021204B0846002E08BF1E463DF02C
:10CDE00027FA002101203DF023FA284639F0E4FE1D
:10CDF000B0B1012100203DF01BFA284639F0D4FEE5
:10CE00000746204639F0D4FE0028FAD0394620469D
:10CE100039F0D6FE3846B047002108463DF008FA02
:10CE2000204639F0C9FE0028DFD0012100203DF066
:10CE3000FFF9204639F0B8FE01462846019139F045
:10CE4000B7FE01990028F8D0284639F0B9FE002134
:10CE500008463DF0EDF9C8E75DD00308F0B50023C2
:10CE60000B604B608B60CB600B610268DFF88CC09D
:10CE700089B004ADC2F385572E4647FA03F0C007C8
:10CE8000344604D513F80C0004F8010B2646013390
:10CE9000062BF2D11748C2F303240444002394F86C
:10CEA000BC4233708DF8184000F5317CC2F3053771
:10CEB0000DF1190647FA03F0C007344604D513F8FC
:10CEC0000C0004F8010B26460133062BF2D1002397
:10CED0003370C2F3834406ABCDE90134084602F057
:10CEE0000F0305490095C2F303124AF04BFA09B04B
:10CEF000F0BD00BF20FA0508EC760608D4FC050852
:10CF000070B5094CD4F82425054662B10026D4F842
:10CF100024052D2101363EF0CDFDAE42F7DBBDE804
:10CF200070403FF0DBBF70BDE04C00202DE9F04FBA
:10CF3000CCB2002185B00746084616463DF078F988
:10CF4000002101203DF074F93CF058FE022E09D07A
:10CF5000042E44F6C01818BF4FF49648072C06D983
:10CF600000200BE0FF2C4FF41648F7D10326CF4DDD
:10CF700095F828352BB90020C5F82C0505B0BDE87B
:10CF8000F08F032E0FD0CA490C44002294F8C70C2E
:10CF9000032138F021FA0028EDD0C64BC3F89C06D7
:10CFA000C3799A07E7D4C34C95F8280584F8B76E7F
:10CFB0000022032138F010FAC4F8A00A0028DAD0C1
:10CFC000BD4BC4F8583604F5D46103234FF4806296
:10CFD000A4F85C36C4F86C16002304F6A4214FF0C4
:10CFE000010A032EC4F86086C4F88436C4F86426A7
:10CFF000C4F87836C4F87436C4F87016C4F86826D5
:10D00000C4F88036C4F87C3684F8A83EA4F8A4AEF0
:10D01000C4F8B03EA4F8B43E84F8B63E04F5CB693B
:10D020000ED0D4F89CB69BF804003CF019FEC4F86E
:10D030009806584612F00EFB5146484612F01EFB69
:10D04000322039F0C1F8002E5FD1D4F8A08AD8F888
:10D05000000007F00BFF4046984A222137F0A6FF58
:10D06000974BC4F8BC3E97493246404637F01EFF06
:10D07000D4F89C86D8F8000007F0F8FE8F4A4FF6E7
:10D08000FF71404637F092FF31464046FEF79EF86A
:10D090008D4B8E49C4F8C03E3246404637F006FFFD
:10D0A000C5F82C954FF0060A022E12D0D5F82C05A3
:10D0B00039F082FD68B1012100203DF0B9F8D5F8C2
:10D0C0002C0539F079FD0146002840F09C803DF0A8
:10D0D000AFF8384639F070FD88B1012108463DF0BF
:10D0E000A7F84FF0050B4FF00008384639F064FD03
:10D0F0000146002840F0908001203DF099F8042E70
:10D10000D4D0052039F060F8CEE7012E09D1D4F84B
:10D11000A00A4146FBF7DCFED4F89C06FEF7E0F8D7
:10D12000BEE7022E09D1D4F89C0612F082FAD4F898
:10D13000A00A4146FBF7CCFEB2E7032E5BD14FF0CD
:10D14000000A84F8B8AE51466148DFF88CB140223D
:10D1500052F015FC8DF80FA0DFF854A19DF80F30A8
:10D16000072B09D95B48012112F088FAD4F8A00AEC
:10D170004146FBF7ADFE93E79DF80F3003EB430309
:10D180000BEBC30393F8453073B39DF80F3003EBFB
:10D1900043030BEBC3039B6C33B39DF80F30534435
:10D1A00093F8C70C00B30022032138F015F9019061
:10D1B000D0B112F03EFA9DF80F3094F8B81E019AE3
:10D1C00003EB43030BEBC30305EBC1009B6CC0F8FF
:10D1D0003035D379DB0748BF012301F1010148BF96
:10D1E00080F8343584F8B81E9DF80F300133DBB277
:10D1F0008DF80F30B2E7042E7FF452AFD4F89C06BE
:10D2000012F017FA83E7D5F82C0539F0CDFC01466A
:10D21000384639F0D5FC52E7384639F0C5FC95F868
:10D220007E3501468BB9242803D14FF0010385F8E0
:10D230007E35012E04D13846019139F0C1FC0199A7
:10D24000D5F82C0539F0BCFC4FE7012B06D14D2851
:10D250000CBF0223002385F87E35EAE7022B06D1B6
:10D260003C280CBF0323002385F87E35E1E7032B20
:10D2700010D10A2802D985F87E85DAE7042385F8DB
:10D28000710585F8708585F8738585F8720585F8D0
:10D290007E35CEE7042B21D195F8723585F87F05D0
:10D2A000434085F8723585F87EB5C2E7E04C002032
:10D2B000F8190020F02A0020ECFC050840420F007D
:10D2C00009F70108AC3900200DD00108B039002061
:10D2D000105200204831002014000010052BA8D166
:10D2E00095F8703595F8719595F872054B4509D20A
:10D2F0005A1C2B44484085F8720585F8702583F840
:10D30000741596E78842B6D195F87F3585F87EA5E5
:10D31000F42B8ED1B9F1000F8BD12421384685F83A
:10D320007E9539F04DFC4D21384639F049FC3E21BF
:10D33000384639F045FC4946384639F041FCF4217D
:10D34000384639F03DFCF421384639F039FC032EDB
:10D350001BD0D4F89C06437901689D080223AB409A
:10D36000DB439BB20B828D892B408B81007920217E
:10D3700012F04EF9D4F89C064A46494637F096FD1D
:10D38000D4F89C36186807F071FD0022D4F8A00A82
:10D39000114637F08BFDD4F8A03A186807F066FD07
:10D3A0000120EBE5114A013002EBC000F0B4D0F8E7
:10D3B00000C30F4E00233360336133623363336441
:10D3C000336533663367BCF1000F0DD090F8FC7203
:10D3D00057B13F0100240CEB04030FCB3519103477
:10D3E000A74285E80F00F6D1F0BC704720FA050887
:10D3F0006052002038B50F4C94F8071601F03F0139
:10D400008B1C024601F10A0584F8053684F80256A1
:10D4100004F5C06084F8032608311BF027F8254482
:10D4200085F8FE0594F802361C44000A84F8FF05CE
:10D4300038BD00BFE04C002070B51D4C0968D4F821
:10D440002C561C4ED4F82846D6EDDE7ADFED1A6A4B
:10D45000491B00EE901A0168F8EEE00A091B60EE25
:10D46000A70A00EE101A20EEA07AB8EEC00A1C46F9
:10D47000A0EE007AB1EE400AF1EEC77A67EEA67A26
:10D48000FCEEE77AC2ED007A4AF060F89FED0B7A85
:10D49000DFED0B7AE0EE077AFDEEE77A17EE902AE1
:10D4A000002ABCBF02F50C42A032226070BD00BF52
:10D4B000E04C0020880100202C7D8E3FA00CB3455D
:10D4C00000A00C4638B50B4C0025012280212046D7
:10D4D00032F030FB30B194F9040032F05FFB08B158
:10D4E000006838BD0135082D04F10C04EDD1002091
:10D4F000F7E700BF2053002038B5041F00F10805EE
:10D5000054F8043FD81780EA430017F0F7FBA54210
:10D51000F6D138BD2DE9F041D24CDFEDD37AD4F805
:10D520005C3A94F8F50A07EE103A2DED028BB8EE4E
:10D53000478A28EE278A002840F0CA80D4F8002BBA
:10D5400094F8F41A94F8113B002A19DD07EE902A9A
:10D55000DFEDC66AF8EEE77AC3F1640386EEA77AD8
:10D5600000EE103AB8EEC00A20EE070A29B920EE04
:10D57000000ADFEDBF7A20EE270A4FF09BFE80B253
:10D58000B4F8F63AA4F8F60A834200F0A18094F8C1
:10D59000607AB84EDFEDB88A4FF00008002594F8A5
:10D5A000143B2B41DB0714D594F8F43A002B7FD1C0
:10D5B000B4F8F63A07EE103A002F00F0FB80B8EE10
:10D5C000477AC8EE877A77EE887A88EE277A86EDF2
:10D5D000027A0135042D06F12406E0D194F8F95AB7
:10D5E000B4F8FC6A002D40F0E880002F5CD194F87C
:10D5F000103B84F81C5B84F8183B002E54D0002D9F
:10D6000052D007EE906A0123B8EE678ADFED9A7A6E
:10D6100084F8203B9D42C7EE888A28D0022D43D152
:10D62000D4F85C1A9548B0EE480A42F045FC94F8EC
:10D630001C3B012B00F01181022B35D1D4F85C1A70
:10D640008F48B0EE480A42F037FC94F81C3B012B9F
:10D6500000F0FE80022B27D1B0EE480ABDEC028B11
:10D66000D4F85C1A8748BDE8F04142F025BC864AF0
:10D67000D2ED007A78EEA76A134687EEA67A0021EB
:10D6800043F8041F83ED017A78EEA76A002187EE44
:10D69000A67A996083ED037A77EEA88A002287EE56
:10D6A000A87A1A6183ED057ABDEC028BBDE8F081A2
:10D6B000B4F8F63AD4F85C1A00EE103A301DB8EE21
:10D6C000400A002F70D142F0F7FB94F8607A80E7AF
:10D6D00094F8607A002F3FF45CAF94F8F95AB4F8EC
:10D6E000FC6A002DE0D0694A94F8FA3AD2F8A426F0
:10D6F00092F883201343D7D1D4F8002B94F8113B30
:10D70000002A65DD07EE902ADFED586AF8EEE77A29
:10D71000C3F1640386EEA77A012D00EE103AB8EE4D
:10D72000C00A27EE000A60D04FF0C4FD80B2A4F812
:10D73000FC0A002F79D08642B6D00028B4D094F8E5
:10D740001C3B002BB0D007EE900AB8EE678ADFEDE5
:10D750004A7A012BC7EE888A4ED0022BA4D1D4F886
:10D760005C1A4648B0EE480A42F090FA94F81C3B26
:10D77000012B6AD0022B97D1D4F85C1A4048B0EE46
:10D78000480A42F083FA94F81C3B012B58D0022B34
:10D790008AD1B0EE480ABDEC028BD4F85C1A394845
:10D7A000BDE8F04142F072BA301D42F06FFA94F8D1
:10D7B000607A0EE7C6F8048001E7344A94F8FA3A32
:10D7C000D2F8A42692F8832013437FF40EAF93E798
:10D7D0000023A4F8FC3A002F7FF466AF94F8103BC6
:10D7E00084F81C5B84F8183B5EE720EE000ADFED4E
:10D7F000207A20EE270A97E7234A1346F3EC017AB2
:10D8000078EEA76A87EEA67A83ED017AD2ED007AE8
:10D8100078EEA76A87EEA67A83ED037A77EEA88A78
:10D8200087EEA87A83ED057A3EE794F8103B84F8FA
:10D830001C5B84F8183B00283FF436AF0646E0E650
:10D84000114AD2ED007A131DE8E70F4A131DDDE7F8
:10D850000D4AD2ED007A131D1EE70B4AD2ED007A75
:10D86000131D11E714000010BD37863500409C459C
:10D87000CDCC4C3C740A001083F9223E380B0010CA
:10D880005C0B0010800B0010A40B0010E04C00207B
:10D89000F8B5214C1D270E46054684F8A8761AF0E7
:10D8A000F9FE00201AF096FE08201AF093FE0E20D2
:10D8B0001AF090FE38461AF08DFE04201AF08AFE07
:10D8C00004201AF087FE00201AF084FE30201AF09F
:10D8D00081FE00201AF07EFE30461AF07BFE00200A
:10D8E0001AF078FE1AF0C0FE04F2A9601AF0DAFD10
:10D8F000234670B194F8A92662B994F8AA26302A72
:10D9000000D03AB993F8AB2622B993F8AC362B7015
:10D910000120F8BD0120FCE7E04C0020104B03443F
:10D9200010B5044693F8D40311F0E8F80D4800EB65
:10D9300044040A23B4F9BC16B1F5FA6FA8BF4FF43A
:10D94000FA61B1F57A7FB8BF4FF47A71A1F57A71B7
:10D95000BDE81040B1FBF3F10920C9B211F0FCB8E9
:10D9600020FA0508E04C00201D4991F81425A2B3C7
:10D97000F0B4002605463346304637461BB991F8C9
:10D9800014452D2C23D02E2A19D0CA1800EB800064
:10D9900092F81445A4F13002092A4FEA40009CBFD6
:10D9A000A0F13002A0180E2B14D80133CA1892F837
:10D9B0001425002AE2D106B14042F0BC7047013381
:10D9C000002DF8D0CA182A4482F81475DDE7012327
:10D9D0001E46EBE70020F0BC70470020704700BFF8
:10D9E000E04C00201FB503AC8DF80C3000940023F0
:10D9F0008DF80D300AF032FB04B010BDF8B50546C5
:10DA0000262024F001FA134C0146F8B9D4F8E006B8
:10DA100090F838301E3B012B01D939F0D1F80E4F68
:10DA20000026AE420ADBB4F804370133A4F8043709
:10DA30000A4BD3F8D038C4F81437F8BD17F8011BD7
:10DA4000D4F8E00639F0BCF80136EAE7002384F8A0
:10DA50001237EDE7E04C0020C4530020F8190020F5
:10DA600010B58021044606F029FB2046002106F06F
:10DA700025FB2046BDE8104006F0FEBE10B5FCF7C1
:10DA800029F81121044637F051FE20463CF0BCFB3A
:10DA9000C82038F099FB2046BDE810403CF0BABBE6
:10DAA00008B53D203CF0DCF8054BC3F8180708B179
:10DAB0002A23C380BDE80840402137F037BE00BFAD
:10DAC000E04C00202DE9F04FB34CD4F8443C5A69A7
:10DAD000D2078BB002D50BB0BDE8F08F5A699B69B5
:10DAE00012EA030AF7D0CAF307431AF4002F00938F
:10DAF00040F00281009B5D0743D41AF0020F5FFAE9
:10DB00008AF503D0D4F8443C02225A61BAF1000FDE
:10DB1000C0F211821AF4006FCAF3072740F0848123
:10DB20002E0708D59D4B9E48D3F888339847D4F8E4
:10DB3000443C08225A61ED0600F1E981F80600F143
:10DB4000A981B90600F12E81009BDA0609D5934B15
:10DB50009348D3F898339847D4F8443C4FF4801254
:10DB60005A61009B9B06B6D58C4B8D48D3F89C33ED
:10DB70009847D4F8443C4FF400125A610BB0BDE80A
:10DB8000F08FD4F8482C9369D26913401FFA83FBB5
:10DB9000BBF1000FB1D0DFF80882CDF80CA04546EC
:10DBA0004FF0000909E05FEA5B0B09F1010908F198
:10DBB000040805F1280500F0DA811BF0010FF2D00E
:10DBC000D4F8481C5FFA89F708694A6B04EB8703AD
:10DBD000FA40D3F8503CD2019B68D2B202431A40BB
:10DBE000D007D3B216D54B6BD8F81820012000FA15
:10DBF00009F023EA00034B63684B6948D3F880338C
:10DC0000012191603946984794F83B6C012E00F051
:10DC1000FE8101231A0703D5D8F818200823936042
:10DC2000DE0603D5D8F8182010239360580603D5D4
:10DC3000D8F8182040239360990703D5D8F8182006
:10DC4000022393601A06AED5D5E94C60D5F824318D
:10DC5000D8F818C0311A8B42DCF8182028BF0B46C0
:10DC6000033392B2B2EB930F9DD9D4F8482C3237DC
:10DC700004EB8703CDE9019890469946B04238D22B
:10DC8000BEB3D5F8241194F83B3CD5F82821371AB7
:10DC9000B94228BF394601F1030E4FEA9E0E83B9FF
:10DCA0008FB20337BF10D9F840AC0AD0013352F815
:10DCB000040BCAF800009F42F8D1D5E94C60D5F8B2
:10DCC0002821DCF8183008440A44B042C5F828215D
:10DCD000C5F834010AD195F81C11D8F83420012771
:10DCE00007FA01F122EA0102C8F834209BB29E45EE
:10DCF000C4D3DDE9019856E7D4F8483C9D69DB6957
:10DD00001D402D0C3FF4F6AE04F63846DFF88CB01B
:10DD1000B046B146002708E06D0807F1010706F19B
:10DD2000040608F128083FF4E5AEEB07F4D5F9B294
:10DD300004EB8102D4F8483CD2F88C2C92685B69E1
:10DD40001A40D007D3B218D594F83B0C726D01235A
:10DD50009842936007D11269D8F87C33C2F312025B
:10DD60009B1AC8F88C33DBF87C334846984794F804
:10DD70003B3C012B00F0598101239A0702D5726DBB
:10DD8000022393601B07C7D5DBF8843348469847C6
:10DD9000736D08229A60BFE7E83B002088010020ED
:10DDA00020480020D4F8483CD4F8501C9A680868F1
:10DDB000C2F34102022A08BF03224FF0000514BF3C
:10DDC00065F30A0062F30A0008605A6842F4807240
:10DDD0005A6006A807F0F8F8D4F8442CD4F8480C98
:10DDE000D368C049079D6FF38D23D3608068C0F36B
:10DDF0004100014491F8EC13032900F0D180BA49A5
:10DE0000BA480126294484F83A6C81424FF0400612
:10DE1000A4F83C6C00F217810E2161F38D234FF4BE
:10DE20000051D36051618FE6B14B94F84A2DD3F87D
:10DE30009033B04800218DF817108DF817209847BF
:10DE4000D4F8481CD4F8442C94F8423C88684FF429
:10DE500000615161002B3FF463AEC3077FF560AEF4
:10DE600094F84D3D012B7FF45BAE9DF81730032BEA
:10DE70007FF456AED4F8443D9F491A6842F001023F
:10DE80001A601A6842F003021A600B6943F0060335
:10DE90000B6145E6D4F8482C964853684FF00008CB
:10DEA00023F001034146536006F080FD94F8396C7D
:10DEB000414656B1914BFF2203EB860653F8045FAF
:10DEC000D86BAA609E428260F8D1D4F8483C894859
:10DED0004FF0FF329A614FF00112DA610B2262F3C8
:10DEE000070162F30708C3F8148019611A686FF319
:10DEF0000A121A6006F0C0FCD4F8442C7C4B7D4812
:10DF0000D3F88C334FF480515161984719E6D4F817
:10DF1000443C9A6922F010029A611A6AC2F34340A3
:10DF2000022802F00F0146D0062823D09A6942F059
:10DF300010029A6102E694F8423C3BB1D4F8442DB9
:10DF4000136823F0030161F307031360D4F8482C2E
:10DF500067495368D1F89413664823F0010353606E
:10DF60008847D4F8443C4FF000425A61D2E5DDF8CE
:10DF70000CA0C2E5D4F8085D41F2042001EB810158
:10DF80002E68265004EBC1012E68D1F8C40F41F26F
:10DF90000825C2F30A1202446651C1F8C42FC5E72E
:10DFA00000214FF4007084F83A1C0921A4F83C0CBD
:10DFB00061F38D2333E747F6F0701042B6D001EBE2
:10DFC0008100C2F30A1204EBC00002F1030C5FEA05
:10DFD000AC0CD0F8B85FD4F808ED4FEA810818BF50
:10DFE000002006D00130DEF8006045F8046B84455F
:10DFF000F8D1414404EBC101D1F8B85FD1F8C40FA6
:10E0000015440244C1F8B85FC1F8C42F8EE7B9F1D6
:10E01000000F7FF4FEAD94F8493D042B7FF4F9AD79
:10E02000344806F029FC3346F4E5002F7FF4A4AE13
:10E0300094F8492D052A7FF49FAE4846019306F0D7
:10E040001BFC019B99E62E48A5F57401A1F5105122
:10E05000814203D80D2161F38D23E0E629492A4846
:10E060002944814203D20C2161F38D23D7E627484E
:10E07000A5F18C71A1F54341814203D80B2161F3D5
:10E080008D23CCE6224923482944814203D20A2128
:10E0900061F38D23C3E6204920482944814203D2FD
:10E0A000092161F38D23BAE61D48A5F1B771A1F5E9
:10E0B0005851814203D2082161F38D23AFE61949FB
:10E0C00019482944814203D2072161F38D23A6E632
:10E0D000164917482944814234BF0621052161F3BE
:10E0E0008D239CE620FA0508401E1BFF3F420F00CF
:10E0F000880100202048002000ED00E03448002086
:10E10000DFC810002013FBFE20D61300FF691800A3
:10E1100000D3CEFE40771B00C05BB3FEC091210050
:10E1200040AC2700C01D6AFE40E13300803C36FE53
:10E13000E09C4100704700BF704700BF704700BFC0
:10E14000704700BF08B5FFF799FC1B203BF088FD26
:10E1500008B12923C380FBF7BDFC08B12923C38084
:10E160000C4B93F81E27022A01D0012008BD93F81A
:10E17000E531012BF9D1084B084A03F1200103F1E5
:10E180004C00C2F8083FFDF7E5F9054B002083F885
:10E19000230008BDE04C002030050020F02A0020BC
:10E1A00000ED00E008B5074BD3F8240740B13DF07F
:10E1B00081F8054B93F89E3813B180F00100C0B28E
:10E1C00008BD00BFE04C0020F8190020BFF34F8FBE
:10E1D0000549064BCA6802F4E0621343CB60BFF303
:10E1E0004F8F00BFFDE700BF00ED00E00400FA051F
:10E1F00008B50021032006F051FC72B6FFF7E6FFD8
:10E2000080B5FFF7CFFF0028FBD1142037F0DCFFEB
:10E21000124F134E00BFFFF7C5FF0446A8B9D7F849
:10E22000D058D6F82837EB1A322B10D8D6F82C371E
:10E23000AB42EFD232353BF003FDC6F82C5700BF9E
:10E24000FFF7B0FF04460028E9D0FFF7D1FF0146F1
:10E250003BF0EEFFC6F82C47DCE700BFF8190020C2
:10E26000E04C002008B50121032006F017FC72B62F
:10E27000FFF7ACFF2DE9F04F8DB0CE4CDFF848939F
:10E28000CD4D00904FF0000854F80B0C002800F022
:10E29000FE8038F091FC0646002800F0D881D9F8BD
:10E2A000D03844F8073CE0260023C44F04F8033C70
:10E2B000A4F10B0B06FB08F654F80B0C38F07CFCB1
:10E2C000002800F0E48054F80B0C38F06DFC14F8D2
:10E2D000023C5A1E82460B2A0DD8DFE812F01F00BE
:10E2E0003A004600530083009B00E300160135010D
:10E2F000400177018E0124280CD0009A3AB995F894
:10E30000A226824240F07F81012204F8032C0D2BCB
:10E31000D2D186E0012304F8023CCDE700234D284A
:10E32000C4F8C53084F8CD3084F8CE3004D05828F5
:10E3300008D004F8023CBFE7022204F8022C84F85B
:10E34000C430B9E7032304F8023C022384F8C43044
:10E35000B2E704233C2804F8023C0BD0BAF13E0F8C
:10E360000CD0002304F8023CA6E70A233C2804F85A
:10E37000023CF3D1002304F8013C9DE7012304F89B
:10E38000013C99E7D4F8C500BB190344421CC4F80A
:10E39000C52083F8E7A694F8CD00022A8AEA000196
:10E3A00084F8CD1088D12378C02BDAD86278FF2A80
:10E3B00008D1052BD5D9012384F8C430072304F8EC
:10E3C000023C79E7A4F8C12000229342C4F8C93086
:10E3D00014BF0523062384F8C320C4F8C52004F81D
:10E3E000023C69E7D4F8C500BB190344421CC4F8D9
:10E3F000C52083F8E7A694F8CD00D4F8C9308AEA9E
:10E4000000019A4284F8CD107FF456AF062304F839
:10E41000023C51E794F8CD308342A2D10D2304F899
:10E42000023C14F8017C002F40F0F380644B089408
:10E430000FCB04AE86E80F00D4F8C930D4F8D10071
:10E44000ADF82C7023440993B4F8C130ADF82830EE
:10E4500094F8C3308DF82A3001238DF82E303246DF
:10E4600003AB08A9039732F001F848B1049B059368
:10E4700094F8C420534B0493314658462FF052FD74
:10E48000039E002304F8023C002E40F0D88008F1DF
:10E490000108B8F1030F04F1E0047FF4F5AE0DB00C
:10E4A000BDE8F08FD4F8C500BA190244431CC4F883
:10E4B000C53082F8E7A694F8CD2094F8CE000193F9
:10E4C0008AEA0202514684F8CD2046F05BF8019BAF
:10E4D00084F8CE00072B7FF4EFAEB4F80530C02BE4
:10E4E0003FF63FAFB4F80320A4F8C120A27884F827
:10E4F000C32000229342C4F8C93014BF0823092363
:10E50000C4F8C52004F8023CD6E6014694F8CE00D3
:10E5100046F038F894F8CD3084F8CE008AEA030348
:10E52000D4F8C50084F8CD30BB190344421CC4F8AC
:10E53000C52083F8E7A6D4F8C9309A427FF4BCAE70
:10E54000092304F8023CB7E694F8CD30434084F840
:10E55000CD3094F8CE3083427FF403AF56E7D4F841
:10E56000C500BA190244431CC4F8C53082F8E7A6B6
:10E5700094F8CE000193514646F004F8019B84F8CC
:10E58000CE00052B7FF498AEB4F80120B4F8033028
:10E59000A4F8C120227884F8C32000229342C4F852
:10E5A000C93014BF0B230C23C4F8C52004F8023C67
:10E5B00082E600BFCF420020E04C0020E83B002074
:10E5C00010FE0508D8F30020F8190020014694F841
:10E5D000CE0045F0D7FF84F8CE00D4F8C500BB19B3
:10E5E0000344421CC4F8C52083F8E7A6D4F8C93018
:10E5F0009A427FF461AE0C239BE694F8CE308342BE
:10E600007FF4AFAE0AE7232804BF022204F8032CEC
:10E610007DE6012F4FF0000602D004F8026C36E7C9
:10E62000D4F8C93008942344099308A8B4F8C13039
:10E63000CDE90A66ADF828302FF06AF8EDE754F816
:10E640000B0C2FF093FE54F80B0CB0471FE714F897
:10E65000033C002B3FF41BAFD9F8D02854F8071C1B
:10E66000521A632A7FF613AF012B32D0022B7FF4AC
:10E670000EAF54F80B3CC5F83437C5F83837C5F839
:10E680004037402385F84437134BC5F82435C5F887
:10E690008837124B85F8450793F8973910480122BF
:10E6A00085F830270F4AC5F83C27003B0E4A18BFB3
:10E6B000012382F8AC3B3EF015FC4FF4005031F0E2
:10E6C0009FFD0A483EF004FC85F88C6785F88D674D
:10E6D000DDE6FFF7C7FD00BF1C540020E83B00202B
:10E6E000FB7606084533040814000010317706084D
:10E6F0002DE9F0414FF0FF35324A33482C460023D4
:10E7000004E001330B2B02F1100215D0917A042999
:10E71000F7D103F5B17100EB0111C979CF07F0D43E
:10E72000661C116801D0A942EBD21C4601330B2BA9
:10E730000D4602F11002E9D1631C02D10120BDE8AF
:10E74000F081214D04F5B17705EB07139988F1B9F4
:10E75000DFF880802601AB19D8F8E8211B4916693B
:10E760001B4A41F2186001EB442118580023B047BE
:10E77000D0B1022808D141F2CC6205EB0717AB58A3
:10E78000013B0121AB50B9710020BDE8F081DFF8F9
:10E79000448005EB0413D8F8E82141F21860D268F0
:10E7A000185826019047D6E741F2CC6205EB0717CF
:10E7B000AB580321B97141F2D061013B0124AB5048
:10E7C0006C54BCE7007D0020E4660020FC6600205D
:10E7D000F1E70008E04C0020044B41F2E472995C40
:10E7E00009B90121995401225A707047E46600204A
:10E7F00038B5174D174B41F2D0640020285504E07E
:10E8000001300B2803F1100314D053F80E4C8C4246
:10E81000F6D11C78032CF3D16AB10F4B03EB4023E4
:10E820009A4201D0FFF7D8FF00F5B17005EB001058
:10E830000123837138BD41F2CC6100F5B1736A5890
:10E8400005EB03130420013298716A5038BD00BFF4
:10E85000E46600200A7D0020FC66002038B5134BDA
:10E8600000209C7B14B11D688D4205D001300B281F
:10E8700003F11003F5D138BD72B10D4B03EB40230A
:10E880009A4210D0FFF7A8FF0A4B00F5B17003EBD6
:10E8900000100123837138BD064B00F5B17003EB06
:10E8A0000010827138BD022CECD1EDE7FC7C002019
:10E8B000FC660020E46600202DE9F84F12F0020EFD
:10E8C0009B4606D028B9FFF787FF02252846BDE8FA
:10E8D000F88F804C41F638056559002D5BD14FF01B
:10E8E000FF367D4FB146B046B24600253B689842A0
:10E8F00000F0B68097F80EC0BCF1000F5BD0BCF101
:10E90000010F15D105F5B17C04EB0C1C9CF807C078
:10E910001CF0010F0CD11CF07E0F09D15FEADC1353
:10E9200040F0A880D7F808C0D44501D2E246A946F5
:10E9300001350B2D07F11007D8D1751C04D1B8F1A2
:10E94000FF3F00F09F80464641F2C86806F5B17768
:10E9500054F80850013544F8085004EB061C41F205
:10E960001C694FEA07184CF8095044F8085041F266
:10E97000186904EB07154FF000084CF80900C5F8BA
:10E98000048004EB0715AD79042D9CD8DFE805F071
:10E990001A330F334D0004F5C25741F63C063F6869
:10E9A000A65907FB0565A84299D3FFF715FF002577
:10E9B0002846BDE8F88F2E4601350B2D07F11007CC
:10E9C00094D1BAE712F0010C70D104EB0710D51006
:10E9D00090F80780BBF1030F65F3C71880F8078034
:10E9E00062D94FF6FF7083455B4628BF03469BB252
:10E9F00004EB07108380BEF1000F16D004EB061362
:10EA000003F5B0531833987B04280ED041F2C86543
:10EA10004FF0040C60590130605141F2CC655860F0
:10EA200083F80EC0635901336351500705D504EBD9
:10EA30000710C37943F00103C371D30608D504EB73
:10EA40000714E379C3F34502013262F34603E3712D
:10EA5000224B012503EB46260E602846BDE8F88FC1
:10EA600005F5B17704EB07164FEA071CB67986B9AE
:10EA70002E4669E7A84601350B2D07F110077FF4F4
:10EA800035AF5AE7B9F1FF3F18BF4E467FF45CAF90
:10EA90008DE741F2C8682E4654F80850013544F815
:10EAA000085044F80C506CE76346A1E70C4B0B4947
:10EAB000D3F8E8310B4AD3F8088001EB4621002354
:10EAC000C04700283FF473AF04EB07140223A3717F
:10EAD000FCE600BFE4660020FC7C0020FC66002011
:10EAE000E04C00205DE80008F0B5124D2B7841F6AF
:10EAF0003002022B0BBF070AC0F3D417C4B200F0D8
:10EB00007F04A85883B00E4600230122384401A98F
:10EB1000FFF7D2FE01280AD12B78022B019B16BFEA
:10EB200053F8243033F8143023F07043336003B0CB
:10EB3000F0BD00BFE466002010B5144602070B4686
:10EB400010D50B4941F2C472581C8B58834204D330
:10EB500005D100232360012010BDFFF73DFE20609A
:10EB6000012010BD21461846BDE81040BCE700BF9B
:10EB7000E46600202DE9F0414268C2F308030B442B
:10EB8000B3F5007F82B004460D4657D390F91A3092
:10EB9000591C0AD0304A03F5B17302EB0313FF216D
:10EBA000DA796FF30002DA71817694F91B305A1C1E
:10EBB0000FD0294A03F5B17302EB0313FF20DA7972
:10EBC000C2F34501013921EAE17161F34602DA71CC
:10EBD000E0762378022B37D01F4A02F5C2531B6818
:10EBE000B5EB432F4FEA432824DC41F6480367681E
:10EBF000D6583E407342AB421CDCAB19434511D39F
:10EC00002169207E01AAFFF797FF012812D16768CA
:10EC1000236963614744019B2361A5EB0801BF1B86
:10EC200067608D192046F9F773FB20B93D44656094
:10EC3000012000E0002002B0BDE8F08115444560ED
:10EC4000012002B0BDE8F0816168012029446160C3
:10EC500002B0BDE8F08100BFE466002070B5154643
:10EC600004460E46FFF786FF50B994F8280028B9ED
:10EC7000022384F82830C4E90B5670BD022070BD11
:10EC80001DB12046A847012070BD012070BD00BF06
:10EC900010B4D0E9011390F91A208B4238BF0B460B
:10ECA000511C83600AD0144B02F5B17203EB0212BF
:10ECB000FF21D3796FF30003D371817690F91B3074
:10ECC0005A1C0FD00C4A03F5B17302EB0313FF2457
:10ECD000DA79C2F34501013921EAE17161F34602B3
:10ECE000DA71C4760022436A5DF8044B42614260E7
:10ECF00011460361B2E700BFE466002038B5442244
:10ED00000021114850F03BFE104B41F602011A78E9
:10ED10004FF6FF745C52022A41F2E87118BF0322D9
:10ED200003F5C05041F64C055A5441F60C0441F627
:10ED3000010203215D5900F8181910211D51995441
:10ED4000FFF7A6FF012038BDCC7E0020E46600203E
:10ED50002DE9F041B1F904300F2B82B00C46164674
:10ED6000054632D02846F9F7F7FA95F91B80B8F135
:10ED7000FF3F074633D02D4B41F2186203EB0811D9
:10ED80008A58904211D1183303EB4823A1880131EE
:10ED900009B203EB4113A18028463360F9F7DCFA8E
:10EDA0002060012002B0BDE8F081FFF715FD284684
:10EDB000F9F7AEFA28B100230120336002B0BDE8B4
:10EDC000F081002002B0BDE8F0814FF40071FFF740
:10EDD000D1FE0028F5D04FF6FF73A380C2E7284686
:10EDE000F9F796FA0028E2D10FB9FFF7F5FC38469B
:10EDF0000023112201A9FFF75FFD0128D7D1019B54
:10EE00000B4A9A1A48BF02F2FF12B2F5B05F4FEAFE
:10EE1000622106D24FFA81F885F81B80002BB5D10C
:10EE2000C5E7FFF7D9FC019BF6E700BFE4660020C9
:10EE3000FC66002030B50446C06983B010B90120DB
:10EE400003B030BD0D460023032201A9FFF734FDB6
:10EE50000128F5D1B4F92030002B03DAFFF7BCFC10
:10EE60000220EDE7019A012D4FEA431102EB431313
:10EE700003D0022D12D1E5255554A268DA6122781B
:10EE8000032A04D100221A775A779A77DA77626ACE
:10EE90005A83C2F30F429A8203B030BDE268DA614E
:10EEA000EDE700BF10B50378023B012B0446037E5B
:10EEB00002D913F0060F5AD198063AD494F91A30B1
:10EEC000591C0AD02D4A03F5B17302EB0313FF213D
:10EED000DA796FF30002DA71A17694F91B305A1CCB
:10EEE0000FD0264A03F5B17302EB0313FF20DA7942
:10EEF000C2F34501013921EAE17161F34602DA7199
:10EF0000E076237E1B070BD51C4841F2C873C35C17
:10EF1000072B01D0FFF760FC41F2C8730022C254F6
:10EF2000E26A0023237084F82830FAB1BDE810406B
:10EF3000104700231249E0691A018A58904206D00E
:10EF400001330B2BBAD01A018A589042F8D10B4AE0
:10EF500003F5B17302EB0313DA79C2F3450101390A
:10EF600021EAE17161F34602DA71A7E710BD0121E0
:10EF7000FFF760FF0128F9D1237E9DE7E4660020BA
:10EF8000FC7C002030B1027822B190F828201AB120
:10EF9000002070470120704710B5D0E90142A2421D
:10EFA000C16238BF22460321826080F82810FFF733
:10EFB00079FF012010BD00BF2DE9F04FDFF8689107
:10EFC0008A4699F80010DAF800300229174683B013
:10EFD000834641F6300240F08B8059F80250DEB291
:10EFE000A6EB030805EB1325B8444FF48072904458
:10EFF000BB4208F1FF38B8FBF2F875D2A8440329E8
:10F0000006EB0704A4EB03040CBF80224FF48072CC
:10F01000944228BF1446A8EB050366B994422CBF5E
:10F020000A220B2201A92846FFF746FC012809D035
:10F0300003B0BDE8F08F0B2201A92846FFF73CFC86
:10F040000128F5D199F80020DAF80010022A01F120
:10F05000010321D0A64210D2019906F18042013A63
:10F06000081F00EB840001EB820242F8043F824259
:10F0700003F10103F9D1DAF80010A61B7318BBF1F4
:10F08000010FCAF800301BD09F4205F101052BD9B2
:10F0900099F800100026B2E7A642EED2DDF804C0CF
:10F0A00006F10042013AACF1020000EB44000CEB27
:10F0B000420222F8023F904203F10103F9D1DCE75A
:10F0C000BB42E1D199F80030022B21D004F18044F9
:10F0D000019B013C4FF0FF3243F82420DAF8003066
:10F0E0009F4205F10105D3D8012003B0BDE8F08FA0
:10F0F00059F8022003F07F060329C3F3D415A6EBC9
:10F1000003081544B84414BF4FF4807280226EE7A0
:10F1100004F10044019B013C4FF6FF72584623F86E
:10F12000142003B0BDE8F08FE46600202DE9F04123
:10F1300090F838300446032B51D8DFE803F0023250
:10F140003B462D4BC0681978E76A03F5C252032984
:10F1500011680CBF80264FF4807601FB06F141F266
:10F16000C47C00EB412041F2A87841F2AC7E53F818
:10F170000C20E06053F80E0053F808502261A5EB14
:10F180004125A0EB4121901943F8085043F80E1097
:10F1900043F80C00C4E90C205FBB6262012384F8D1
:10F1A000383016480021FFF745FE012811D102230F
:10F1B00084F83830626B04F130010120FFF7FCFE67
:10F1C000012806D1032384F8383000212046FFF7B8
:10F1D00031FE431EDBB2012B02D9BDE8F0810220D3
:10F1E00094F82830062B04BF002384F82830BDE8AB
:10F1F000F081921B2263D1E7E4660020847E002028
:10F200002DE9F04FDFF8248198F80060012887B0DD
:10F210008CBF00230123032E02930C460B68154676
:10F2200039D0022E62D14FF480724FEA1329DFB237
:10F2300001920138012823D8012203929D421AD954
:10F24000384E06F1880A06F11C0B32681AB1DBF859
:10F25000001099424ED0DAF80000002348440922F9
:10F2600005A9FFF729FB01281FD002280FD020B1E4
:10F2700023689D42E9D82560032007B0BDE8F08FE0
:10F2800087B1FFF7A9FA022007B0BDE8F08F02208E
:10F2900007B0BDE8F08F80220192C3F3D41903F0C8
:10F2A0007F07C6E7019A0392C8E7DDE902C1059A24
:10F2B000DDF804E098F80030022B14D0032BE6D1DF
:10F2C00052F8273023F07043B3FA83F35B096345A8
:10F2D0000F44236823D00B4477452360EAD309F118
:10F2E00001090027C5E732F81730EDE74FF48072C7
:10F2F0000192D2E70C490968013A02EB4122490226
:10F30000B2FBF1F203991344B3FBF1F201FB1232A9
:10F310000AB10B449B1A9D42236096D8ABE7AB42DF
:10F32000ABD3A8E78C7E0020247F0020E466002079
:10F33000F0B5104D2B7841F63002022B0BBF070AB7
:10F34000C0F3D417C4B200F07F04A85883B00E46AF
:10F3500000230322384401A9FFF7AEFA012807D1A0
:10F360002B78022B019B0CBF23F8146043F8246018
:10F3700003B0F0BDE46600202DE9F04390F83C3086
:10F38000002983B0044614BF02210021042B7BD83E
:10F39000DFE803F0030C3C476900FFF74BFD012851
:10F3A00070D1626B002A75D184F83C00404EDFF8C2
:10F3B0000881404D4FF6F7771DE01FFA80F9B945F7
:10F3C00094BF4FF000094FF0010901A9B9F1000FF6
:10F3D00046D1FFF789FB0128494650D1206BFFF742
:10F3E000A7FF01284BD1019B2A682363013B93426D
:10F3F00028BF13462B603378206B032BDDD14045AB
:10F4000094BF4FF000094FF00109DEE7426B04F1B1
:10F4100030010020FFF7D0FD012833D1032384F809
:10F420003C30234BE16A41F2C47003F5C2521D58CF
:10F430001268195041F2A87741F2AC76D8596D1A8A
:10F44000995902FB05F200EB422501EB422203F53C
:10F45000BD500021DD519A51FFF7ECFC012811D17C
:10F46000042384F83C3094F82830042B04BF002394
:10F4700084F82830A36B8BB120469847012003B055
:10F48000BDE8F0830228FAD194F82830042B09D083
:10F490000220F4E7022384F83C30B8E7012003B0EF
:10F4A000BDE8F083002384F828300220E7E700BF9E
:10F4B000E4660020287F0020F7FFFF0F38B590F8A2
:10F4C00034300446052B46D8DFE803F01F033F1015
:10F4D0001963006B4FF0FF31FFF72AFF01283AD183
:10F4E000E06A002839D1032384F834300021204613
:10F4F000FFF7A0FC01282ED1042384F8343094F8BF
:10F500002830082B2DD0012038BD41F63803224D7C
:10F51000EA5800F1300102320120FFF771FE0128A4
:10F5200024D00238C0B2012815D8052384F834301D
:10F5300094F82830082B04BF002384F8283041F2C7
:10F54000E5730122EA54022038BDC06A216BFFF73F
:10F55000EFFE0128C7D0002038BD022384F83430E4
:10F56000F4E7002384F82830012038BD05F5C252A5
:10F57000E3681168D4E90B2003EB412341F6440111
:10F580006850C4E9033002B96062012384F8343062
:10F59000A0E7014DCCE700BFE46600202DE9F04F65
:10F5A000436883B0C3F308081646002A00F0E180E0
:10F5B000714B05468946A3F1180B4FF0000AC8F5B8
:10F5C000007495F91A70B44228BF3446791C284655
:10F5D0002ED0F8F7C1FE0BEB071341F218629B58CF
:10F5E000984205D0FFF7F8F8504603B0BDE8F08F19
:10F5F000614B03EB472022464946404450F05EF9F8
:10F60000002221462846FFF729FBA2440028EBD020
:10F610002B7E1B0706D5594B2A691B689A4201D3DA
:10F62000FFF7DAF8361BA1444FF00008C7D1DBE73B
:10F63000F8F76EFE002849D12846F8F78DFE696874
:10F64000C1F308032BBB21F4FF7323F0010303F57F
:10F650000072AB689A422CBF062207222B7E03F071
:10F660000C030C2B1CD0002301A9FFF725F901285E
:10F67000BAD10198404BC31A48BF03F2FF13B3F548
:10F68000B05F4FEA63224FD257B2AF760028B2D1B3
:10F69000AAE72B7E03F00C030C2B4FF00702E2D1FC
:10F6A0009BF800C0364BBCF1030F1B680CBF4FF03A
:10F6B000800C4FF4807C03FB0CF34FEA432C0CF1DD
:10F6C000FF3C0CEA0101A3EB5123CDE72B7E1A0787
:10F6D0002ED59BF800102A4B95F828201B6803298B
:10F6E0000CBF80214FF4807103FB01F3062A4FEA1F
:10F6F00043233FF479AF23490868834230D891F817
:10F700003D30002B7FF470AF002A7FF46DAF6B6942
:10F7100085F83820062185F82810EB622846FFF787
:10F7200005FD012888D05FE7FFF756F80198ACE7A0
:10F73000154B1A78002A7FF457AF95F82820002A35
:10F740007FF452AF082185F8342085F82810D3F8CB
:10F750005F206B692846C5E90B32FFF7AFFEE0E793
:10F7600041F2E573012250460BF8032003B0BDE8D7
:10F77000F08F924638E700BFFC660020A87E00208C
:10F78000247F00208C7E0020C97E00202DE9F043DC
:10F7900090F8384083B00546032C00F2A180DFE8E2
:10F7A00004F0021A8B0BFFF789FE012811D0022802
:10F7B0000BD1032385F838302B6C002085F8280006
:10F7C000002B00F0898098470224204603B0BDE852
:10F7D000F08385F838002B78022B79D0414A6F6886
:10F7E00041F64803D3581F40C7F34F272846F8F780
:10F7F000B3FDDFF8F48006463F1A0AE0D8F800307F
:10F800005A1E91454AD2FFF7B5F908B9FEF7E4FF51
:10F810000136022201A900233046FFF74DF8BC193A
:10F8200001281FFA84F94FF400724FF000010446DA
:10F83000CBD1019850F0A3F8EB694FF40071284642
:10F84000002BDBD06B68002BD8D1019B4FF020320E
:10F850004FF02E0C1A605A6083F800C0C3F80720DE
:10F860004FF0100E6C6A1A625A6283F820C083F857
:10F8700021C0C3F8272083F80BE0EA6B5C83C2F356
:10F880000F4CC4F30F4483F82BE05A879C82A3F8F3
:10F8900034C0D8F800305A1E9145B4D3C3EBC353DB
:10F8A000590201F500712846FFF764F908B9FEF71F
:10F8B00093FF022385F838302B6C002285F828202E
:10F8C00063B1284698470124204603B0BDE8F08381
:10F8D0006F68C7F34F2789E7022476E7012474E7AE
:10F8E000002472E7E4660020247F00202DE9F04F19
:10F8F00090F8303089B00446042B00F2A880DFE88D
:10F9000013F0A900B20005008A00E800C64D41F6D8
:10F910001003EB5C002B40F09A80C44F04F11C09EB
:10F92000B84607F1380BBA4601AE32464946404662
:10F93000FFF70EFA012840F03F810198002800F0FF
:10F9400021810378E52B01D0002BEED1B84A821A31
:10F9500048BF02F2FF12B2F5B05F4FEA622380F0B7
:10F960006F811B01B34A13449A7B042A0CD041F2E5
:10F97000C86104266A5801326A5041F2CC615A606B
:10F980009E736B5801336B5041F60202AB565E1CFE
:10F9900009D003F5B17305EB0313FF26D979AE54F3
:10F9A0006FF30001D97141F603016B565A1C0ED05A
:10F9B00003F5B17305EB0313FF26DA796E54C2F336
:10F9C0004501013921EAE17161F34602DA71202231
:10F9D00000214FF0D4FF2346019A53F8311F586895
:10F9E0005060116019899B7A93721181019B627E2C
:10F9F000DA7205A844F0DCFABDF81430002B40F0B0
:10FA0000578144F28172019903200A82CB810A83D3
:10FA1000CB8284F83000237E980600F1D080204607
:10FA2000FFF736F92369002B00F0D580237E03F021
:10FA3000F70213F00403227640F0DB80122A00F074
:10FA4000E180002384F828302046E36A984709B013
:10FA5000BDE8F08F7548FFF71BF94FF6FF720123E1
:10FA6000228484F83030714F04F11C0501AE04F19A
:10FA70003109324629463846FFF76AF901282FD066
:10FA80000228E4D1684D41F60202AB56591C09D058
:10FA900003F5B17305EB0313FF20D979A8546FF375
:10FAA0000001D97141F603016B565F1C0ED003F5BE
:10FAB000B17305EB0313FF20DA796854C2F34501F3
:10FAC000013921EAE17161F34602DA71042384F815
:10FAD00030300020E36A2070984709B0BDE8F08F0D
:10FAE000DDF804800B2249464046B8F1000F00F0D3
:10FAF000AD8098F80030002B00F0A8804FF06BFF2D
:10FB00000028B6D1B8F81410B8F81A304A4A43EAB7
:10FB1000014312686362D8F81C30A3605202B3FB41
:10FB2000F2F102FB113109B113445B1AE36098F85A
:10FB30000B303D4D637641F60202AB565E1C09D098
:10FB400003F5B17305EB0313FF20D979A8546FF3C4
:10FB50000001D97141F603016B56581C0ED003F514
:10FB6000B17305EB0313FF20DA796854C2F3450142
:10FB7000013921EAE17161F34602DA71032384F865
:10FB8000303048E73B782D49022B4FF009025046B0
:10FB90009CD00B78002B99D1C1E905330A708BF802
:10FBA00000304A6B0B7351F8143CC1E90132FFF786
:10FBB000EDFD01283FF4B9AE022887D047E7E069A0
:10FBC0000023112205A9FEF777FE01283FF427AF95
:10FBD00009B0BDE8F08F237E19077FF532AF124AD6
:10FBE00041F2C873D15C00297FF431AF0721D154B1
:10FBF00027E70023E26AA16884F828302046FFF74F
:10FC00002DF824E7626AE06AA0630421C4E90233A4
:10FC1000C4E90B2284F83C30636384F828106362E3
:10FC20002046FFF735F812E7E4660020CC7E00207E
:10FC3000FC660020FC7C0020247F0020F47E002055
:10FC4000FEF7CAFD01986FF00F038BE6294D41F6D0
:10FC50000202AB56591C09D003F5B17305EB03132F
:10FC6000FF20D979A8546FF30001D97141F603013F
:10FC70006B565A1C0ED003F5B17305EB0313FF202E
:10FC8000DA796854C2F34501013921EAE17161F37F
:10FC90004602DA71237EDF067FF518AF1648FEF7BD
:10FCA000F7FF4FF6FF720223228484F830302EE6ED
:10FCB000124B05A9B3F9902702A844F0CDF99DF89D
:10FCC0000C309DF80D609DF80A509DF80B20BDF892
:10FCD00008109DF80E00DB0243EA461342EA451283
:10FCE000A1F2BC7143EA500342EA41229BB292B2B4
:10FCF00089E600BFE4660020CC7E0020E04C0020B6
:10FD00002DE9F04390F82830013B83B00446082BDE
:10FD100041D8DFE803F048054D525865406A43007A
:10FD2000384B4668056B41F6480103F5C2525F58EF
:10FD300013683740EA19B2EB432F4FEA432816D233
:10FD400058E02169207EFEF7F7FE012823D1256BBC
:10FD5000666823696361A5EB08053D444644F61BCC
:10FD6000019B6660A84525634F46236142D8204623
:10FD7000F8F7CEFA01AA81460028E2D06668A368A7
:10FD8000E26A9E4238BF1E460023A66084F82830EF
:10FD90000AB12046904703B0BDE8F083FFF7F6FCB8
:10FDA00003B0BDE8F083FFF7A1FD03B0BDE8F08329
:10FDB000FFF778F803B0BDE8F0830021FFF7DCFA25
:10FDC00003B0BDE8F0830121FFF7D6FA0128E2D1A4
:10FDD0000023216C84F828302046FFF7D3F8DAE7B7
:10FDE000FFF7A4F903B0BDE8F083FFF767FB03B0AA
:10FDF000BDE8F0832046F8F78BFA0028BFD12E44E7
:10FE00006660BCE7E4660020024BD3F8E8311B6A69
:10FE1000184700BFE04C002038B514460D46FFF7E8
:10FE2000F3FF4FF4007302682A600020236038BD9E
:10FE3000034BD3F8E80108B183691847704700BF46
:10FE4000E04C0020034BD3F8E80108B143691847A0
:10FE5000704700BFE04C00202DE9F04113B3124F72
:10FE600015460E4603EB020801E0FFF7EBFFD7F85B
:10FE7000E81100230C691A4631462846A04700289D
:10FE8000F3D1FFF7DFFF0028FBD00135A84506F5C9
:10FE90000076ECD1054BD3F8D038C7F828370020CE
:10FEA000BDE8F081004FF5E7E04C0020F819002094
:10FEB0002DE9F041FBB1114F15460E4603EB020848
:10FEC000D7F8E81100238C681A4631462846A04727
:10FED0000028F5D0FFF7B6FF0028FBD00135A84574
:10FEE00006F50076ECD1064BD3F8D038C7F82837A2
:10FEF0000020BDE8F081014FF5E700BFE04C002095
:10FF0000F819002008B5FFF79DFF80F0010040427E
:10FF100040B208BD002108B508463AF089F9FBF760
:10FF200099FEFFF78FFF0028FBD0044A044BD2F85C
:10FF3000D028C3F82827002008BD00BFF8190020EA
:10FF4000E04C002010B5074C606D40B13BF0B2F9B9
:10FF500094F8513013B180F00100C0B210BD0120FF
:10FF600010BD00BFF819002010B5FFF7EBFF0E4CD5
:10FF700048B194F82430032B10D8237E0133DBB230
:10FF8000072B237603D9002384F8243010BDD4F83E
:10FF9000D0386361012384F8243010BDE06D4FF444
:10FFA000807147F043FEE8E7F819002070B51D4C5A
:10FFB00094F82430042B06460D4608D0082B20D197
:10FFC000E36983422BD0F8F7B9FA022819D1206EE1
:10FFD0003AF01AF900213720F8F7ECFA29461720F1
:10FFE000F8F7E8FAA8B9A37E6BB971021920F8F7FF
:10FFF000E1FA70B90823C4E9076584F824300220C7
:020000040801F1
:1000000070BD012070BD31461920F8F7D3FA0028E1
:10001000F0D0F8F7D7F9FFF7A7FF032070BD022053
:1000200070BD00BFF81900202DE9F043644D91B078
:1000300006460F469046994695F82430042B0DD07D
:10004000082B07D1EB69B34200F0B680F8F776FAD7
:100050000228F1D0012011B0BDE8F083286E3AF0FB
:10006000D3F8AB7E002B40F0968071021820F8F791
:10007000A1FA002840F09A8095F82440F8F716FA83
:10008000082C0CBFFC22FE22E86D818940F2E93386
:100090000189013B11F0020F9BB249D093B28381D9
:1000A00040F2E9340389013C13F0010FA4B26FD090
:1000B000838995F86430002B42D001A804F0FEFC3F
:1000C000EB6DAA6E95F86C10506803970C334022C4
:1000D000029300234906CDE9083304920B934FF4B1
:1000E000806206930A934FF400730792019105937F
:1000F00004F022FDAB6E01A9586804F0F1FCAB6E70
:10010000EA6D59680B6843F001030B6093889BB25A
:1001100043F002039380012206230020C5E90389EE
:100120002F606E602A7285F8243011B0BDE8F0832C
:10013000002BADD13BF0E8FA95F86430002BBCD130
:10014000E86DBE4683894FF480724FF47A744FF69F
:10015000FF71BEF1000F19D01EF8013BB0F808C0C6
:10016000013C1CF0020FA4B217D09BB283814FF464
:100170007A74B0F808C01CF0010F04F1FF3311D0FD
:10018000013A8389C7D0BEF1000FE5D1FF23E5E72F
:10019000002C87D1CEE7314668E78C42DED13BF0B8
:1001A000B3FAB8E79CB28C42E3D1F8E7F8F70AF962
:1001B000FFF7DAFE03204EE7F8F778F9FC2263E751
:1001C000F81900202DE9F04F9E4C94F8506087B04C
:1001D000002E00F0C08194F82420DFF87092DFF840
:1001E0007082994F4FF6FF75531E082B00F29380D3
:1001F000DFE813F0A500CB005D019100800009004D
:100200000A019100F50094F86430002B40F025823B
:10021000E06D236894F808E0828903EB0E2C4FF41C
:1002200080714FF47A73BCF1000F00F0A2811CF8CA
:1002300001AB0289013B92079BB240F1D6811FFAC4
:100240008AF383814FF47A730289D20703F1FF3A6C
:1002500040F1D38101398289E5D10EF1010E5FFAB7
:100260008EFEBEF1020F84F808E051D1E06D838963
:1002700040F2E9330289013B12F0020F9BB200F019
:10028000B0810023838140F2E9330289013B12F0FF
:10029000010F9BB200F09E818389838940F2E9338C
:1002A0000289013B12F0020F9BB200F08F81002304
:1002B000838140F2E9330289013B12F0010F9BB2C6
:1002C00000F07E818389F8F7F1F800F01F0005281F
:1002D00000F08382FFF748FED4F80CA0BAF1000FBB
:1002E00000F0B5810022236961680120D04794F8AD
:1002F000242079E720684FF40071F8F7FFF801280F
:1003000000F08D81022800F09181002800F0D68154
:1003100094F82420531EDBB2022B00F22681D4F87D
:10032000D03861695B1AC82B00F21B81A2F1080664
:10033000B6FA86F67609304607B0BDE8F08F206E33
:1003400039F062FF00210846F8F734F98246F8F7E1
:1003500039F8BAF1010FDBD10023206E637639F052
:1003600053FF40F2AB110820F8F724F9052800F0FC
:100370007181012800F00081F8F724F8627E002ADC
:1003800000F02882022384F82430206E39F03CFFEC
:10039000637E022B0CBF4FF0804A4FF0000A002111
:1003A0003720F8F707F951462920F8F703F9824674
:1003B000F8F708F8BAF1000FAAD1637E022B00F01B
:1003C000918184F81AA0206E39F01EFF00210920C7
:1003D000F8F7F0F800283DD0F7F7F4FF98E74FF072
:1003E000080AF8F763F8FF2800F00A82BAF1010A58
:1003F000F7D16369D4F8D028FA33934288D2FFF753
:10040000B3FD94F82420EFE6F8F750F8FF284FF0FA
:10041000080A06D0BAF1010AEBD0F8F747F8FF282E
:10042000F8D1236A0022012B227640F2EF81E269A3
:1004300008210132013BC4E9072384F824100A464D
:1004400074E700BFF8190020006402400F64024006
:1004500000600240BF481021F8F750F8834600289A
:10046000BAD101217F20F7F7CBFD01288246B3D115
:1004700058460221F7F7C4FD002800F08D810128BD
:10048000AAD116213A20F7F7BBFD01308002A06205
:10049000F7F798FF206E39F0B7FE00210A20F8F731
:1004A00089F8002840F04E81032384F8243010217D
:1004B00002A8F8F723F800287FF42AAF9DF815303A
:1004C0009DF816109DF810209DF809009DF80AC0AF
:1004D0001B01DBB243EA111303F5FA636387DDF80E
:1004E000113001F00F0184F83C101BBA110902F021
:1004F0000F024CEA002084F8381084F839209DF867
:1005000008109DF80B206363039B2363A08584F888
:100510002E1084F82F20F7F755FFA37E73B9206EB5
:1005200039F072FE4FF400711020F8F743F882465C
:10053000F7F748FFBAF1000F7FF461AFE06D0421D7
:1005400047F074FB002204233046226284F82430F2
:1005500007B0BDE8F08F304684F8246007B0BDE8EE
:10056000F08FFFF701FD94F82420042A7FF4DEAE1B
:10057000E1E64FF0FF0A5CE6E06D4FF0040E838980
:1005800002A94FF47A734FF0FF0C028992073AD513
:10059000A0F80CC04FF47A730289D20703F1FF3A36
:1005A00038D5828992B209B101F8012BBEF1010E52
:1005B000EBD19DF80B30AB2B04BF02236376DBE657
:1005C000002B7FF478AE3BF09FF87CE6002B7FF4A5
:1005D00067AEF8E7002B7FF458AE3BF095F8E06D7E
:1005E0005BE6002B7FF446AEF7E7AB427FF421AE2B
:1005F0003BF08AF894F808E02FE61FFA8AF3AB4242
:100600007FF422AEF4E7013B9BB2AB42BDD13BF09D
:100610007BF8CEE71FFA8AF3AB42BDD1F7E76369F7
:10062000D4F8D02864339342BFF472AEF7F7CAFE11
:10063000FFF79AFCD4F80CA0BAF1000F07D0002203
:10064000104623696168D04794F82420CCE594F8DB
:100650002420C9E584F819A08EE6A36E5968DB69E9
:10066000494594BF4046384613F0005F00F086804D
:10067000D0F804C0DFF8E0E003EA0C0C1CEA0E0F2F
:100680003FF454AE03EA0E03C3600B68E06D23F041
:1006900001030B600389D90703D583890389DA072E
:1006A000FBD403899B07FCD503891906F9D48388F9
:1006B00023F002031B041B0C8380D8E50190F7F79D
:1006C00081FEE56801982076042384F82430002D0B
:1006D0003FF431AED4E900212369A84794F82420DF
:1006E000531E18E6206E39F08FFD51463A20F7F779
:1006F00061FFE16D82468B894FF0040E4FF47A73EF
:1007000002A84FF0FF0C0A89920727D5A1F80CC068
:100710004FF47A730A89D20703F1FF3B29D58A89FE
:1007200092B208B100F8012BBEF1010EEBD1BAF183
:10073000000F07D1F7F746FE029B1BBAC3F3807385
:10074000A37640E6F7F73EFEFFF70EFC94F8242070
:100750004AE500BF381A00207D0F7D0F013B9BB298
:10076000AB42D0D108463AF0CFFFBAF1000FE9D141
:10077000E0E71FFA8BF3AB42CCD1F3E7D0F800C02F
:10078000DFF8A8E003EA0C0C1CEA0E0F3FF4CEAD34
:1007900003EA0E03836078E704212C20F7F730FC8E
:1007A000032183464E20F7F72BFC0C21034636200D
:1007B0000193F7F725FC019B421C02339A400AFA89
:1007C0000BFAA2FB0A01420A42EAC152A262F7F7FF
:1007D000F9FD5FE684F82420A8E5E568D4F8D03870
:1007E0006361072284F82420002D3FF49FADD4E9F3
:1007F000002123690120A84794F82420531E8AE58C
:10080000F7F7E0FD042384F8243094E508D00423AE
:1008100084F82430F7F7D6FD94F82420531E7AE5A7
:10082000F7F78CFE02287FF473ADD5E57D0F7D0FC1
:1008300010B5002304220446194680F811211A46F7
:1008400003F0B4FE204604F017F8002010BD00BFEE
:1008500038B5134602250A46C0E94E3380F81151D7
:10086000002103F0A3FE002038BD00BFF8B50B78CF
:1008700013F060050C4606461DD0202D18D14A788D
:10088000FE2A45D0FF2A3ED14A88002A58D1CD8879
:10089000002D55D11B0653D4384B012103F6CC62F1
:1008A00083F8005F83F8EC1E1F2303F0A1FE00E035
:1008B00000252846F8BD4B780A2B4CD00B2B45D091
:1008C000012BF6D191F904308988002B48DB04F024
:1008D00053F82179294F304603F0EEFE02232179A7
:1008E0004022304603F01EFF97F8EC3E022B3CD02E
:1008F00094F90420002ADCDA012BDAD030460121F9
:10090000F8F7D8FBD5E70225FDF7AAF82846F8BD89
:100910004D88ADB9CC88012C12D11A0610D5174BD1
:10092000D3F8083F9B6998471549C0B281F89207F0
:1009300030B1224601F292713046FFF789FFB8E7E5
:1009400030460225FDF78CF82846F8BD0C4B4A8846
:1009500083F89327ADE70B490122FFF779FFA8E75A
:1009600001F07F0104F022F8B3E73046812103F063
:10097000A5FB002387F8EC3E9BE700BFF02A002090
:10098000E04C00207354002010B50C7814F0600483
:1009900013D0202C0AD14B78023B092B18D8DFE862
:1009A00003F01B21171717171717272E22490122AB
:1009B000FFF74EFF0024204610BD4B78062B24D0B5
:1009C0000A2BF3D01D4B8A78C3F89C27204610BD14
:1009D000FDF746F80224EEE719490122FFF738FF38
:1009E0000024E8E717490122FFF732FF0024E2E77D
:1009F0004B88124A1B0AC2F898370024DBE70F4BDA
:100A00008A78C3F894270024D5E74B881B0A222B49
:100A10000CD0212B04D021462246FFF719FFCAE74C
:100A2000CA880949092A28BF0922F6E7CA8807495E
:100A3000362A28BF3622F0E77C540020E04C002004
:100A40007854002074540020E2050020980500200E
:100A5000F8B50B7813F060050C46064611D0202D32
:100A600016D1CD88D5B11B062AD52A4620496078F3
:100A7000F7F760FBE2881E493046FFF7E9FE0025E4
:100A80000AE04B780A2B16D00B2B0ED0062B03D185
:100A90003046FCF7E5FF02252846F8BD02226078C3
:100AA0001144F7F747FB2846F8BD8B78E3B9114BA3
:100AB000C3F8A057F0E710490122FFF7C9FEEBE7A2
:100AC0000E4B4A780E4FC3F8282103230021C0E9BA
:100AD000E45580F8113107F6C8022B46C7F8C45810
:100AE0000D4603F085FDD7E7FCF7BAFFD4E700BF5A
:100AF000C0220020E04C002080540020880100200B
:100B0000F81900200B7803F00303012B03D0022B0C
:100B100004D0002070478B881BB935E78B88832B66
:100B2000FBD095E710B5114C94F8423C23B9104B1B
:100B30004FF480225A6110BD0E4A136823F0060359
:100B400013604AF075FE94F8423C002BEFD0D4F8C5
:100B5000483C9B68DB07EAD5D4F8442D136823F0A2
:100B6000030161F307031360E1E700BFE83B0020E6
:100B7000003C014010ED00E02DE9F04704460D4631
:100B80009046002144221E46089F4EF0F8FE0123A5
:100B90004FF6FF722676628384F828302B782E2B4E
:100BA0004CD02E4604F1310A307804F1390968B18D
:100BB0002E280BD03FF08CFEC0B20AF8010BCA45BC
:100BC00006F1010607D030780028F1D120200AF87C
:100BD000010BCA45F7D130782E2808BF707804F190
:100BE000380908BF013604F13B0A58B13FF070FEE6
:100BF000C0B209F8010FD14506F1010607D03078DF
:100C00000028F3D1202009F8010FD145F7D118F0C1
:100C1000100F14BF0323012384F819802370E762A7
:100C20002B782E2B26D16B7823BB0323204684F808
:100C30003030FEF75BFE2046BDE8F0876B78002B76
:100C4000AFD1114B41F2F47241F60C0041F2F07158
:100C50009A5818585958E26041F601026062A16042
:100C60009A5C627641F2E8729B5C2370E7622B78B3
:100C70002E2BD8D00023204684F83030FEF736FEE5
:100C80002046BDE8F08700BFE466002000000000B9
:100C9000D0F8E43510B504461B689847D4F8E83519
:100CA0009B689847002010BD08B5D0F8E435DB6993
:100CB00003B19847002008BD08B5042290F812112E
:100CC000D0F8E83580F8131180F81221DB689847D6
:100CD000002008BD10B5D0F8E83504461B699847D8
:100CE000032384F81231002010BD00BF70B44B788C
:100CF000012B26D00B784A6900EB83035C6D2568D5
:100D00002369D2B18A684A6102F07F0223F400238A
:100D100023F07F0342F4002213432361C378012BA5
:100D200004BF0B696361C5F3076363F07B0363F37F
:100D30001F652560002070BC70478A6802F07F0242
:100D4000E4E782694C691568136944B38E68B4425C
:100D50008CBF06F07F0404F07F0423F4002323F00B
:100D60007F0344F4002443EA040388BF4E61136107
:100D7000C378012B1DD0C5F3076464F07B0464F3D2
:100D80001F651560002BD5D14B69002BD2D00269AD
:100D90000878516B012383400B435363CAE723F464
:100DA000002323F07F0343F400231361C378012B56
:100DB000E1D10B780C6900EB8300C5F3076381690F
:100DC00063F07B0363F31F654C610020156070BC0A
:100DD000704700BF2DE9F0434B78012B30D00B78E2
:100DE0004C6900EB83035E6D356837691CB38B6813
:100DF0001C44013CB4FBF3F4C4F3090203FB02F30B
:100E0000C3F312034B61144643EAC44363F31C0764
:100E10003761C378012B04BF0B697361CB78012B59
:100E200044D0C5F3076363F07B0363F31F6535604C
:100E30000020BDE8F0838A680124C2F31203E3E7CF
:100E400091F800804E6900EB880EDEF818C0DCF8DF
:100E50000050DCF8107076B3D1F80890384A06EBF1
:100E60000904013CB4FBF9F402EAC444C6F31202DB
:100E70002243CC7807F060473A43012C174649D00B
:100E8000CCF81020C278012A55D00269516B03FAC0
:100E900008F30B435363C5F3076363F07B0363F30A
:100EA0001F65CCF800500020BDE8F0834B7973B388
:100EB00045F00055B5E707F0604747F40027CC78C8
:100EC000CCF81070C378012B2FD0012CE3D102692C
:100ED0009268D20554BF45F0005545F08055C5F3E2
:100EE000076262F07B0262F31F65CCF80050002BB2
:100EF0009ED1B0B203308010DEF8D04098D0CA68DE
:100F000052F8041B216001339842F9D190E745F073
:100F1000805586E764F35E77CCF81070C378012BB8
:100F2000D5D10A69CCF81420D1E70A69CCF814208D
:100F3000012CB0D1CBE70B69CCF81430ABE700BF84
:100F40000000F81F0E4BDA68D20310D4DA68D1061D
:100F50000FD4DA68D20510D4DA6812F0E00F0AD1A3
:100F6000DB6813F0020F14BF08200920704701202E
:100F7000704706207047072070470220704700BF67
:100F8000003C024000207047704730B1034B93F99A
:100F900000000028D4BF002001207047387F0020C7
:100FA00008B5FFF7F2FF50B1054A537892785B001D
:100FB00003F00203002A18BF43F001030B6008BDD1
:100FC000387F002008B5FFF7E0FF10B1014B5B68E8
:100FD0000B8008BD387F002070B5FFF7D6FF78B1D1
:100FE000084A158965B1D6680023B3421C4607DA62
:100FF00002EB44040133248AAC42DBB2F5D30B701C
:1010000070BD00BF387F002008B5FFF7BEFF10B1EC
:1010100000230B70137008BD0420704728B1034BE8
:1010200093F90000003818BF01207047180600200F
:1010300008B5FFF7F3FF48B1054B93F90020012AEB
:10104000C3BFDB78C3F340030B60002008BD00BFC3
:101050001806002008B5FFF7E1FF10B1014B9B789F
:101060000B7008BD1806002070B5FFF7D7FF30B130
:101070000D4CE378DB0703D500230B70137070BDB4
:101080000A4D94F9013095F8206093FBF6F3013393
:101090000B7094F9014095F8201094FBF1F301FBDB
:1010A000134301331370EAE718060020387F00204D
:1010B0000320704770B50A4A92F8243006255E1C5A
:1010C000B6FBF5F405FB146492F82550AC4205D04C
:1010D00002EBC303C3E90A0182F8244070BD00BFDC
:1010E000387F0020002230B504461046914200DCD3
:1010F00030BDA35C0825584010F0800F4FEA400334
:1011000018BF83F0D503013DD8B2F5D10132EDE728
:1011100010B5C9B10D4B986D814215DCA2B11B6AA7
:101120009A4211DC0A4C013A013903FB0121A173F7
:1011300004F10A000521FFF7D5FF0621E07304F151
:101140000A00BDE81040B5E710BD00BF387F0020A1
:10115000180600200023038083708380C3800372FD
:10116000704700BF074A084992F85C30097801339C
:10117000DBB2994282F85C3004BF002382F85C3015
:10118000704700BF387F0020C40B0010F8B5754CC5
:10119000236E83B1744B1B6893F82E305BB1734B95
:1011A00094F86420A3FB0013012A4FEA93132ED076
:1011B000022A08D002B1F8BD6D4B9842FBD9012339
:1011C00084F86430F8BDA26E64329A423BD894F839
:1011D0005C3004EB031393F87C20FF2A05D06549AB
:1011E0000132012083F87C200874FFF7BBFF624BBB
:1011F0001B780122092B84F86420DCD1B4F8FE307E
:101200005E4A01339BB2A4F8FE305380F8BD5C4DBA
:1012100094F85C105848A3668C2303FB01530078B4
:101220009A70002384F87A3004F170050A220223B0
:101230000928E56684F87B2084F86430BBD14F4BE5
:1012400001311980F8BD94F87A2094F87B309A42E5
:10125000B1D104F16F0004F17805002310F8012FDB
:10126000082153405A0013F0800F08BF5B0082F042
:10127000070214BFD3B2DBB20139F3D18542EDD1FD
:1012800094F879209A4238D194F85C6094F87750B9
:1012900094F87830B4F87300B4F8752094F871C0FD
:1012A00004EB061743EA052394F8725087F87C1084
:1012B00040BA52BA81B292B245EA0C202D4DC7F81D
:1012C00080101BB294F97010C7F88420032E4FF0E1
:1012D0000102A7F87E00A7F8883087F87D102A74ED
:1012E00008D8254A12780C2A28D00D2A02D1234B7F
:1012F00023F81610FFF736FF61E794F85C3004EB33
:10130000031393F87C20FF2A05D01A4901320120EB
:1013100083F87C200874FFF725FF174B1B78012208
:10132000092B84F864207FF446AFB4F8FC30134AEC
:1013300001339BB2A4F8FC309380F8BD1149124AE6
:10134000897E0E4803EB830303EB830349089B006C
:1013500093FBF1F382FB0312DB17C3EBA20320F82C
:101360001630C7E7387F00205C090010D34D6210AB
:101370003F4B4C0018060020A1260020A426002088
:10138000103E0020B8260020676666660A4B93F878
:101390007A1093F87B2091420DD010B493F87A2004
:1013A000DC6E511CD2B2C0B2C9B283F87A10A0541C
:1013B0005DF8044B70477047387F0020FD2870B5FA
:1013C00022D0F02804D0EF2822D00224204670BD7D
:1013D000114D0320052641282E444FF0000405F14D
:1013E000010580F080030DD0042B0BD9FFF7E6FF39
:1013F0002044B542C4B2E9D015F8010B412880F071
:101400008003F1D10420F3E7044D0B200426E2E72A
:10141000034D0C200626DEE72803060824030608F1
:10142000300306080E4B0F4AD3F80031B2F904001E
:101430005B0707D400EB8000400080B200F5C87065
:1014400080B27047084B094A9B6B323382FB031210
:10145000D817C0EBA20080B200F5C87080B2704708
:10146000387F0020C40B0010744200206766666657
:101470000C4AD2F8183130B41C68D2F810515D60B3
:1014800019810025611C19609D812070D2F81831E6
:10149000D2F810111A685A604FF6F67230BC196013
:1014A0009A817047387F00200E4B30B4D3F8BC22AD
:1014B000C3F8C02203F5CE7503F52B7403F58E70C7
:1014C00003F5D6710132C3E94554C3E9670030BC66
:1014D000C3E9AB11C3F8BC22C3F80C01C3F8101167
:1014E000704700BF387F002000B583B00268084B0A
:1014F0008188CDF801203222D3F8C432ADF805102E
:101500008DF800206846984703B05DF804FB00BFE3
:10151000387F00205E2810B511D05D2805D00D4B16
:10152000BDE81040D3F8C83218470A4CD4F8C83286
:101530009847D4F8C8323D20BDE810401847054C04
:101540005D20D4F8C8329847D4F8C8323E20BDE8B0
:1015500010401847387F002030B401234FF48075C5
:1015600015244FF4167140F2D932038000234580D0
:101570008471018130BC4281838083817047094B33
:10158000B3F8CE22B3F8CC32801A9B1AC00090FB7D
:10159000F3F00628A8BF062020EAE070C0F196000C
:1015A000C0B27047387F0020094B03EB4002B2F80D
:1015B000E612084A527C02EAD122520707D0D3F839
:1015C0005C23511CC3F85C13134483F86003704719
:1015D000387F00201806002010B5154A416892F89F
:1015E0009B3303F00303032B1FD1B2F89C33CBB121
:1015F000B2F99E33B2F9A4230A2492FBF4F29B1AA7
:101600001B0103F5B95314334FF4B472B3FBF2F377
:10161000C3F1080303F00F0360330B70436800222B
:101620005A7010BD05230B70F8E72D230B70F5E7FA
:10163000387F0020436872221A70436873225A7000
:10164000436874229A7043680022DA7070470F4B27
:101650004268B3F9A4330A2193FBF1F31B0110B5DF
:1016600003F5B9530A4C4FF4B4711433B3FBF1F3DF
:1016700003F00F03E118E35813604B6853600B7AD3
:101680001372436800225A7210BD00BF387F0020D9
:1016900036030608084B93F8AD3333B942F21073A2
:1016A0005843064B90FBF3F07047242358434FF404
:1016B0007A7390FBF3F07047387F002040D2060029
:1016C000054B93F8AD332BB94FF4A47358436423FF
:1016D00090FBF3F0704700BF387F0020831E00F1BD
:1016E0007402EA2123F8021F9342FBD143F6491307
:1016F0004385CD2383804E23C380CE2303812323C0
:10170000A0F872307047254A00234361D2F8BC1319
:1017100041F45C5130B541F02C010124C2F8BC13F6
:101720004471D2F8B41304FA03F50133112B41EAE2
:101730000501F8D14FF4206321F4F031C2F8B4135D
:10174000C38040F601230381154B0360142303710A
:101750008023037642F6140303824FF6FF7343831C
:1017600003F58C03C36140F20123038400230D4A77
:1017700080F8223080F8333080F844305023A0F8CD
:1017800056306FF07E43C0E916234FF0A063036626
:1017900040F61833A0F8643030BD00BF387F002019
:1017A00098086400C4FF00FF134B10B400220F24FC
:1017B00083F81214090A83F8110483F81314C3F888
:1017C0001424C3F81824C3F81C2483F8104403F528
:1017D0008260012110F8014F013122440E29D2B25A
:1017E000F8D183F81E240549D3F820045DF8044B92
:1017F000102235F0B1B900BF387F002048830020A7
:10180000054B002183F82414C3F82814D3F820349E
:1018100003B1C9E7704700BF387F002013B5044605
:10182000FFF7FCFBF0B100230DF106022046ADF8F6
:1018300006300DF04DFBA8B10B4C9DF8062094F935
:101840000010A275032908BF62F07F024FF0050166
:10185000064808BFA275FFF745FC0621E07503485E
:10186000FFF728FC02B010BD180600202A06002051
:10187000034B0449B3F918304068012245F082BD9A
:1018800018060020EB7906081E4A9FED1F7AD2F851
:101890003414B2F8A833406807EE901AF8EEE76AFD
:1018A00007EE903AF8EEE77A67EE877AF4EEE76AA9
:1018B000F1EE10FA02D8154945F064BD8B4202DA08
:1018C000134945F05FBD5B1A07EE903A02F5876356
:1018D000B8EEE77AD3ED007A0E4AF8EE677A3C214B
:1018E00067EE277A87EEA67AFDEEC77A17EE903A72
:1018F000B3FBF2F3B3FBF1F201FB1233064945F0FF
:1019000041BD00BF387F0020CDCCCC3D36770608E6
:101910003C77060840420F004277060806494068B7
:10192000B1F83C24D1F82C340449534342F21072EC
:1019300093FBF2F245F026BD387F00204C77060875
:10194000044A05495378127840680133013245F062
:1019500019BD00BF7C4500205177060837B51C4CE7
:101960004568D4F8002112F0200F02F0040328D0BB
:1019700094F89B23910724D5B4F94404FFF7A0FE03
:101980006421002890FBF1F301FB13014FF00A00E2
:1019900091FBF0F194F8AD03B4BF762275220029D3
:1019A000B8BF494200280CBF99209F20002BCDE9E9
:1019B0000010B8BF5B420749284645F0E3FC03B07E
:1019C00030BD002BD8D12D222A7042685370F6E723
:1019D000387F0020577706080B4B4068B3F9A433D3
:1019E0000A2293FBF2F31A0102F5B9524FF4B471D3
:1019F0001432B2FBF1F2C2F1080202F00F02034905
:101A0000603245F0BFBC00BF387F00206577060814
:101A100037B5194B456893F84624B3F83C14022AAD
:101A200004461AD093F84704B1FBF0F0FFF7A7FD86
:101A30002870B1F57A7F606811DB0A23062405312E
:101A40000094B1FBF3F10130B1FBF3F203FB12138D
:101A50000A4945F097FC03B030BD9720E8E76423BE
:101A60000624B1FBF3F2009403FB12130130044986
:101A700045F088FCEFE700BF387F00206C77060850
:101A800034B60608034A0449D2F8342440680723D0
:101A900045F078BC387F00207477060807B5114AF6
:101AA000406892F84A34B2F84814012B09D10091E9
:101AB00092F84B340C497B2245F064FC03B05DF88E
:101AC00004FB0A234B4340F2FF32B3FBF2F39BB219
:101AD000092B064928BF09237B2203B05DF804EBDC
:101AE00045F050BC387F00207A77060884770608D6
:101AF00013B51F49D1F8002112F0200204461AD074
:101B000091F84C2412F0010215D091F89B2312F0A9
:101B1000020210D0174BDB89632B20D96420584375
:101B2000FFF7B8FD00281ADDD1F82C344FF47A7293
:101B30005A4392FBF0F291F8AD336068002B02F14A
:101B4000FF3442F20E710CBF7E237D238C4208D8F5
:101B500000930949072345F015FC02B010BD00228F
:101B6000E9E70649072202B0BDE8104045F00ABC8B
:101B7000387F0020085300208A77060893770608EC
:101B800013B50D4A446892F857140C4B89B19889E3
:101B9000FFF780FD92F8AD230949002A0CBF9D2272
:101BA0009E22034600922046702245F0EBFB02B0D5
:101BB00010BDD889ECE700BF387F00200853002013
:101BC0004B78060830B5124A124B92F8022440684E
:101BD0001C7D85B0AAB10A215A8AB2FBF1F5B5FB8A
:101BE000F1F301FB13539BB202930B496423B2FB45
:101BF000F3F21F23CDE900421E2245F0C3FB05B0DE
:101C000030BD064900941F231E2245F0BBFBF6E7BA
:101C1000387F0020085300209D770608AB77060820
:101C20000C4B40685B689822002B10B402700EDAEF
:101C30002D2242705B4202240749B3FBF1F220449B
:101C400001FB12335DF8044B044945F09BBB0124B2
:101C5000F2E700BF0853002080969800B37706088B
:101C60000C4B40681B688922002B10B402700EDAFE
:101C70002D2242705B4202240749B3FBF1F220445B
:101C800001FB12335DF8044B044945F07BBB012492
:101C9000F2E700BF0853002080969800B37706084B
:101CA000044B93F84C34DB0703D40349406845F0F8
:101CB00069BB7047387F0020BB77060807B5094A23
:101CC0000949B2F906300193B2F904300093B2F930
:101CD00002304068B2F9002045F054FB03B05DF8D3
:101CE00004FB00BFA4260020C477060813B5094BE7
:101CF000D3F82C349A24002BB8BF5B4264210094A3
:101D0000B3FBF1F2406801FB1233034945F03AFBA3
:101D100002B010BD387F0020D877060837B5104ACA
:101D2000456892F84734B2F83C14B1FBF3F192F8ED
:101D30004634022B044611D00846FFF720FC2870D9
:101D4000606864230624B1FBF3F2009403FB1213D2
:101D50000130044945F016FB03B030BD9720EEE793
:101D6000387F002034B6060837B50378114A1A2B9D
:101D70000CBFB2F9A253B2F9A0530A211A2B95FB5A
:101D8000F1F408BF152201FB145118BF1422002DD5
:101D9000B4BF2D2320230029B8BF4942002CB8BF6F
:101DA0006442019100940449406845F0EBFA03B0A5
:101DB00030BD00BF387F0020E377060837B51E49E5
:101DC0004468D1F8002112F0200F02F0040329D05A
:101DD00091F89B23920725D5D1F85C04FFF770FC9E
:101DE0007F220A2390FBF3F309302270BCBF2D221F
:101DF000627091F8AD13B4BF02200120002BB8BF70
:101E00005B4200294FF00A050CBF0F210C21009105
:101E1000B3FBF5F2094905FB1233204445F0B2FA51
:101E200003B030BD002BD7D17F22227042682D2114
:101E3000517042689370F3E7387F002059770608A5
:101E4000084BD3F86024002A0ADD074B03EB82031A
:101E50009A6A2AB1054B0649DB69406845F092BA97
:101E6000704700BF387F00202403060818060020B2
:101E7000F177060807B593780193537800931378A8
:101E80000A46034945F07EFA03B05DF804FB00BF43
:101E9000F9770608024B03491A6840681432E9E7EB
:101EA0008453002008780608024B03491A684068EA
:101EB0000832DFE7845300200C780608024B034900
:101EC0001A6840680E32D5E784530020107806085F
:101ED00037B5044608461546FFF7F2FB02460DB13A
:101EE00004F8015B1A4B93F8AD33002B0BBF4FF492
:101EF000A5514FF47A717E207D200CBF0F230C2357
:101F0000914206DD1349204603B0BDE8304045F05C
:101F100039BA64235A43B2FBF1F1B1F57A7FB1FBD0
:101F2000F3F20DDB0A230090B1FBF3F12046B1FB85
:101F3000F3F503FB1513084945F024FA03B030BD4F
:101F4000009003FB12132046044945F01BFAF5E705
:101F5000387F00206F7706086C77060834B60608CD
:101F600010B40D49446891F89B3303F00303032B2D
:101F700006D12046B1F89C135DF8044B1122A7E767
:101F80001123237043682D225A70436800229A70EF
:101F90005DF8044B704700BF387F0020094A406855
:101FA00092F89B3303F00303032B06D1D2F8641499
:101FB00064237122B1FBF3F18AE703492D237122D7
:101FC00045F0E0B9387F0020147806082DE9F84F75
:101FD0001B4C05461E2094F868A494F869B494F844
:101FE0006A64B4F86C94B4F86E8494F870741FF05A
:101FF0000BFF30B1B8F1000F03D0C14601264FF0FE
:10200000000A94F84C34DA070AD494F877243AB9E1
:10201000012F12D0022F03D113F0020F08BF0126A7
:1020200085F800A085F801B0AE70A5F80490A5F879
:1020300006802F722846BDE8F88F3E46F0E700BFC5
:10204000387F00202DE9F84F2DED028BFEF7E6FFDB
:10205000002844D0264B93F9000001283FDD93F877
:102060002040DFF894809FED238A0FF27C0BDBE9A0
:1020700000AB15468E1E02EB44094D4504D1BDEC64
:10208000028B2046BDE8F88F38F8027B26F8027FE5
:1020900007EE907AF8EEE77A67EE887A17EE900A04
:1020A00049F0D2FD52465B4649F026FE41EC100B4A
:1020B0004DF096F951EC100B4AF046F90E2F80B214
:1020C0000AD919303223B0FBF3F080B200EB800064
:1020D00000EB8000400080B225F8020BCDE7002421
:1020E000CDE700BFAFF300801655B5BBB16B024022
:1020F00018060020CDCCCC3DD483002038B50D4649
:10210000FEF78CFF044628B10B48C378DB0703D5E4
:1021100080882880204638BD084A90F9013092F81E
:10212000202093FBF2F102FB113201320131243005
:102130000CF0E2FEEDE700BF18060020387F00201B
:1021400038B5134C94F8253094F824209A4219D0CD
:1021500004EBC3030F49D3E90A200023984212DCA1
:1021600093780D4AC4F8AC045B081370FBF746FC87
:1021700094F8253006210133B3FBF1F201FB123351
:1021800084F8253038BDD55C01F8015B0133E5E703
:10219000387F0020C4530020F2530020F0B52C4CAF
:1021A000D4F8B05494F8681487B0074628460CF069
:1021B0000BFF94F86914064628460CF0F1FE002245
:1021C000059294F86A248DF81320034675B10390A4
:1021D00005A928460CF00AFF94F87024039B2AB145
:1021E0000DF1130128460CF007FF039B9DF8132007
:1021F000DDB1D2B1E1688A4217DC04EB8204D4F885
:10220000B444039326201FF0FFFD0599039B70B98A
:1022100011F0010F14BF502200228907786808D5F9
:102220000C4945F0AFF807B0F0BD0B4CE9E744228C
:10223000F3E732B1CDE900420849324645F0A2F851
:10224000F1E707490094324645F09CF8EBE700BF00
:10225000387F0020197806082D84060821780608A2
:102260002D7806082DE9F04FA84B1B788BB08146DE
:10227000002B40F0B480A64DD5F8B064002E00F0DD
:10228000AE80A44A946A04F0F021B1F1E02F6DD140
:102290009362D5F8D824944268D004930593ADF89E
:1022A0001830B5F86C3495F868E4ADF8143095F84A
:1022B00069C495F8703495F86AA48DF818300DF15A
:1022C00010088DF810E08DF811C08DF812A098E874
:1022D000070007AB03C3904F1A80C4F342533B443B
:1022E000C4F3034293F8B010C5F8D8448E4502F108
:1022F000010201D1944508D030468DF81C108DF8AC
:102300001D200CF0F9FDADF8200030460DF022F94B
:10231000032804F0070B34D0042836D000239A4554
:1023200001A9304618BF8DF81E300CF05FFE48B191
:10233000019BC4F3001103F001038B4202D030462D
:102340000CF0FAFF0A2207A940464DF0F0FA68B1F6
:102350009DF81E30BDF81C2085F86A34BDF8203089
:10236000A5F86824A5F86C343DF056FC95F8DCA47B
:1023700004AF95F8DC34032B7BD8DFE803F00A3395
:1023800076A35F4497F8B530C9E75F4497F8BD304E
:10239000C5E7394630460CF02FFE044658B107A871
:1023A000FFF714FE9DF81E109DF810308B4260D090
:1023B00030460DF037F895F8DC34013303F00303B1
:1023C00085F8DC340CB99A45D3D195F84C34DB0749
:1023D00000D524B1336849461B68304698470BB096
:1023E000BDE8F08F01A8FFF7F1FD95F84C849DF84A
:1023F000044008F00108ECB1B8F1000F39D13A46B9
:102400000DF1030130460CF0FAFD044688B307A82D
:10241000FFF7DCFD9DF81C109DF803309DF81D2092
:102420008B4203D19DF81030934222D030460DF0FC
:1024300003F8C0E7B8F1000FBDD1394630460CF0C3
:10244000D8FD0446A8B107A8FFF7C0FDBDF82010CD
:10245000BDF810308B420CD085F8DD8485F8DE8421
:10246000336830469B699847A5E795F84C34D80700
:1024700001D500249FE707A930460CF0B7FD0446BC
:102480000028F6D01E201FF0BFFC95F8DF348342F1
:102490008046EED085F8DF0460B1B5F86E34002BCD
:1024A000E7D1079BD907E4D4012130460CF044FF63
:1024B000444680E7079BDA07DBD5014630460CF03F
:1024C0003BFF78E73846FFF781FD97E8070007AB49
:1024D00003C31A809DF810309BB10DF11D0207A9AE
:1024E00030460CF08CFD0DF11E0130460CF084FDE1
:1024F0000A2207A938464DF01AFA041E18BF012413
:1025000059E708A930460CF074FDECE710540020A0
:10251000387F00201806002024030608024B0146DD
:10252000D3F8E00434F04CBB387F00202DE9F041B3
:10253000FD2984B0044600F0DE80F02900F0BD8063
:10254000EF2900F031814AB10346861803AD00201F
:1025500003F8010B9E4205F8010BF9D19A4B0B20B1
:1025600003F1090501E013F8010F814200F0C88072
:10257000AB42F8D14B1E832B00F29380DFE813F0BF
:102580003201390143014E01BE018400580163014B
:102590006F01910091007501750175018B018B012F
:1025A0008B016F019100910096019E0191009100B5
:1025B0009100910091009100910091009100910093
:1025C0009100910091009100910091009100910083
:1025D0009100910091009100910091009100910073
:1025E0009100910091009100910091009100910063
:1025F0009100910091009100910091009100910053
:10260000B40191009100910091009100910091001E
:102610009100910091009100910091009100910032
:102620009100910091009100910091009100910022
:102630009100910091009100910091009100910012
:102640009100910091009100910091009100910002
:1026500091009100910091009100910091009100F2
:1026600091009100910091009100910091009100E2
:1026700091009100910091009100910091009100D2
:10268000910091001F011F01504BB3F8D81200298F
:1026900000F0668101922BF033F9019A80B2ADF817
:1026A0000C003AB1224403AB13F8011B04F8011BE0
:1026B000A242F9D104B0BDE8F081454F03214FF0AB
:1026C0000508B844002501370CE0FEF777FE064602
:1026D00060193246FFF72AFF70194745C5B2E9D0A5
:1026E00017F8011B412981F08003084601D0042B13
:1026F000EBD80426ECE7374F0B214FF00408E0E756
:10270000324BD3F8000180060CD4002AD2D02244E8
:1027100003AB13F8011B04F8011B9442F9D104B078
:10272000BDE8F08193F89B03870742D52A4D287DA9
:10273000052834BF02260326142917D97C39C8B2CC
:102740000628E2D80629E0D801A050F821F000BF01
:102750003929010839290108232901080B27010813
:1027600049290108432901084F2901080929CCD921
:102770000A390A29C9D801A757F821F009290108FF
:10278000552901080B2701080B2701080B27010811
:102790000B2701080B2701080B2701080B2701084D
:1027A0001B290108392901080C4F0C214FF006089C
:1027B00087E7094B0B29187DA7D10126CBE0084BF1
:1027C0005B6B03936DE700BFEC030608387F0020C6
:1027D00028030608240306080853002030030608CF
:1027E000744200200192FEF71DFE019AADF80C0024
:1027F00057E76C4BD3ED037AFDEEE77A17EE903A8C
:10280000ADF80C304DE7684B93F8EF04B3F83C1487
:10281000002840F0AB80ADF80C1042E76249B1F8F7
:102820003C3491F84714B3FBF1F3ADF80C3038E7C2
:102830005D4D95F84C34DE0700F19D80B5F8D83237
:10284000ADF80C302DE7584B5849B3F9A43381FB50
:102850000301DB17C3EBA103ADF80C3021E7524BAA
:10286000B3F84434ADF80C301BE7514BDFED516A3F
:10287000D3ED027A0C39C9B203EB810393ED167ADA
:1028800067EEA67A67EE877AFDEEE77A17EE903A62
:10289000ADF80C3005E7444B03EB4101B1F882334E
:1028A00003EB83035B00ADF80C30FAE63E4B93F884
:1028B0004C3403F00103ADF80C30F2E63A4BB3F8B8
:1028C0001815CD055ABFCB4303F00103032311F0C4
:1028D000440F18BF042311F0020F18BF072311F48F
:1028E000806F18BF0923ABE70192FEF79BFD324BC7
:1028F000019ADB6B43EAC0400390D2E62A4BD3F83F
:102900002C34ADF80C30CCE62B8A03EB830303EBBD
:1029100083039B00ADF80C30F7E6EB89ADF80C3083
:10292000F3E6EB89254903EBC3039B00A1FB0313EB
:102930005B09ADF80C30E8E6B3F89C33ADF80C3029
:10294000E3E66B680393E0E62B680393DDE6AB6890
:102950000393DAE6F6B28DF80C608DF80D00D4E63C
:10296000D3F8340480F3100080B298E693F847342B
:10297000B1FBF3F14FE705F5A16501921FF056FC9D
:10298000D5ED037A019AFCEEE77A17EE903A9BB206
:1029900000287FF455AF0A49096811F0100F18BFDD
:1029A00000234DE740840020387F0020676666667C
:1029B000C40B001000007A44744200201F85EB51C4
:1029C000E451002070B5214D95F81A35EA181C46DF
:1029D00092F81C258AB11E4E09225C1CA6FB04132A
:1029E0005B0803EBC303E31AE918DCB291F81C158A
:1029F00009B1013AF1D185F81A4502681549561C0A
:102A000006600C2616700268561C066000261670BA
:102A10000268561C066003EB430603EB8603147042
:102A200019440D223CF032FB95F81A15084B4A1C4C
:102A3000A3FB02035B08294403EBC3030120D31A61
:102A400081F81C0585F81A3570BD00BF387F00205D
:102A5000398EE338608400200A4B93ED000A10B5EC
:102A6000F2EE047A20EE270A04464AF023FC0A23F9
:102A7000054990FBF3F203FB12036068BDE81040C8
:102A800044F080BCD884002036780608084B93F8C0
:102A9000AD3307EE900A4BB9F8EEE77A9FED057A71
:102AA0009FED050AA7EE870A4AF004BC704700BFF5
:102AB000387F00206766E63F000000420D4B1B6830
:102AC0001B0137B514D50C4C4568D4F8A43593F9DF
:102AD0000100FFF7DBFF94F8AD230849002A0CBF83
:102AE0000D220E220346009228467A2244F04AFC28
:102AF00003B030BDE4510020387F00204178060843
:102B000037B50A4C4568B4F9A805FFF7BFFF94F83C
:102B1000AD230749002A0CBF0D220E220346009266
:102B200028467A2244F02EFC03B030BD387F0020C6
:102B30004A780608032815D8DFE800F00F02060AD5
:102B4000094BD3F838047047074BD3F8AC057047EE
:102B5000054B93F84C24D20701D433F0B7BAD3F81D
:102B60003804704700207047387F002073B52B4E23
:102B700006EB43030446B3F8AE5305F00F0049B12A
:102B8000022804F101011DD8002814BF9C239B23B7
:102B900023700C460AB3C5F30315FFF7CBFF3C21A6
:102BA000012D1F4BB0FBF3F3B3FBF1F201FB12332A
:102BB00015D0022D23D01B49204602B0BDE870403D
:102BC00044F0E0BB032806D196F84C3403F001032F
:102BD000653BDBB2DCE72023DAE71546DDE7642559
:102BE00042F21071B0FBF1F1B1FBF5F005FB1010F2
:102BF00000900D49204644F0C5FB02B070BD0A2587
:102C00000A49B0FBF1F1B1FBF5F005FB10100090A3
:102C10000749204644F0B6FBEFE700BF387F0020AD
:102C200040420F004277060853780608A08601004C
:102C300062780608037840680122053B114695E753
:102C40002DE9F041684ED6F8B07484B00446384699
:102C50000D460CF07FFC86F8D40557B10DF1090242
:102C600002A938460CF0CBF9002840F08E8096F887
:102C7000D4050023ADF808308DF80A301A46431EFB
:102C8000DBB20021FF20FD2B8DF80C20ADF80E10DB
:102C90008DF80B0003D9002004B0BDE8F0819DF849
:102CA0000830042B00F09680052B00F09980032B50
:102CB00000F09880022B00F08C80012B08BF0421CB
:102CC00000F088809DF809309DF80A10D6F8B0040D
:102CD000013B0DF10E028DF809300CF0F9F896F871
:102CE000D435032B73D0042B0CD1404A9DF80A0035
:102CF0000121002301E012F8011F81426DD201334E
:102D0000082BF8D1D6F8D825029B394F9A420DF1FD
:102D100008084FD023680D22591C21601A702368BF
:102D20000022591C21601A7023689DF80820591C44
:102D300021601A7023689DF80920591C21601A70BF
:102D400023689DF80C20591C21601A7023689DF897
:102D50000A20591C21601A70BDF80E1020463CF064
:102D6000DDF923689DF80B20591C216020461A705C
:102D70000721FAF719F898E8030087E80300012013
:102D8000C6F8E05504B0BDE8F08101A938460CF062
:102D90002DF900283FF46BAF38460DF10A010CF015
:102DA0002BF900283FF463AF019B96F8D40503F09C
:102DB000010264E77A68D8F804309A42AAD1D6F8BA
:102DC000E0350C4AEB1A93427FF665AFA2E70A4A58
:102DD0008CE703218DF8081074E78DF80A3091E72D
:102DE0000121F7E70221F5E7387F0020E10306081B
:102DF0001085002080841E00D90306082DE9F041CB
:102E00002A4C2B4AD4F82C34B4F8E475B4F8346462
:102E100082FB0352DB17C3EBA2031FFA83F847457B
:102E200082B00D4603D1B4F8E635B34233D0026820
:102E30000190511C34230160137002680023511C5F
:102E40000160137041463CF069F9019831463CF04D
:102E500065F9019847F6FF713CF060F9019847F673
:102E6000FF713CF05BF9019847F6FF713CF056F9B1
:102E7000019847F6FF713CF051F901980221F9F7EA
:102E800093FF0120A4F8E485A4F8E665C4F8E855AA
:102E900002B0BDE8F081D4F8E835064ACB1A934277
:102EA000C5D8002002B0BDE8F08100BF387F002007
:102EB0006766666680841E00026810B57F21541C18
:102EC0000460117002680024511C01600E2114700E
:102ED000F9F76AFF012010BD2DE9F04FC24B1B68C6
:102EE000804613F0800083B000F07181BF4B93F8EF
:102EF0009B0310F0020000F06A81DFF810B39BF82A
:102F00001430052B40F26881DBF80030B84D009397
:102F1000002BB8BF5B42A5FB0342B648B649920DF1
:102F200000FB0233C3EB03139B0085FB034502EB5D
:102F30008202DC1702EB8202C4EBA55400FB0433CF
:102F400004EB8204A4B281FB0321DB17C3EBA111C4
:102F5000BCB10025A94F2E46A7FB0432D20802EBD4
:102F60008203A4EB4303E8B2A4469BB280008340F3
:102F7000BCF1090F94B246EA030605F10105EBD84E
:102F8000340489B2B9B100259C4F2E46A7FB01320B
:102F9000D20802EB8203A1EB4303E8B28C469BB25A
:102FA00080008340BCF1090F91B246EA030605F1A7
:102FB0000105EBD83443DBF804E08D4D8D4E8E498E
:102FC0008EEAEE70A0EBEE70A5FB0032920D06FBD0
:102FD0000200C0EB0010830085FB035002EB82026D
:102FE000DD1702EB8202C5EBA05506FB053305EBAE
:102FF0008205ADB281FB0321DB17C3EBA111C5B183
:103000000020DFF8F8C10646ACFB0532D20802EB1F
:103010008203A5EB4303C7B2A9469BB2BF00BB40E6
:10302000B9F1090F95B246EA030600F10100EBD8A9
:10303000350489B2C1B10020DFF8C0C10646ACFB3F
:103040000132D20802EB8203A1EB4303C7B28946E7
:103050009BB2BF00BB40B9F1090F91B246EA03062B
:1030600000F10100EBD83543DBF80830634A0193E7
:10307000002B1846B8BF5842A2FB0030604E614991
:10308000030AA6FB0363DB0901FB03F1C1EBD001DB
:1030900089B2B9B1002691463746A9FB0132D20860
:1030A00002EB8203A1EB4303F0B28C469BB280009B
:1030B0008340BCF1090F91B247EA030706F101060C
:1030C000EBD8B9B2BBF81070DFB10026DFF82CA145
:1030D000B446AAFB0732D20802EB8203A7EB4303F4
:1030E0005FFA86F938469BB24FEA890903FA09F379
:1030F000092897B24CEA030C06F10106E9D81FFA39
:103100008CF7BBF812303D4AA2FB0306F608632E8B
:1031100028BF6326092B63D9002093468146ABFB69
:103120000632D20802EB8203A6EB43035FFA80FA71
:10313000B4469BB24FEA8A0A03FA0AF3BCF1090FBC
:1031400096B249EA030900F10100E8D85FFA89F96B
:10315000009B019A002BCCBF392338231616BEF1F1
:10316000000F26F07F0635DD274A3343964543F0AE
:103170000206C8BF43F00606D8F800301622581CD5
:10318000C8F800001A70D8F800300022581CC8F89F
:1031900000001A7040463BF0C1FF214640463BF01C
:1031A000A5FF294640463BF0A1FF404639463BF08B
:1031B000B5FFD8F800305A1CC8F8002083F80090FA
:1031C000D8F800305A1CC8F8002001201E7003B047
:1031D000BDE8F08F1E43CFE7002003B0BDE8F08FBD
:1031E0004FF00009B4E700BFE4510020387F002011
:1031F0006BCA5F6B806967FFD34D6210CDCCCCCCBE
:10320000C55A7C0AA0860100FFC99A3B08530020DA
:103210002DE9F047AB4B1B68064613F0800084B0E5
:1032200000F09E80A84B93F89B0310F0020000F082
:103230009780A64F397D052940F29780632900F2D7
:1032400092800024DFF898C289B22546ACFB013297
:10325000D20802EB8203A1EB4303E0B28E469BB29D
:1032600080008340BEF1090F91B245EA030504F1E5
:103270000104EBD8EDB2BB68954A82FB0312D91763
:10328000C1EB623189B2002900F018814FF0000CC7
:10329000DFF84CE26446AEFB0132D20802EB820357
:1032A000A1EB43035FFA8CF088469BB28000834019
:1032B000B8F1090F91B244EA03040CF1010CEAD809
:1032C000E4B2FB8983494FF4F36707FB03F7A1FBE3
:1032D0000737C7F38F1742F20F739F4249D8CFB118
:1032E0000020DFF8FCE18446AEFB0732D20802EB97
:1032F0008203A7EB4303C1B2B8469BB289008B405F
:10330000B8F1090F97B24CEA030C00F10100EBD8B9
:103310001FFA8CF7704BD3E9002313433ED14FF0D3
:10332000FF3833681722591C31601A703368002245
:10333000581C306039461A7030463BF0EFFE41466B
:1033400030463BF0D3FE33685A1C32601D70336840
:103350005A1C326030461C700621F9F725FD012009
:1033600004B0BDE8F087992585E7002004B0BDE8EA
:10337000F0870021DFF868C10F46ACFB0302D208DA
:1033800002EB8200A3EB40039BB28B400431102977
:1033900047EA030793B2F0D1BFB2BBE701A840F000
:1033A00007FE9DF80810002900F08A804FF0000CFD
:1033B000DFF82CE1E046AEFB0132D20802EB8203DB
:1033C000A1EB43035FFA8CF089469BB280008340F7
:1033D000B9F1090F91B248EA03080CF1010CEAD8DF
:1033E0004FEA08289DF80910E1B10020DFF8F0E06D
:1033F0008446AEFB0132D20802EB8203A1EB430309
:103400005FFA80F98A469BB24FEA890903FA09F309
:10341000BAF1090F91B24CEA030C00F10100E8D8AF
:1034200048EA0C089DF80A104FEA0828E1B100208C
:10343000DFF8ACE08446AEFB0132D20802EB820337
:10344000A1EB43035FFA80F98A469BB24FEA8909F0
:1034500003FA09F3BAF1090F91B24CEA030C00F137
:103460000100E8D848EA0C08BDF80C301B49632B72
:10347000A1FB03214FEA08184FEA51117FF651AF23
:103480000020DFF85CE08446AEFB0132D20802EB9C
:103490008203A1EB43035FFA80F98A469BB24FEAAD
:1034A000890903FA09F3BAF1090F91B24CEA030C46
:1034B00000F10100E8D848EA0C0832E70C4600E7C2
:1034C00088468FE7E4510020387F00200853002011
:1034D00089B5F814D34D6210288500201F85EB5163
:1034E000CDCCCCCC08B5A0F10103B3FA83F302280C
:1034F0004FEA531301D0184608BD0F201EF0FCFB05
:1035000030B9064B93F84C3403F00103184608BD5C
:10351000BDE808400F201EF077BC00BF387F0020B8
:1035200038B5224D4468B5F818355A0505D52046FA
:103530001F49BDE838404CF046BA180505D520466D
:103540001C49BDE838404CF03EBA590605D5204626
:103550001949BDE838404CF036BADA0705D520469F
:103560001649BDE838404CF02EBA9B0705D52046D9
:103570001349BDE838404CF026BA25201EF044FC23
:1035800028B120460F49BDE838404CF01CBA95F8E8
:10359000F8352BB120460C49BDE838404CF013BA41
:1035A00020460A49BDE838404CF00DBA387F00206B
:1035B00071780608767806087B7806088078060811
:1035C000857806088A7806088F78060894780608B1
:1035D000074B93ED1A7AD3ED1B7AB4EEE77AF1EE4E
:1035E00010FA03DD034940684CF0EDB9704700BFA5
:1035F000C40B0010A582060810B5044621F094FB08
:103600000349034604226068BDE8104043F0BABE97
:10361000EB790608F8B50446274B4178827893F891
:10362000C90323780138302B244B4FEA8000034430
:1036300023480BBF93F8D25093F8D45093F8D3603B
:1036400093F8D56030F9153030F9160040F2CF7597
:10365000AB42A8BF2B46B3F57A7FB8BF4FF47A735D
:10366000A8424FF47A77A8BF2846A3F57A73B842E8
:10367000C3EB0313B3FBF7F3C3F10E03B8BF384634
:10368000DBB24FF0030CB3FBFCFC0CEB4C0EA3EBDA
:103690000E03A0F57A706244C0EBC0000833B0FBA3
:1036A000F7F73944DBB2D2B2C9B22046FAF79AF939
:1036B00000232373F8BD00BF387F002024030608D1
:1036C0009C5300202DE9F04790F8029090F801807B
:1036D00009F1020704460026FFB2002508EB060A9E
:1036E000032E1BD108F10301022DC9B20ED10B2309
:1036F0003A462046FAF776F90135052DF0D1013624
:10370000072EEAD100232373BDE8F08709EB0502F9
:103710001623D2B22046FAF765F9EDE7022DEBD178
:1037200017233A465FFA8AF12046FAF75BF9E3E796
:1037300070B504466FF00205A278617852FA85F2FE
:1037400007391323D2B2C9B22046FAF74BF9A2784F
:103750006178EEB2324407311323D2B2C9B22046A7
:103760000135FAF73FF9042DE6D16178A2780639E0
:103770000323C9B22046FAF735F96178A2780631F9
:103780000223C9B22046FAF72DF90023237370BD36
:103790002DE9F8432B4A054692F8B91392F8C7036E
:1037A000B2F9A04392F8B833002801EB810114BFAD
:1037B0004FF0FF30012049004443C1F1000803EB02
:1037C000830344454FEA430303DB8C42A8BF0C4606
:1037D000A046B2F9A2235C424243A24203DB9A42D2
:1037E000A8BF1A4614461BB11922544394FBF3F4A4
:1037F000293C4FEA88066FF003074FF00909002EB5
:103800003346B8BF06F13F03C4EBA313512B0FD8C7
:1038100093FBF9F101EBC1029B1AAA780A4469787B
:10382000803B3944DBB2D2B2C9B22846FAF7DAF8A3
:103830000137052FA6EB0806E1D100232B73BDE865
:10384000F88300BF387F002010B5044613F06AFCEF
:10385000642202FB00F3C3F38F23632B60680449E7
:10386000BDE8104028BF6323012243F08BBD00BF99
:10387000AD770608F8B5194D064600241CF0CEF8C1
:10388000882705F1740C2B787168A342214402DC6F
:1038900000230B70F8BDF8B1D5ED1C7AFDEEE77A88
:1038A0000CEB840317EE90EAD3ED007AFDEEE77A95
:1038B00017EE902AD5ED257AFDEEE77AA2EB0E02FF
:1038C00017EE903AD200A3EB0E0392FBF3F3C3F191
:1038D00088030B700134D6E70F70FBE7C40B0010B0
:1038E0001F4AB2F8D832D2F8342413B50446D3B103
:1038F0009A1A9A42A8BF1A4622EAE27207EE902A62
:103900000B22B3FBF2F300EE103AF8EEE77AB8EED2
:10391000C00A87EE800A49F087FCFCEEC07ACDED44
:10392000017A9DF8043062688A2111700122616871
:103930009342ACBF8B208D20885401320C2AF6D1E3
:1039400062688F2111735A1E092A03D862681344D2
:103950008E225A70636800225A7302B010BD00BFF5
:10396000387F002010B5044613201EF04DFA50B3E6
:1039700010F092FF30B960681349BDE81040102282
:1039800043F000BD114B60689B78022B15D1104AA3
:1039900041F2E573D35C2BB1BDE810400D49102214
:1039A00043F0F0BC0C4BD3F80C36002B05DBBDE824
:1039B00010400A49102243F0E5BCBDE81040084918
:1039C000102243F0DFBC10BD99780608FC5300209C
:1039D000E46600209D780608387F0020A17806085C
:1039E000EBB9060870B52D4D0A24B5F9A02392FB5A
:1039F000F4F484EAE473A3EBE4739BB25A2B064617
:103A000005D90A32CCBFB4236FF0B3031C1B95F861
:103A1000143633B995F84C34DB0729D41CF060F820
:103A200030BB95F81C36B32B02D81CF059F8F8B906
:103A3000B5F9A2130A2391FBF3F304B9C3B1002B28
:103A4000B8BF5B4284EAE4709BB2A0EBE470B3EBD6
:103A5000400F726813DAB0EB430F10DA092908DD62
:103A6000002CCCBF6E2362231370736800225A703F
:103A700070BD002CCCBF6A2366231370F5E7834228
:103A800005DD0929CCBF602368231370EDE7002C06
:103A9000CCBF6C2364231370E7E700BF387F00209E
:103AA00030B585B0054601A840F082FA044618B941
:103AB0002870204605B030BD044A0123B2F9002029
:103AC00001A9284640F0EEFAF3E700BF7054002049
:103AD0004068E5E773B50D4D009104461646002396
:103AE00002460221286837F08BFD094B00932246DD
:103AF00028680023142137F083FD286800960023EE
:103B00002246162137F07CFD02B070BD64450020CE
:103B10005DBB06082DE9F04704468AB0E8B1A94B21
:103B20001868037A9C422246A8BF1A469C42B8BF36
:103B30000132A3EB020303EBD373B4BF01210021D5
:103B4000C3F3470449B1A04B00932246002302214E
:103B5000651C37F055FDEDB22C46DFF8B8829B4F5F
:103B6000DFF8B4920026454617F8013BD8F8BC139D
:103B700001229A400A4230D0172B2ED8DFE813F0EA
:103B8000180034004D0077009000B300C700DB0040
:103B9000EF00FE0010015B004E0184019701B401AB
:103BA000C901D401A000E401090214022702FD01A9
:103BB0000DF1080A5046FFF773FF18B984495046C3
:103BC00043F0E0FB7F48CDF800A0006800232246C8
:103BD000022137F015FD0134E4B20136182EC3D1AD
:103BE00020460AB0BDE8F087B5F8AE23002312F0F6
:103BF0000F02194618BF012202A8FEF7B7FFB5F859
:103C0000AE3303F00F02734B03EB82032046D3F86D
:103C1000FC1002AAFFF75EFFDDE7B5F8B023012331
:103C200012F00F0218BF1A46002102A8FEF79EFFED
:103C3000B5F8B033E5E7D5F8BC05FDF741FD95F8DB
:103C4000AD1300290CBF0F210C210A23009190FB1A
:103C5000F3F0614990FBF3F203FB120302A843F077
:103C600091FB5E4902AA2046FFF734FFB3E75C4BA5
:103C70001B681B06B1D5B5F9B005FDF70BFD95F82E
:103C8000AD335849002B02460CBF9D239E2302A84A
:103C900043F078FB544902AA2046FFF71BFF9AE73E
:103CA0004F4B1B68180698D5B5F9C01502A800221D
:103CB000FEF70EF94D4902AA2046FFF70BFF8AE7EF
:103CC000474B1B68190688D5D5F86414642302A8ED
:103CD000B1FBF3F10022FEF7FBF8454902AA2046AA
:103CE000FFF7F8FE77E7B5F9B215642391FBF3F21D
:103CF00003FB1213062100911BB23E4902A843F0B8
:103D000041FB3D4902AA2046FFF7E4FE63E7B5F810
:103D1000B4156423B1FBF3F203FB121306210091E7
:103D20009BB2344902A843F02DFB344902AA204635
:103D3000FFF7D0FE4FE7B5F83C146423B1FBF3F274
:103D400003FB1213062100919BB22A4902A843F0FB
:103D500019FB2B4902AA2046FFF7BCFE3BE702A94C
:103D600095F8B805F8F796FE264902A84BF00FFE25
:103D7000254902AA2046FFF7ADFE2CE795F8D6327A
:103D8000002B3FF42AAFB5F9B62516499A2302A8AD
:103D900043F0F8FA1D4902AA2046FFF79BFE1AE7F6
:103DA00095F8D632002B3FF418AFD5F834240D49DE
:103DB000072302A843F0E6FA154902AA2046FFF7B6
:103DC00089FE08E764450020A67806080604060870
:103DD000B6780608240306086C770608BD7806083E
:103DE000E45100206F770608CA780608D4780608E0
:103DF000E178060834B60608F1780608FD7806086A
:103E0000017906082A790608097906081279060850
:103E10001E790608387F0020C1790608DFF8FCA16A
:103E20009AF80230002B3FF4D8AE032B3FF4D5AE06
:103E300010F032FD9AF80230022B1DD1F8B1FBF7D9
:103E4000E3FF724B02684FF4FA61B2FBF1F11A68BA
:103E50004FF47A23B2FBF3F28B1A64225A4302A87E
:103E6000B2FBF1F26A4992B243F08CFA694902AAB4
:103E70002046FFF72FFEAEE6002840F0C6806649D8
:103E800002A843F07FFAF1E7644B9B78022B7FF4A2
:103E9000A4AED5F80C060028FFF69FAE02A9F8F7ED
:103EA000F9FD5F4902AA2046FFF714FE93E6D5F814
:103EB00000319A077FF591AE5A4B93ED060AF2EE68
:103EC000047A20EE270A49F0F5F90A23564990FBB7
:103ED000F3F203FB120302A843F054FA534902AA77
:103EE0002046FFF7F7FD76E6B5F9C805FEF7CEFDEB
:103EF00095F8AD334E49002B02460CBF0D230E231F
:103F000002A843F03FFA4B4902AA2046FFF7E2FD20
:103F100061E602A9D5F8CC05F8F7BCFD464902AA2E
:103F20002046FFF7D7FD56E6B5F8D025434902A84D
:103F300043F028FA424902A84BF029FD414902AA60
:103F40002046FFF7C7FD46E63F4B1B689B007FF509
:103F500044AE3E4BB3F898204AB13D4902A843F025
:103F600011FA3C4902AA2046FFF7B4FD33E63A4A6B
:103F700038492046FFF7AEFD2DE6B5F9D225374981
:103F800002A843F0FFF9364902AA2046FFF7A2FD36
:103F900021E602A9D5F82006F8F77CFD314902AAEE
:103FA0002046FFF797FD16E63C21D5F82436B3FBF3
:103FB000F1F302A8B3FBF1F201FB12332A4943F0FB
:103FC000E1F92A4902AA2046FFF784FD03E695F8A5
:103FD000AD33D5F8282673B940F249617E23B2FB90
:103FE000F1F202A8124943F0CDF902AA494620464F
:103FF000FFF770FDEFE54FF47A717D23B2FBF1F22C
:1040000002A80B4943F0BEF9EFE7FFDE8C7E0020EB
:1040100027790608327906082C790608FC53002017
:104020003B790608E48400203678060846790608BD
:104030006F770608527906085F790608A9B706085F
:104040002A7906086B790608E4510020C40B001099
:10405000747906087979060882790608F5770608E2
:104060008B79060898790608A6790608AF790608BC
:10407000037870B4FBB10446C0F10106A31914F82B
:10408000015FDBB2002DF9D101335B00DCB2032507
:1040900013800C704D7004785CB1022300255A1C0B
:1040A000D2B2CC548D5410F8014F0233DBB2002C45
:1040B000F5D170BC704702242346E8E70B0617D4FD
:1040C00001EB810300EBC30310B400EB810001247A
:1040D000002283F8764383F8741383F87523426DC6
:1040E0005DF8044B136843F400130020136070471D
:1040F00001F07F0101EB810300EBC303012200EB20
:10410000810083F81C1183F81E2183F81D21826928
:104110001368002B01DA43F0804343F4001313606B
:1041200000207047F0B5012190F8D17590F8D36563
:1041300090F8CFC590F8CE5590F8D03590F8D225AC
:1041400080F8111190F8CC1585B005EB0C2503EB28
:10415000072302EB062201F01F06AFB292B290F8DD
:10416000CD558DF808109BB2012E0446ADF80A70AB
:10417000ADF80C30ADF80E20C0F840218DF8095094
:1041800017D0022E1FD036B101F08001FFF796FF45
:10419000002005B0F0BD092D0FD8DFE815F0BF00F5
:1041A000AC000E00D5000E00EA0085000E0077007E
:1041B000540090F81221032A2FD02046F9F750FC22
:1041C000002005B0F0BD01F060012029DAB234D042
:1041D000012D00F02081032D00F00681002DD7D1A4
:1041E00090F81211022900F0DF800329E5D11B06A7
:1041F00000F14B8102EB820200EBC20393F87633AD
:10420000002B00F04D81BF4B0122C3F84026BE4970
:1042100020460222FCF71CFBBAE7DAB2012ACCD80E
:10422000D0F8E43502A99B689847BDF80E30002B02
:10423000AED12046FCF7FCFAAAE7D0F8E43502A993
:104240009B689847A4E7F9B2AE4D012985F830166E
:10425000B3D890F81231022B00F02781032BACD198
:10426000002900F0868190F810110129E1D0D0F8E2
:10427000E4355B68984795F8301684F810112046AD
:10428000FCF706FD2046FCF7D3FA81E7012A94D11A
:1042900090F81231022B00F01781032B8DD100F51D
:1042A0008871FCF7D5FA73E73D0A022DADF80620B8
:1042B00000F05081032D00F00B81012D7FF47DAFC4
:1042C000D0F8EC3580781B680DF106019847BDF8F1
:1042D0000620002A3FF45CAFBDF80E30002B3FF4FF
:1042E00057AF9A4228BF1A4601462046ADF806202D
:1042F000FCF7AEFA4CE790F81231023B012B3FF687
:104300005CAF012F7FF444AFD0F8E43500229B6806
:10431000C0F8182102A9204698478AE790F8123180
:10432000023B012B3FF649AF764BD0F81821002114
:10433000C3F8381612B10222C3F838267349204652
:104340000222FCF785FA23E7012F00F09880022F64
:104350007FF41EAF13F0FF0F7FF41AAF02691B0A40
:10436000023B5268032B00F21D81DFE803F0393570
:1043700031241A437FF421AF90F81231032B3FF41C
:104380001CAF036907F07F0580F81451196867F3C3
:104390000A120A431A60FCF74BFA002D00F0E58080
:1043A000022384F81231F3E651063FF4F1AE1146D0
:1043B000FFF784FEECE6052363F30612514B01215F
:1043C00084F816112046C3F83C26FCF731FADFE6E4
:1043D000042363F30612F1E7032363F30612EDE708
:1043E000022363F30612E9E790F81231022BDBD0C7
:1043F000032B7FF4E2AE27B9550602D01146FFF732
:104400005DFED4F8E43502A99B6820469847204613
:10441000FCF70EFABCE690F812110229C4D0032969
:104420007FF4CBAE002F7FF4B3AE12F07F013FF4E8
:1044300000AF180600F1A78002EB820304EBC30370
:1044400004EB810083F8767383F8741383F8757333
:10445000282303FB0243416D03F55D73DA780B6893
:10446000023A6FF35553012AD4F8E42598BF43F07C
:1044700080530B602046936802A99847D9E6D0F88C
:10448000E435C0F818719B6844E702F07F0202EB44
:10449000820200EBC20393F81E31002B7FF4B3AE0F
:1044A000184B0022C3F84026B1E600293FF4C1AE04
:1044B0000121032380F8101180F81231FCF7E8FB8A
:1044C0002046FCF7B5F963E61149FCF7C1F95FE650
:1044D000FDB2052D3FF671AEDFE805F0342C241C4B
:1044E0000B03D0F8EC3580789B690DF106019847F5
:1044F000EDE6D0F8EC3580785B690DF10601984760
:10450000E5E600BF387F0020788500207085002018
:104510006C850020D0F8EC3580781B690DF1060120
:104520009847D4E6D0F8EC358078DB680DF10601C9
:104530009847CCE6D0F8EC3580789B680DF1060101
:104540009847C4E6D0F8EC3580785B680DF1060139
:104550009847BCE6D0F8E43580789B6A0DF10601F7
:1045600098474570C4F8F005B1E6012384F812318C
:104570000EE60222D0F8E43580F8101180F81221FE
:104580005B68984755E6282202FB014304EB810053
:1045900083F81E7183F81C1183F81D51816903F59E
:1045A0008E735BE7012363F3061207E770B501F032
:1045B0007F0505EB850400EBC404282101FB050100
:1045C0000126C4F830310023C4E94A2284F81C5182
:1045D00084F81D61C4F8343101F58E711DB9FCF702
:1045E00085FB002070BDFCF7F5FB002070BD00BF0F
:1045F00038B501EB810400EBC4040D46002184F8BA
:104600007453C4F88C1384F87513C4F88833C4F851
:104610008023C3782821012B01FB050108BFEDB2DF
:1046200001F55D7108BFC4F884231DB9FCF75EFB7A
:10463000002038BDFCF7CEFB002038BD10B5044685
:1046400029B990F81131032B0DD0002010BDD0F8FE
:10465000E4359B69002BF8D090F81221032AF4D19D
:104660009847002010BDD0F89013D0F87C339942C1
:1046700014D9C078D4F880230128A1EB030104BF2A
:10468000D218C4F880238B4228BF0B46C4F890137D
:104690009BB220460021FFF7ABFFD6E7D0F8E43508
:1046A0001B691BB190F81221032A03D02046FCF7A6
:1046B000BFF8CAE79847F9E70B0630B41CD401EB02
:1046C000810200EBC202002300EB810582F8741323
:1046D00082F8753301241A4604FA01F16D6D61F315
:1046E0001F4201696FF3CF332B60CB6923EA0203CA
:1046F000002030BCCB61704701F07F0101EB8104E9
:1047000000EBC404012200EB8105002384F81C1196
:1047100084F81D2102FA01F11A46AD6961F30F0216
:10472000DFE700BFF0B416460A063AD401EB810574
:1047300000EBC5052824002204FB0104022B85F8A8
:104740007413C5F87C6385F8773385F8752304F511
:104750005D7448D0154600EB8107012202FA01F191
:104760007F6D61F31F45D7F800C01CF4004F11D1D5
:10477000E488204946F0805242F4004242EA8342F3
:1047800004F00F041C4B42EA845211400CEA03036C
:10479000194339600269D3692B430020F0BCD3610F
:1047A000704701F07F0101EB810500EBC50528246E
:1047B000012204FB0104022B85F81C11C5F82461B9
:1047C00085F81F31A5F8221185F81D2104F58E7496
:1047D0000CD0002500EB8107012202FA01F1BF692C
:1047E00061F30F05BFE722711546B4E70025257177
:1047F000F0E700BFFF87CC13007833EC002310B53F
:10480000194604464022FFF78DFF802120460023F1
:104810004022FFF787FFD4F8E835A078012284F81A
:1048200012215B689847002010BD00BF82B00023B2
:10483000016801930B6901930E4B03E00A69019231
:10484000013B13D0019A002AF8DA019A094B42F091
:1048500001020192019A0A610A69019203E00A6960
:104860000192013B02D0019AD207F8D4002002B095
:10487000704700BF400D0300436D064A1A61C278BD
:10488000012A06D100F2CC5058614FF080221968FD
:104890001A6070471800086070B5044649B990F86E
:1048A0001131022B1BD094F81631012B0DD00020B2
:1048B00070BDD0F8E4355B69002BF8D090F8122178
:1048C000032AF4D19847002070BD2A4A2369D2F800
:1048D0003C265A60002384F81631002070BDD0F8C1
:1048E0003831D0F82451AB4217D9C278012AD0F818
:1048F0002821A3EB050308BF5219C0F8383108BFBF
:10490000C0F828219BB20021FFF750FE00231A4671
:1049100019462046FFF76CFEC5E7D0F83C31B3FBE3
:10492000F5F605FB163666B99D420AD8D0F8402147
:10493000934206D233463246FFF738FEC4F8406150
:10494000E4E7D4F8E435DB681BB194F81221032ABC
:104950000CD00023052284F8112119461A4620465E
:10496000FFF746FE2046FFF787FF9CE72046984763
:10497000EFE700BF387F002082B000230193019A47
:10498000094B42F010020192C168019A0A610A695A
:10499000019203E00A690192013B02D0019AD2061A
:1049A000F8D4002002B07047400D030082B000230D
:1049B0000193019A0B4B42F020020192019A61F39C
:1049C0008A120192C168019A0A610A69019203E0A0
:1049D0000A690192013B02D0019A9206F8D40020A4
:1049E00002B07047400D0300104B70B4DA68437892
:1049F000017886780E4CD243C2F30222C2F104053C
:104A0000E8B283400F2040FA02F23240DBB2134397
:104A100060181B0101F01F0501224909DBB2AA4001
:104A200080F8003344F8212070BC704700ED00E0AE
:104A300000E100E0C27802B1D6E7037805485A09E0
:104A4000203203F01F03012101FA03F340F8223062
:104A5000704700BF00E100E000B583B009238DF886
:104A60000730FCF76FFA8DF807009DF80730012B2F
:104A7000F7D09DF8070003B05DF804FB82B0064B49
:104A8000002201920193019B03EB80000190019BA6
:104A9000186802B0704700BF5028004082B0064B33
:104AA000002201920193019B03EB80000190019B86
:104AB000196002B0704700BF502800400023C0E9D1
:104AC0000033C0E90233C0E90433C0E90633C0E96A
:104AD0000833C0E90A33C0E90C338363704700BF71
:104AE0000B6870B4D1E90524CD682B431343D1E999
:104AF000072523431343D1E909422B43D1E90D652F
:104B00002343134304680B4A334322402B4313438C
:104B10000360D1E90B3442690D6922F00702234397
:104B20001343D1E9014243614560846070BCC260B7
:104B3000704700BF3F801CF002683649002310B464
:104B400022F00102212488420260036043608360F6
:104B5000C3600361446138D02F4B98422ED02F4B55
:104B600098423CD02E4B984240D02E4B984232D0A7
:104B70002D4B984241D02D4B984246D02C4B984219
:104B800017D02C4B98423CD02B4B984216D02B4B35
:104B9000984224D02A4B984228D02A4B98421AD0C7
:104BA000294B984229D0294B98422ED0284B984225
:104BB00008D14FF03D5243F8AC2C03E04FF474623F
:104BC00043F8202C5DF8044B7047224B5DF8044BF2
:104BD0003D229A607047204A43F8642CF2E74FF474
:104BE00074125DF8044B43F8382C70474FF0746230
:104BF0005DF8044B43F8502C7047184A43F87C2C5E
:104C0000E0E73D2243F8082CDCE7154A43F8942CF2
:104C1000D8E700BF106002402860024040600240B8
:104C2000586002407060024088600240A06002400C
:104C3000B8600240106402402864024040640240B0
:104C4000586402407064024088640240A0640240DC
:104C5000B8640240006002403D000020400F002088
:104C600000003D200B88F0B433BB028C4C880E89C9
:104C70008B88C98822F001021204120C0284058B71
:104C8000028CADB225F0F30592B22B4322F00A025A
:104C900043EA061322439BB242F0010203830284DB
:104CA000038B23F00C031B041B0C0383038B9BB2AD
:104CB0001943F0BC01837047042B048C2CD0082BC3
:104CC0004E888A880D89C98851D024F480542404E0
:104CD000240C0484838B078C2C0344EA022440F6C2
:104CE000FF421A4045F6FF733B4043EA0633224336
:104CF0009BB292B243F4805382830384828B22F46A
:104D000040621204120C8283838B9BB243EA01231C
:104D10009BB2F0BC8383704724F010042404240C5D
:104D20004D880F898A88C9880484068B038C1202F7
:104D30009BB242EA073423F0A00340F6FF42324020
:104D400043EA051322439BB292B243F0100302835D
:104D50000384028B22F440621204120C0283038B40
:104D60009BB243EA01239BB2F0BC0383704724F457
:104D700080742404240C0484848B038CA4B29BB21E
:104D800024F0F30423F42063224343EA062342EA97
:104D900005129BB243F4807392B282830384838BA7
:104DA00023F00C031B041B0C8383838B9BB21943DE
:104DB000F0BC8183704700BF214A038890429BB2B8
:104DC00012D002F5806290420ED0B0F1804F0BD02D
:104DD000A2F58032904207D002F58062904203D063
:104DE00002F58062904203D14A8823F07003134396
:104DF000144A904218D002F58062904214D030B428
:104E000023F440730C894D6802F56C429BB2234336
:104E100090420C880380C56204850DD18B7A03868D
:104E2000012330BC8382704703800B884A68C262CA
:104E30000385012383827047034B9842EED0EFE74E
:104E4000000001400010004000040140024A536A83
:104E500023EA00005062704700380240024A136A99
:104E600023EA00001062704700380240484B984225
:104E70002ED0B0F1804F32D0464B984236D0464BC0
:104E800098421ED0454B984237D0454B98423BD074
:104E9000444B98423FD0444B98424BD0434B9842AE
:104EA00040D0434B98424CD0424B984251D0424B59
:104EB000984256D0414B98425AD0414B98425ED0CE
:104EC0007047404A136A43F0040313620420C5E7A5
:104ED0003C4A536A43F0010353620120B6E7394A62
:104EE000136A43F0010313620120B7E7354A136ADE
:104EF00043F0020313620220B0E7324A136A43F020
:104F0000080313620820A9E72E4A136A43F010032E
:104F100013621020A2E72B4A136A43F020031362A6
:104F200020209BE7274A536A43F4803353624FF4AF
:104F300080308BE7234A536A43F002035362022016
:104F400084E7204A536A43F4003353624FF400303D
:104F50007CE71C4A536A43F4802353624FF4802059
:104F600074E7184A136A43F040031362402075E760
:104F7000144A136A43F08003136280206EE7114ADB
:104F8000136A43F4807313624FF4807066E700BFC6
:104F9000000001400004004000080040000C0040F8
:104FA0000010004000140040000401400040014097
:104FB000004401400048014000180040001C00402F
:104FC0000020004000380240224A936803F00C039E
:104FD000042B10B421D0082B22D01F4B03601D4C92
:104FE0001E4AA168C1F30311114491F82C10CB4063
:104FF0004360A168C1F38221114491F82C1023FA77
:1050000001F18160A1685DF8044BC1F342310A44AB
:1050100092F82C20D340C3607047114B0360DEE749
:105020005468516852686302C2F388124CBF0C4B3B
:10503000094B01F03F01B3FBF1F303FB02F3054A17
:105040005268C2F3014201325200B3FBF2F3036033
:10505000C5E700BF003802400024F4001806002015
:1050600000127A002DE9F04700230F6801264FF067
:10507000030C02E00133102B41D006FA03F232EAAE
:105080000704F7D1D0F800E05C000CFA04F52EEA32
:10509000050EC0F800E091F80490D0F800A009FADD
:1050A00004FE09F1FF394EEA0A0EB9F1010FA846D4
:1050B000C0F800E06FEA050515D8D0F808E005EA69
:1050C0000E0585604D79D0F808E0A54045EA0E054B
:1050D0008560456825EA020242608A7945689A40FF
:1050E00092B22A434260C26822EA0802C260CA79C8
:1050F000C568A24001332A43102BC260BDD1BDE870
:10510000F0870D4B93F84C24D20703D5012283F886
:105110004426704793F8442662B9D3F8B0244AB1C4
:1051200093F86824104493F8692483F868041144C0
:1051300083F86914704700BF387F0020044B93F94F
:105140000000012806BF02221A700020704700BF2D
:10515000387F0020114AD2F84806A0B1D2F84C3668
:105160008BB188420DD88B4234BF002301239BB101
:105170005368C2F8501699421CBF142382F8543663
:10518000DCE70023F3E7A1F59C53083BB3F57A7FF6
:105190002CBF00230123EAE7704700BF387F0020BF
:1051A00007B500230DF10602ADF8063009F090FEB8
:1051B00060B1084BBDF806201989A3F85626914224
:1051C0001CBF142283F85826FFF7B8FF03B05DF820
:1051D00004FB00BF387F002013B504462620019150
:1051E0001CF012FE019948B9054BD3F820342BB1BD
:1051F000204602B0BDE81040FCF7D6BA02B010BDA0
:10520000387F0020B1FA81F149094920E4E72DE90E
:10521000F341BE4C94F9003001330D4600F0668135
:10522000D4F82034002B00F0B380022700264FF082
:105230000108D4F8200431F0BFFC002800F0A88059
:10524000D4F8200431F0B0FCD4F828345A1C23449C
:10525000C4F8282483F8590694F82434012B09D083
:10526000022B15D063B90F280CBF84F82484C4F82E
:105270002834DEE7A0F17203012B06D9762804D08A
:1052800084F82464C4F82864D3E784F82474D0E74D
:10529000102ACED19E490023012211F8010F0132BC
:1052A00003440E2ADBB2F8D194F8672684F824640C
:1052B0009A42C4F82864BCD194F86836002BB8D15F
:1052C00094F85A36732B59D0762B1BD0722B5FD1A2
:1052D00094F85C2694F85B3694F9001053EA0223A4
:1052E00056D0C4F848360029B4F85D36C4F84C36B8
:1052F0004EDC94F8762601232370002A48D184F8E6
:10530000763645E094F85C2694F85B3653EA02233F
:105310003ED0D4F86C2694F85E1694F8620663606A
:1053200093421CBF142284F8542694F85D26C4F8D6
:105330006C3642EA0122B4F87016228191421CBFF9
:10534000142184F8581694F85F16617094F860166A
:10535000A17094F86116A4F8702641EA0021A4F81F
:105360007216D4F8501609B9C4F85036B4F8563647
:105370000BB9A4F856260223237009E094F860269E
:1053800094F85F3643EA02231AB20BB1A4F87426EC
:1053900094F90030022B35D00FDCDAB2012A15D98E
:1053A000A36D13B1E368002B6CD15A495A481F22F0
:1053B00002B0BDE8F0414AF020BB032BF0D1D4F895
:1053C0007836564AEB1A9342EADD13E0D4F8782691
:1053D0005349AA1A8A42E3DD2BB97220FCF710FA6E
:1053E000C4F87856DCE7D4F87C365A1CD907C4F8E0
:1053F0007C2603D47620FCF703FAF1E77320FCF750
:10540000FFF9EDE7D4F85016D1B194F85436BBB19A
:105410006368994214D06378DA0703D489B24620CE
:10542000FFF7DAFE94F85436013B84F8543605F55C
:105430009225032305F578752370C4F87856AFE7F5
:10544000B4F85616238981B194F858266AB18B4274
:105450000BD06378DB0702D45020FFF7BDFE94F831
:105460005836013B84F85836E1E701222270A4F84F
:1054700056366268C4F85026002384F8583684F8FB
:1054800054368DE7274DD4F8B0742A2385F83C3084
:105490000DF1070220230DF10601384685F83D3055
:1054A00009F0ADFD30B19DF806109DF8076051EA96
:1054B00006031ED1552385F83E30462385F83F303C
:1054C00062681948202385F84030002A34D01749F3
:1054D00041F058FFB4F8723615488BB3228915494C
:1054E0009A420CBF20222A2241F04CFF02B0BDE8B4
:1054F000F081384609F068FD314685F83E003846AF
:1055000009F04EFD037885F83F30D9E7387F002059
:1055100091850020D079060854060020400D030034
:1055200040420F001806002059060020CFAF0608A1
:105530005D060020EA790608034941F023FFC9E728
:10554000024941F01FFFD1E7F2790608F179060818
:1055500010B50D4C40F0080284F85F2094F900204B
:10556000022A05DD420703D583071CBF01232372EE
:1055700005210648FBF7B6FD062184F86000BDE86A
:1055800010400248FBF796BD180600207306002065
:1055900010B5FBF743FD98B31A4C94F90030012B7A
:1055A0002EDD49B3022B2BD0237A9BB971B1802316
:1055B0000521154884F86530FBF794FD062184F831
:1055C0006600BDE810401048FBF774BDBDE8104010
:1055D0000420BDE7002914BF00200420E3781A0747
:1055E00048BF40F002005B0701D411B108B940F098
:1055F0000100BDE81040ABE7022BD5D10420EDE758
:1056000010BD00BF1806002079060020F8B5214C17
:1056100004F16707030A84F86C0005460621384642
:1056200084F86B30FBF75EFDE37884F86D00DB07F0
:1056300029D4A288AA4226D1174DD4F86730C5F8DC
:105640008036C3B285F8863641F26F714FF6FF732C
:105650008A4218BF0123134405F5D066C3F307221D
:105660000621304685F8842685F88536FBF73AFD15
:10567000072185F886063046FBF71CFD052104F15D
:105680006E00FBF717FDBDE8F84004480721FBF763
:1056900011BD00BF18060020387F00207F060020C3
:1056A00008B5FBF7BBFC48B1A1F59C53083BB3F52B
:1056B0007A7F03D2BDE808400846A7E708BD2DE978
:1056C000F8436A4E3368002B38D0694C694D306816
:1056D00031F072FA002833D1674B198809291D4629
:1056E00009D95F8864227A43B2FBF1F2452A40F37C
:1056F0009C811880588094F8C136012B00F0BC8141
:10570000022B00F0D58133B95C480521FBF7D2FCB0
:10571000012384F8C1365A4B1D685A4B1B78002B65
:1057200000F0CF81584B1B68EB1A782B40F2C981EF
:10573000D4F8AC04F8F762F9C4F8C456BDE8F883AD
:10574000306831F031FA94F887360746052BBED819
:10575000DFE803F00309171D3745AA28B7D1012355
:1057600084F88736B3E7552803D1022384F88736B7
:10577000ADE7414A938801339380002384F887364C
:10578000A5E7032384F8880684F887369FE7132863
:1057900084F88906C4F8A40607DD374AD3880133A4
:1057A000D380002384F8873691E718B9052384F85D
:1057B00087368CE70023C4F8A836042384F887369C
:1057C00085E7D4F8A836E218013382F88A06D4F8BF
:1057D000A426C4F8A83693427FF479AFE6E7D4F85C
:1057E000A4362A4803F102094FFA89F1FBF77AFC43
:1057F000874294F8888640F00F8126201CF004FB35
:10580000204B48B100221A701B4A53880133538041
:10581000002384F887365AE71A78424519D10022C6
:105820001A7008F1FF33102B00F2F180DFE813F05B
:1058300030008A008A00DB008A00EF00EF00EF00F2
:105840003000EF00EF00EF00EF00EF00EF00EF009F
:105850003000B8F1090F02D0B8F1110F01D1012ABF
:10586000DDD0054A538901335381DAE7C053002064
:10587000387F002018060020E45300208606002010
:10588000C8220020F2530020F4530020C0850020DD
:10589000B9F1060F56DDB8F1010F06D0B8F1090FC6
:1058A0000CBF4FF002084FF0030894F88D0694F8EF
:1058B0008E1694F88C2694F98AC694F98C7694F80E
:1058C0008B3685F8008041EA002109B2900785F8FF
:1058D00001C0EF70A98005D512F00C0F14BF012292
:1058E00000222A72B8F1030F13D1B9F1090F29DD93
:1058F00094F99026082AA8BF082222EAE27285F8C5
:105900002020002358B2824203F1010359DC94F8AD
:105910008F36D4F80C90002002469BB24A4596463A
:1059200057DB784BA8701B78232B0BD108EB88032F
:10593000754A03EB830307EB83031380A2F802C0CD
:105940009180D08071490A22284649F0F0FF10B1B9
:10595000002384F8B6366D4B2A681A606A685A606C
:105960002A891A8194F8B63633BB2B7A94F86824C6
:1059700084F8B826002B14BF0223012384F8B6361E
:10598000EB7894F86A0484F8BC0613F001031CBF9A
:10599000B2FA82F35B0994F8692484F8B926D9B283
:1059A000B4F86C2484F8B716A4F8BA2613B10AB177
:1059B000A4F8BE2684F8C0160AF04AFD0AF048FD95
:1059C00022E704EB400E204490F89206AEF89C04C7
:1059D00098E704EB4E0E0132BEF810E052B29E453D
:1059E00008BF10469AE7B9F1040FABDD94F88A2698
:1059F00094F88B3643EA022359041AB203D5C3F351
:105A00000D03EB809EE7002AF9DBAB809AE7404A62
:105A1000938901339381F7E618F0010F7FF4F8AE14
:105A20003B4A138901331381F2E63A4B5A6FB3F8BC
:105A30007810012A18D141F25632914202D14FF02A
:105A4000FF325A675A6F306802EB820202EB820221
:105A500001EB420189B2A3F8781003681B699847EB
:105A600000232B806B8046E60132EBD1B1F5965FC7
:105A700004BF01225A67E5E7264D95F90060002E24
:105A80003FF449AE022E0FD14FF48040FFF7BEFD28
:105A900084F8C16695F90030012B7FF73CAEEB78B6
:105AA000C3F340032B7236E6032384F8C136F1E7D3
:105AB000184BDB88002B3FF42EAE032384F8C1364D
:105AC00029E694F8242094F825309A4204D0FCF773
:105AD00037FBC4F8C45631E6D4F8C436EB1AB3F534
:105AE0007A7FBFF42BAE0C4B1B68ED1A952D7FF619
:105AF00025AE0A480521FBF7DDFABDE8F843FCF7BF
:105B00001FBB00BFA1260020A4260020E4850020A2
:105B1000E453002018060020F453002086060020DD
:105B200010B5134CD4F8B00400B394F8681459B10C
:105B300094F8692409F0E0F9B4F86C3483421ABF90
:105B4000A4F86C0401210021B4F86E2462B141F282
:105B500088339342B8BF13469A4205D0A4F86E34F6
:105B6000BDE810403AF058B80029F9D110BD00BF87
:105B7000387F002010B401440446002014F8013B93
:105B800008225840430010F0800F08BF400083F007
:105B9000070314BFD8B2C0B2013AF3D18C42EDD1A1
:105BA0005DF8044B704700BF30B54FF4806085B09E
:105BB00029F0D4FF40B3154C90F9040094F8C8368E
:105BC000134A002B18BF08234FF4E1310125CDE91A
:105BD0000153009100234FF480612AF020F8FF2345
:105BE0002066003818BF012084F87C3084F88C309F
:105BF00084F89C3084F8AC3084F8BC3084F8CC3025
:105C000084F8DC3084F8EC3005B030BD387F0020FB
:105C10008D130108364B1B6813F000635AD02DE931
:105C2000F04F344B1F78B8424FD3FF2854D1324B3A
:105C30001B7C002B46D0DFF8D4A00022CAF8CC266B
:105C4000CAF8D026CAF8D426AAF8D826002F4BD0F6
:105C50000AF17C031046144611461546164603EB1E
:105C6000071BB946B3F802C09F8993F8008093F9E7
:105C700001E061443A444645D3E901C738BF46468E
:105C800010337545B8BF75469B4509B212B26444DE
:105C90003844E7D191FBF9F192FBF9F28AF8CC662E
:105CA0008AF8CD56CAF8D046CAF8D406134BAAF8DB
:105CB000CE161B781049AAF8D826092B4FF00002FF
:105CC0000A740CD00E48BDE8F08F0E4A02EB0010AB
:105CD000BDE8F08F184670470020BDE8F08F0A4BF2
:105CE0009AF8CC26DA80EDE73A463946DEE700BF7F
:105CF000E4510020C40B001018060020A12600204B
:105D000004860020B47F0020A4260020387F0020D5
:105D10000268F8B53A4E3B4CB6F9A835511C016003
:105D20007E2111700168054603EBC30384FB030267
:105D3000481CDC17002328600B70FF20C4EB6204B2
:105D4000FFF768FF2034304BA4B200284DD01B78F9
:105D5000B0F90C102BBB2D4BA1F57A729A4246D8A4
:105D60002B48B0FBF1F189B2284639F0B1F996F829
:105D7000EF34B6F83C1483B196F84734B1FBF3F135
:105D8000284639F0A5F92146284639F0A1F92846D8
:105D90000821F7F709F80120F8BD284639F098F9ED
:105DA000F1E71C4B1F78002FD5D01B48002300EBD8
:105DB000830201339289BB421144F8DB174B9FEDFC
:105DC000186A9B7E07EE103A07EE901AB8EEC77A73
:105DD000F8EE676AC6EE077A67EEA67AFCEEE77A17
:105DE00017EE901AB1FBF7F1B5E71B7813B94EF631
:105DF0009C21B9E7074B1F78002FF8D00146D4E764
:105E0000387F002067666666600900101783930379
:105E100000879303C40B0010600C0010B82600200C
:105E2000000048432DE9F04FAF4C89B094F8468408
:105E3000054630F04BF9D4F8DC36D4F8B46323F4DB
:105E40000013C4F8DC36F307074649D500201BF0E1
:105E5000DBFF002841D0D4F8E426002A3DD0900191
:105E600004D5B2F1007F18BF02F17E42D4F8E816E3
:105E70009FED9E7A7B1A07EE903AF8EE677AF4EE81
:105E8000C77AF1EE10FA05DCD4F8EC060123834062
:105E9000134212D111B91923C4F8EC36D4F8EC36F8
:105EA000C4F8E876012001331A2B28BF002300FA3A
:105EB00003F11142F7D0C4F8EC36D4F8EC268C4B41
:105EC0008C49686803EB8203D3F80C2141F05AFA3D
:105ED00002236B7309B0BDE8F08F0023C4F8E836E5
:105EE000D4F8F0367BB394F84C34D9072BD4D4F8DB
:105EF000F4369FED817A686803F5921303F57863B1
:105F0000DB1B07EE903AF8EE677A67EE877AFDEED4
:105F1000E77AB8EEE77A17EE903AF1EE0C7AB4EE43
:105F2000E77AF1EE10FA05DB744941F02BFA012310
:105F30006B73CFE70A21B3FBF1F201FB1233704917
:105F400041F020FAF3E7B2050FD594F8773463B146
:105F50006C49686841F016FA03236B73D4F8DC3699
:105F600043F40013C4F8DC36B4E7B30609D594F85B
:105F7000143633B16449686841F004FA01236B7345
:105F8000A8E7770536D594F8F836012B32D1D4F846
:105F9000003168689E0729D5B4F90A37B4F9A223FD
:105FA000D21A6FF463739A421BDB40F28D339A422C
:105FB0001ADC0A2392FBF3F2544941F0E3F91EF094
:105FC000B3FE534B1B6893F865300A3B23EAE37337
:105FD0009842ACDBD4F8DC3643F40013C4F8DC366A
:105FE000A5E76FF05902E7E75A22E5E7494941F092
:105FF000C9F9E4E7B00412D511F058F894F8AC33BD
:1060000083420CD94449686841F0BCF902236B73A0
:10601000D4F8DC3643F40013C4F8DC365AE7310414
:1060200008D53E4BB4F90024B3F918309A4201DD8B
:106030003B49E8E7720407D511F020F8B4F8FE33C5
:10604000834201D93749DEE7330704D5B8F1020F9F
:1060500001D135497DE737050FD594F84C34D80781
:106060000BD51BF06FFE40B194F89B33D90704D5D4
:1060700094F845370BB92D49C5E7F20414D594F8C7
:106080004C34DB0710D51BF05DFE68B194F89B33F0
:10609000DF0709D4D4F8AC35A3F53713A3F5D863DB
:1060A000002B01DA2249AEE7B4F81835580601D5BD
:1060B0002049A8E7310641D5B4F9A80594F8C633BC
:1060C00098423BDBFCF7E2FC94F8AD236E681A497A
:1060D000002A0CBF0D220E220346009230467A227F
:1060E00041F050F992E700BF387F00200024F448C7
:1060F0002403060809B90608ACC52737F77906084E
:10610000027A06080F7A0608197A0608247A060821
:10611000845300202E7A0608357A060818060020D7
:106120008F7906083E7A06084B7A0608557A0608E3
:10613000607A06086B7A0608747A0608604B1B685A
:106140001A016CD573066AD55E4B93F8009004AAC9
:10615000C9F1090676080023934620219E421AD1F0
:106160000BEB060058494FF0000A49F02CFC0336AF
:106170005246914501D90B2E11D908AB1E4400237C
:1061800006F8103CBAF1000F49D0504968685A46E9
:1061900041F0F8F83AE702F8011B0133DEE7D7B225
:1061A00038460392FFF736FD94F84CC4039A313712
:1061B0001CF0010CFFB230D0B4F9C2E3BEF1FF3FD6
:1061C0002BD08189642311FB03F1414B9B7E5B083B
:1061D00091FBF3F39E45B4BF3B46522394F9C013A1
:1061E00011F1800F04D090F901E08E45A8BF54232F
:1061F000BCF1000F08D0B4F9C413B1F1FF3F03D0D4
:1062000040688842A8BF43239F420BF8063018BF5E
:106210000AF1010A01320136ABE73B46DEE7D4F86A
:10622000B4335A0704D5B8F1010F01D12949EAE680
:10623000DF050DD594F84C24D60709D5264A92F8E7
:106240002520012A04D1254A12780AB92449DAE620
:10625000D8030CD594F84C24D10708D5B4F8A8235A
:106260002AB1D4F834148A4201DC1E49CBE69A07DD
:1062700018D594F84C2494F8461402F003020A430B
:1062800010D1B4F8DE12B4F83C2494F84704B2FB01
:10629000F0F2914206D91449686841F073F801237D
:1062A0006B7317E6DB067FF515AE94F84837002BC5
:1062B0003FF410AE0D49686841F064F837E600BF5E
:1062C000E4510020C40B00107778060809B90608CD
:1062D000B8260020837A0608FC4E0020740A0010BD
:1062E0008F7A06089B7A0608A47A0608B07A060810
:1062F00010B5184CA379CBB1A37EDFED176A07EE7A
:10630000903AF8EEE77A154B86EEA77AC0B203EB27
:106310008000B0F8A83007EE903AF8EEE77A67EE22
:10632000277AFDEEE77A17EE900A10BD0C4B1B683A
:1063300013F000630BD0C0B2FFF76CFC80896423BC
:1063400010FB03F0A37E5B0890FBF3F0EDE718462B
:10635000EBE700BFB826002000004843C40B001044
:10636000E451002008B5FFF7C3FF3C2390FBF3F096
:1063700008BD00BF2DE9F8434A4C427894F84937EC
:1063800002F00F05C3B9EDB92B46002184F84C1774
:10639000EB1AD9B20E290BD8234493F8F01439B173
:1063A00002F0F002802A4AD0902A5FD0A02A0DD0B5
:1063B00000273846BDE8F8830021AB4284F84C172B
:1063C000F6D8E5E784F849572B46DEE7412966D041
:1063D00081F08003042B62D90846FAF7EFFF031D12
:1063E0000246DBB2304884F84C3765F05F0584F82C
:1063F0004D57FCF79BF894F84C77002FD8D0BE1E71
:1064000016F0FF0024D1FF25A946022756B1DFF878
:106410009C80464418F8011BD4F8700730F0D0FB7C
:106420004645F7D1D4F87007494630F0C9FBD4F897
:106430007007294630F0C4FB3846BDE8F88365F0A4
:106440007F050427022684F84D5784F84C773046A0
:10645000164A4FF6FF71104412F8015B491B904237
:1064600089B2F9D15FFA81F90D0ACFE7412914D039
:1064700081F08003042B10D90846FAF79FFF65F0DE
:106480006F050627042684F84F0784F84D5784F8D3
:106490004E1784F84C773046DAE70420EFE70823FC
:1064A00004229FE7387F0020868600208486002013
:1064B0002DE9F047C31DDFF8348182B003F4FC738B
:1064C00000AFD8F81861ADEB030DC7F800D0326803
:1064D000D8F8103168449A420C4698F874377860BE
:1064E0006D4658D0591C0DF1010203F00F0388F8D6
:1064F00074178DF800303A60A0EB0209D6E900125B
:106500005FFA89F9521A09F107035FFA82FA03F474
:10651000FC73CA45ADEB030D55D25246684649F0AF
:10652000CDF933685344336052466946384638F0F3
:10653000ADFDD8F81821D8F810313068117A7060A4
:10654000C21A4A40D2B28342336088F8752709D014
:106550000133336013F8011C984282EA0102F7D13B
:1065600088F875273B68591C39601A70D7E90032E2
:10657000D21A012A08DD00215A1C3A601970D7E9A5
:106580000032D21A012AF7DC2846A047002008373B
:10659000BD46BDE8F087B6F90C20591C03F00F0387
:1065A00043F01003002A2A46B8BF43F0200302F844
:1065B000023B88F87417691C3960D6E900135B1A2E
:1065C0003A606B7098E74A46684649F077F9336855
:1065D0004B4433604A466946384638F057FD2846F2
:1065E000A04701200837BD46BDE8F087387F00206E
:1065F0002DE9F04F7A4C83B0D4F81851D5E9005307
:106600005B1B002B00AF83460D46164628DD00239A
:1066100084F87637FAF748FF00200BEB05030BF1FF
:10662000010AC4E941A39BF80050D4F81481690918
:10663000012940F09D8005F00F0915F0100514D1D7
:1066400050B194F87827013202F00F024A4500F069
:10665000988084F8765728460C37BD46BDE8F08F01
:1066600094F876070028D8D1D4E70BF10203C4F8D8
:1066700004310BF103029BF80130D4F80C01C4F88B
:1066800004219BF80250C8F80000C218C8F8042082
:106690006B4084F87737D4E941A34FF0000C84F8BD
:1066A0007617A8F80850A8F80CC0A3EB0A03DDB2CF
:1066B000121AEB1D5FFA82FB03F4FC73AB45ADEBE2
:1066C000030D6BD25A465146684649F0F7F80AEB7B
:1066D0000B035A4640466946C4F8043138F0D6FCEC
:1066E000D4F80C31D8F8000094F877278342C8E931
:1066F00000300AD00133C8F8003013F8011C98426A
:1067000082EA0102F6D184F87727D4F804311B78A5
:10671000934239D1B8F90830FA2B54D0D8F8002078
:10672000D4F80C31D4F81411D4F8C002C8E90032FE
:10673000D4F81821D4F810315360002515819581C3
:106740003B1D84F876577D6029F090FE01303FD0E4
:106750007B680BB100209847D4F81831D4F8102189
:10676000196801200C37C3E90021BD46BDE8F08F50
:1067700000210846FAF77CFE01200C37BD46BDE833
:10678000F08FD8E9000290E700230120B8F9081043
:1067900084F87637FAF76CFE01205DE72A46514609
:1067A000684649F08BF80AEB050340462A466946DD
:1067B000C4F8043138F06AFC00200C3784F878976C
:1067C000BD46BDE8F08F002EA8D005233370A5E7A5
:1067D000D4F8182113680221581C10601970B7E70B
:1067E000387F00200B4B93F8D62212B1B3F8002566
:1067F0004AB9B3F9A433084AD81782FB0323C0EB84
:10680000A30000B27047D3F8340490FBF2F000B25A
:10681000704700BF387F002067666666F8B5184C81
:10682000C6B205463146D4F87C0730F0C9F994F871
:106830008017D4F87C07C5F307274E40394684F803
:10684000806730F0BDF994F88017D4F87C07C5F361
:1068500007464F40314684F8807730F0B1F994F81C
:106860008017D4F87C072D0E4E40294684F88067A7
:1068700030F0A6F994F880174D4084F88057F8BDA1
:10688000387F002070B50C4DC6B231460446D5F8AD
:106890007C0730F095F995F88017D5F87C07240A25
:1068A0004E40214685F8806730F08AF995F88017C8
:1068B0004C4085F8804770BD387F002038B50B4CC0
:1068C000002305462421D4F87C0784F8803730F073
:1068D00077F9D4F87C07542130F072F9D4F87C07AA
:1068E0002946BDE8384030F06BB900BF387F002042
:1068F0002DE9F043DFF854932DED028B99F8814791
:1069000083B00E461546002C00F0E381013C89F867
:106910008147C74F9FEDC78ADFF834833378002B58
:1069200000F08E8099F88147002C40F0898035B1C5
:106930002FF0CCFB2B68C01A002880F2D98399F87D
:106940008247002C40F0788399F88307062840F2AC
:106950008181B94991F8813091F880209A4200F004
:10696000A88151F87C4F99F8842734F813401444D7
:1069700001300133A4B2C0B2DBB2B4F5C06F89F804
:1069800083074B7100F07D817CD8B4F5806F00F0F7
:10699000288224D8B4F5067F4FD8B4F5007F54D3AD
:1069A000A4F50073182B48D8DFE813F0E601DD01E9
:1069B000DD01DD01DD01DD01DD01DD01DD0147007E
:1069C000470047004700470047004700C501AA01AC
:1069D000AA01AA01AA01AA01AA01AA01AA01B4F561
:1069E000846F00F0E58140F2E280B4F5A06F00F022
:1069F00063826FF4A06C04EB0C03072B1DD8601EA0
:106A0000C0B2FFF707F9C0B1B0F90C308B4AADF84E
:106A10000140917ED9F8C42203EB830303EB830387
:106A200049089B0093FBF1F31021CDF803308DF85A
:106A300000106846904700233370002D7FF46EAF3E
:106A400003B0BDEC028BBDE8F083B4F5807F00F0AD
:106A5000FC81B4F5887FF0D1B9F94434CDF8033026
:106A6000012210238DF800308DF801308DF80220BE
:106A7000D9F8C4326846002498473470002D7FF45A
:106A80004DAFDDE7B4F5046F00F0A48265D8B4F52E
:106A9000006F00F081821AD9B4F5026F00F0F08126
:106AA000B4F5036FC9D199F89B339807C5D5644BEA
:106AB000D9F8C422D9894FF4F36303FB01F3A7FB90
:106AC00003135B091020CDF8033030218DE2B4F5BB
:106AD000E26F00F03682B4F5E46F1FD1594B93EDAD
:106AE000180AD3ED027A20EE270A002420EE080AC5
:106AF00046F0E0FB102320228DF800300723CDF86C
:106B000003008DF802308DF80120D9F8C4326846B0
:106B100098473470002D7FF401AF91E7B4F5E06F32
:106B20008BD1484B93ED160AD3ED027A20EE270A5B
:106B3000002420EE080A46F0BDFB10220723CDF802
:106B400003008DF802308DF80020D9F8C4328DF89A
:106B50000140684698473470DCE740F678339C4241
:106B600048D8B4F5376F00F2E181B4F5116F00F049
:106B70007F81B4F5376F7FF460AFFF20FFF74AF8ED
:106B800000283FF45AAF90F90130CDF803301021BE
:106B900070220B238DF802308DF80010D9F8C43222
:106BA0008DF80120684600249847347066E740F26B
:106BB00001439C4200F02882B4F5826F7FF43DAF20
:106BC000D9F80031980600F146821F4B1B681C065D
:106BD00040F194820024102304228DF800308DF8B7
:106BE00001308DF803408DF804408DF805408DF894
:106BF0000640BAE145F230239C4200F0838145F221
:106C000040239C427FF419AFB9F9A033CDF803308B
:106C10001021402252238DF802308DF80010D9F84F
:106C2000C4328DF80120684600249847347025E767
:106C30001F85EB510000C84218060020B82600202E
:106C400008530020C40B0010E4510020387F0020BE
:106C5000C5B3A2910130CA49C0B291F8892091F818
:106C60008830934220D0531CDBB25200D1F88440CC
:106C7000C449A45A89F88307B4F5C06F4B717FF4F7
:106C800083AED9F83434CDF8033010220024062323
:106C90008DF802308DF80020D9F8C4328DF801400B
:106CA00068469847347035E7002281F8892001232F
:106CB000DCE7B54A99F88437127881F881400133CE
:106CC000DBB20132934289F8843700F0B1810120B0
:106CD000C3E700283FF41DAE0378303B012B3FF69D
:106CE00018AE013009F281720621FFF781FC99F894
:106CF000813789F88207002B3FF40BAE347008E629
:106D0000A4F11100C0B2FEF785FF00283FF495AE54
:106D1000B0F90230CDF8033010238DF80030ADF813
:106D20000140D9F8C4326846984700233370002DDB
:106D30007FF4F4AD84E699F8EF24B9F83C34002AE6
:106D400040F0D08110220221CDF803308DF80020D0
:106D5000D9F8C4328DF801208DF80210684600245D
:106D6000984734708AE6601EC0B2FEF753FF0028D1
:106D70003FF463AE4368CDE7D9F82C348349D9F8A2
:106D8000C42281FB0301DB17C3EBA1030024102104
:106D9000CDF8033002238DF800108DF801408DF8F6
:106DA0000230684690473470002D7FF4B7AD47E657
:106DB00099F89B339A077FF540AEB9F89C33CDF82C
:106DC00003301021202204238DF802308DF80010AA
:106DD000D9F8C4328DF801206846002498473470F1
:106DE0004CE699F885370133DAB2042A00F06F8156
:106DF00042F2107389F8852703FB02F3D9F8E426E1
:106E0000002A00F02681023399F84C24D007B9F803
:106E1000182548BF0433D10748BF0A33940748BF39
:106E20001433D00548BF2833510748BF6433540694
:106E300048BF03F57A63102100240422CDF8033003
:106E40008DF800108DF801408FE0D9F85C34CDF852
:106E500003301022002401238DF802308DF8002029
:106E6000D9F8C4328DF8014068469847347051E62D
:106E700099F84734002B40F030811022092163E754
:106E800099F89B339B077FF5D8AD414AD9F8C432B6
:106E90009268CDF80320102220218DF800200822CE
:106EA0008DF801108DF80220684600249847347050
:106EB000002D7FF433ADC3E5FF20FEF7ABFE0028C5
:106EC0003FF4BBADB0F90C303249D9F8C422897E09
:106ED00003EB830303EB83031020490800249B008A
:106EE00093FBF1F305218DF80000CDF803308DF808
:106EF00001408DF80210684690473470002D7FF4F1
:106F00000DAD9DE5B9F9A233CDF803301021302243
:106F100052238DF802308DF80010D9F8C4328DF864
:106F200001206846002498473470A7E5A4F1710059
:106F3000C0B2FEF76FFE00283FF47FAD90F901303C
:106F4000E8E6114B93ED170AD3ED027A20EE270AFB
:106F5000002420EE080A46F0ADF91023CDF8030016
:106F600007228DF800308DF80130D9F8C4328DF841
:106F70000220684698473470002D7FF4CFAC5FE55F
:106F8000180600209C060020C40B00106766666689
:106F900008530020B826002099F89B2391077FF51D
:106FA0004CAD13F0010F814B00F0B5805A6882EAB6
:106FB000E273A3EBE27303EB5303A7FB0313DB08BA
:106FC000002AACBF43F0004343F0404310210024AB
:106FD000082233E7B9F9A433D9F8C42203EB8303B9
:106FE0005B001020CDF80330402108238DF800000D
:106FF0008DF801108DF802306846002490473470F7
:10700000002D7FF48BAC1BE5B9F9A835CDF8033022
:107010001021012204238DF802308DF80010D9F8D8
:10702000C4328DF80120684600249847347025E565
:1070300089F88447012010E65D490620FFF738FAF9
:10704000002389F88207337003B0BDEC028BBDE8E2
:10705000F0830133D8E6554A99F89B13538A643B71
:10706000C3EB4370C3EBC00388FB03401844DB173A
:10707000C3EB20230933092BA8BF092323EAE373B9
:1070800003EB830311F0020F03EB830314BF4FF4F0
:107090007A7000209B00C90748BF00F5FA60117D97
:1070A000D9F8C4229BB203440B44042010218DF86C
:1070B0000200CDF803308DF800108DF801106846FD
:1070C000002490473470002D7FF428ACB8E40123ED
:1070D00089F8853742F2107390E6B9F83C24B2FB88
:1070E000F3F3CAE699F84724002A57D1134629E654
:1070F000347003B0BDEC028BBDE8F08399F8EE3438
:10710000002B3FF49AAC99F88637032B49D8DFE877
:1071100003F03B3122111A6882EAE273A3EBE273B7
:1071200003EB5303A7FB0313DB08002AB8BF43F0AC
:1071300080434BE7D9F88827537A907AD17A03F1C4
:10714000407303EB0023002203EB014389F88627F9
:1071500010220421F8E5174A11688A7D087C897A93
:10716000120402EB00220A44591C89F8861702EB2C
:107170000363EDE70F4A11684A7DC87B497A120420
:1071800002EB00220A44EFE70A4A11680A7D887B75
:10719000097A120402EB00220A44E5E7B3FBF2F39A
:1071A000D0E55A1C89F886271B06D1E70853002032
:1071B000E91401088453002030B5A0F17D03012BB0
:1071C000044683B00D46104608D921462FF0F8FC3E
:1071D00015B1288804442C8003B030BD7D21019274
:1071E0002FF0EEFC019884F020012FF0E9FCEFE78E
:1071F00030B50F4B85B0D3F88C2700230446C51D4E
:10720000ADF80E3014F8010B01920DF10E01FFF7ED
:10721000D3FFA542019AF5D10DF10E0011F0AAF8A5
:10722000019A9DF80E000021FFF7C6FF05B030BDA2
:10723000387F0020044AD2F8903743F4DF2343F428
:107240008063C2F890377047387F0020013070B5F6
:10725000094EC4B203E040F0CBF8013448B9E5B2BE
:10726000152D21463046F6D9162D04BF034B93F851
:107270009457284670BD00BFC8860020387F002084
:1072800000B1D7E7044AD2F8903723F4DF2323F480
:107290008063C2F890377047387F002070B5114C7A
:1072A00084B00546D4F898070E4628F02BFC94F8D5
:1072B000E82494F8E934003A18BF01220BB142F0F7
:1072C0000802CDE9016200234FF4964195F90000D0
:1072D00000911A46082128F0A2FCC4F8980704B0CF
:1072E00070BD00BF387F002010B5064C03E0D4F815
:1072F00098072FF059FCD4F898072FF05DFC002870
:10730000F5D110BD387F002010B50D4CD4F89C3756
:107310001B791E3B012B0DD9D4F898070121383079
:10732000FFF7BCFF0023C4F8A03784F8A437BDE8FA
:107330001040D9E7D4F8980701212FF02DFCF1E790
:10734000387F002070B50A4E0546D6F8C8325E2058
:107350000C469847D6F8C83228469847E0B2FAF764
:10736000D9F8C4F30720BDE87040FAF7D3B800BFDE
:10737000387F002003682DE9F041002B3D4D3E4F42
:107380003E4EB8BF5B42A5FB0321890D07FB0137C9
:10739000C7EB0717BF0096F8EA3485FB0725FA17F5
:1073A0000446C2EBA555002B57D101EB810101EB3F
:1073B000810105EB810109B2DFF8BC801320FFF7E2
:1073C000C1FF2F4908FB057581FB0531ED17C5EBA2
:1073D000A11109B21B20FFF7B5FF2368254D002B33
:1073E000B4BF53214E212320FFF7ACFF636896F80A
:1073F000EA2483EAE376A6EBE376A5FB0631890D62
:1074000008FB0168C8EB08184FEA880885FB0835B7
:107410004FEAE873C3EBA5552ABB01EB810101EBF1
:10742000810105EB810109B21220FFF78BFF124B9E
:10743000134903FB058581FB0531ED17C5EBA11150
:1074400009B21A20FFF77EFF6368002BBDE8F04108
:10745000B4BF57214521222074E7C1EB011105EB90
:10746000810109B2A8E7C1EB011105EB810109B265
:10747000DAE700BF6BCA5F6B806967FF387F002067
:10748000D34D62100B2814D810B401EB4103094C02
:1074900001EB83032344184490F82835934205D028
:1074A0002144002380F8282581F81C355DF8044B21
:1074B00070477047387F0020F0B5464C94F8A537E8
:1074C000012B83B0054650D994F8A6074249434E94
:1074D00094F8A777421CA1FB02C1184406EB800078
:1074E00001F4FE7606EB9101521AD0F8746184F82B
:1074F000A6272FB1D4F8A81704F2AC7291420DD090
:107500006EB9374A0133A2FB031222F0010101EBED
:1075100052029B1A84F8A53703B0F0BD314E94F89F
:10752000C03793B9304B019348F2A501123B1522A5
:107530006F46A4F8C417009384F8C6272946384636
:10754000B04758B994F8A537DBE76F4638460FF0D7
:1075500073FD29463846B0470028F3D094F8C01789
:1075600059B138460FF0E2FCECE71C4A02EB83020B
:10757000D2F87461002EC4D0D1E7009E1B4A964217
:1075800014D9013A013E41F2210512F8013F81EA86
:107590000321082311F4004F85EA41000ABF490086
:1075A00081B289B2013BF5D19642EED1384637F02F
:1075B000B5FD0F49009D6D1A152DA8BF15252A464A
:1075C00001F1180048F07AF994F8A53784F8F157DA
:1075D00097E700BF387F0020CDCCCCCC2403060831
:1075E000ABAAAAAAC529010811870020FF8600209E
:1075F000FC86002070B50B4E054606F2F6713CF095
:1076000081FF2C686C6006F2F471641A402CA8BFEC
:1076100040242960224606F6340048F04FF986F8E7
:10762000744870BD387F002030B50C4B0C4AC3F84D
:10763000F42783B0C822014603F6340503F2F97437
:1076400083F8F82768463A22CDE9004537F01EFD59
:107650006846FFF7CFFF03B030BD00BF387F002082
:10766000C83E7BEA044BD3F8043530EA030314BF69
:1076700001200020704700BF387F0020CB4A38B57A
:107680000820002382F88930FFF7ECFF50B1D2F8D0
:1076900084304FF4806402204FF482611C8082F8B1
:1076A000890059804FF40020FFF7DCFF50B192F8B9
:1076B0008930D2F884105C1C40F2014082F8894085
:1076C00021F81300BA4991F8D532002B6AD191F80C
:1076D000D632002B40F041814FF40070FFF7C2FF1B
:1076E00050B192F88930D2F884005D1C4FF40464E4
:1076F00082F8895020F81340D1F80011880700F172
:10770000DD80490700F1B780AA4B1B681B066AD4CD
:1077100092F8893082F888304FF48030002382F864
:10772000893082F88130FFF79DFF30B1D36F01209F
:107730004FF4047182F8810019804FF40040FFF784
:1077400091FF48B192F88130D16F5C1C4FF400700A
:1077500082F8814021F813004FF40030FFF782FFD8
:1077600048B192F88130D16F5C1C4FF4A06082F870
:10777000814021F813004FF48020FFF773FF48B1D8
:1077800092F88130D16F5C1C4FF4376082F88140F1
:1077900021F8130092F8813082F88030002382F8BB
:1077A000813038BD0120FFF75DFF00288FD04FF4F6
:1077B0008030FFF757FF50B992F88930D2F8840033
:1077C0005D1C4FF4047482F8895020F8134092F83D
:1077D0008930D2F884005D1C4FF4116482F889501E
:1077E00020F8134073E74FF40050FFF73BFF50B110
:1077F00092F88930D2F884105C1C4FF4036082F850
:10780000894021F813004FF48050FFF72BFF78B127
:1078100092F88930D2F88400591C1D46C9B24FF441
:107820000064023320F8154082F8893020F81140B6
:107830004FF48040FFF716FF50B192F88930D2F82C
:1078400084105C1C4FF4846082F8894021F8130096
:107850004FF48060FFF706FF00283FF459AF92F81D
:107860008930D2F884105C1C4FF4026082F88940A1
:1078700021F813004CE74FF48060FFF7F3FE50B19E
:1078800092F88930D2F884105C1C4FF4807082F832
:10789000894021F813004FF40060FFF7E3FE002851
:1078A0003FF432AF92F88930D2F884105C1C4FF468
:1078B000887082F8894021F8130025E78020FFF7BF
